:100000000C9459370C948A370C948A370C948A379D
:100010000C948A370C948A370C948A370C948A375C
:100020000C948A370C948A370C948A370C948A374C
:100030000C948A370D94C1A70C948A370C948A3794
:100040000C948A370C94DCF10C948A370C948A3720
:100050000C948A370C948A370C94A3EE0D9477A7EE
:100060000C948A370D940B7F0D94017F0C948A3782
:100070000C948A370C948A370C948A370C948A37FC
:100080000D94024F0C948A370C948A370C948A375B
:100090000C948A370C948A370C948A370C948A37DC
:1000A0000C948A370C948A370D94D44E0C948A376A
:1000B0000C948A370C948A370C948A370C948A37BC
:1000C0000C948A370C948A370C948A370C948A37AC
:1000D0000C948A370C948A370C948A370C948A379C
:1000E0000C948A37084AD73B3BCE016E84BCBFFDD7
:1000F000C12F3D6C74319ABD56833DDA3D00C77FF8
:1001000011BED9E4BB4C3E916BAAAABE0000008090
:100110003F05A84CCDB2D44EB93836A9020C50B91F
:10012000918688083CA6AAAA2ABE000000803F0744
:10013000634236B79BD8A71A39685618AEBAAB5582
:100140008C1D3CB7CC5763BD6DEDFD753EF6177247
:1001500031BF000000803F08000000BE9224491219
:100160003EABAAAA2ABECDCCCC4C3E00000080BE3D
:10017000ABAAAAAA3E00000000BF000000803F001A
:1001800000000000084178D3BB4387D1133D190E0E
:100190003CC3BD4282AD2B3E68EC8276BED98FE176
:1001A000A93E4C80EFFFBE01C4FF7F3F000000006E
:1001B00000000C9447910C9463430C94FB9B0D94AA
:1001C00025B10D94834E0C94DE9B0C94409D0C94B1
:1001D00090C70D9463A20D945B7D0C948A910C944E
:1001E000EAA00D94F4A10C946DE00C940B9D0D9479
:1001F000BDA00C94B18D0C9481A30C942A960C9400
:10020000F7A40C9494920D9470500D9413A10C9437
:1002100036960C9454960C94BC8D0C9482C70D9415
:10022000EDA00C9499C70C94AAB00C94059B0C9467
:1002300057580C947B920C94A3370D94DCA00D942A
:1002400005A10C944BB00D94A57F0D94E9A00D94DD
:1002500008A20C94E2910C94ACCC0C944E960C94A5
:10026000A2C70C947E9D0C9499900C945A960C9471
:1002700023C80C9457B90D94C2A00C94BA460D949F
:100280003EA10C94BD370C949CC70C940C960D9415
:100290004B7D0C9419C20C94ACE00C94D5A70C9433
:1002A000319D0C94A0B40C94A5A70C94CBCD0C94C8
:1002B0009FC70D941A7C0D94D07A0D94DDA10D94F6
:1002C00001A10C94EF980C9409A90C940DAC0C941A
:1002D0001AA40C949EB00C94E9BD0C94BD960D9498
:1002E0009E4E0D94E3A00C94F0380C9493C70C949C
:1002F000D6370C946FDC0C94369D0C9499A70C9413
:100300008CD10C943B470C94F39B0C9449920C9425
:1003100020990C94ADD50C94F45C0C942BA90D94FD
:10032000227B0C9430960C94B5CE0D9418A20D94AB
:1003300059A20D94997F0C94E9580C94E7C70C943A
:10034000FB960C9438910C9418960C9497A00C94EE
:10035000ADA70C9432C80C94BF9D0D94BB7F0C9438
:100360003DB00C9465CA0C94F6370C943FB00C94D5
:100370007A9A0C94E1A90D9442800C9431B30C94B8
:1003800056C70C9448960C94FB8D0C9490DF0D94FA
:10039000F7A00C94F6460D94FEA10C940A9B0D94C4
:1003A00088A10C94E2A20D9496B10C9473CF0C9496
:1003B00030900D948EA10C944C440D94684E0C9486
:1003C00046A00C9450B00C9462920D9477A20C94B9
:1003D00052390C944FD70C94F19B0C94AD920D9420
:1003E00049500D94F3A00C9426BC0C94FD9D0C94E4
:1003F00039C40C94B1A70C9479390C940D920C94D7
:10040000BA370C9462900C94D4DF0D9436A20C94FD
:1004100095A70C94238E0D9429490C94EDDB0C9434
:10042000D05A0D946DA20C947FE00C94DADE0C94FB
:10043000EFDF0D94A17F0C9495440C9439C10C947A
:100440005F9D0C948DA70C9445B00C943B9D0C942F
:100450009DA70C94B3CB0C948C370C946FDF0D9448
:1004600078B10D946C7F0C94DE9D0D949D7F0C945F
:10047000A9C70C9488A00C9470DC0C941D8E0C946D
:10048000AC900C94C3DD0D94917F0C945F430C945D
:100490001F910C948E8D0C94BAA70C94ACC70C943D
:1004A000A7C70C9415920D94957F0C94009C0C9406
:1004B0004DB00C9432AA0C94B7A70D9477A10C946C
:1004C0003C960D94E0A00C94B8920D94A3A10D94C9
:1004D000437F0C94A9A70C94A3C30C94DA900C94BA
:1004E00047B00C9449900C947F930D94283E0D9442
:1004F00009A10C943BAA0D94D77A0C9413A90C94DF
:1005000089A70C94B1B50C948DC70D944FA20C948F
:10051000BF900D942CA20D94C37F0C94F3900C9477
:1005200023AA0C9476E10D9445A20D94B07F0C940F
:1005300061D30D9491800C9423A20C94109B0C9485
:1005400042960C94F59B0D947B7F0C94D9910C945E
:10055000F1B00D9423A10C94F7DE0C94A1A70C9498
:1005600071900C9424960C9412960C9443B00D94B4
:1005700022A20C9424940C945A910D94EAA10C9408
:10058000048E0C9441B00C9491A70D94A97F0C9407
:10059000F3A00D940FA10C940ABB0C9456990C94E3
:1005A000C7380D94D4A00D94B94E0C9467430C94A5
:1005B00073910D94547D0C9449B00C9450A00C94FC
:1005C0004BA00C948A900D94FBA00C94A7A90C94BA
:1005D000EE910C942C9D0C945B9B0C9406910D94C5
:1005E0006F800D94D8A00C9480B70C945BDE0C94B3
:1005F000B4A70D9410A20D94E5A10D943A400D946A
:100600008A7F0C9496C70D9498A10D947CA10C94AC
:10061000009B0C9418A20C941E960C940CAF0C9496
:1006200084B84E414E494E495459494E46CDCCCCE2
:100630003D0AD7233C17B7D13877CC2B329595E6B6
:10064000241FB14F0A000020410000C84200401C96
:100650004620BCBE4CCA1B0E5AAEC59D7400407AE3
:1006600010F35A00A0724E18090010A5D4E800003B
:10067000E87648170000E40B54020000CA9A3B00D9
:100680000000E1F505000080969800000040420F50
:10069000000000A08601000000102700000000E814
:1006A00003000000006400000000000A00000000D9
:1006B000000100000000002C76D888DC674F08237A
:1006C000DFC1DFAE59E1B1B796E5E3E453C63AE6E0
:1006D00051997696E8E6C28426EB898C9B62ED40C0
:1006E0007C6FFCEFBC9C9F40F2BAA56FA5F490050F
:1006F0005A2AF75C936B6CF9676DC11BFCE0E40D43
:1007000047FEF520E6B500D0ED902E030094357736
:10071000050080841E080000204E0A000000C80C5E
:10072000333333330F986E12831141EF8D211489C7
:100730003BE65516CFFEE6DB18D1844B381BF77C21
:100740001D901DA4BBE424203284725E228100C966
:10075000F124ECA1E53D27434F4D4D554E49434112
:1007600054494F4E0044525952554E004552524F33
:10077000525300494E464F004543484F00473236DA
:100780002048656174696E67204E6F7A7A6C6500E7
:100790004732362048656174696E6720426564009F
:1007A00057616974696E6720666F7220686561744D
:1007B00075702E0A004669786564204C656E677412
:1007C00068205072696D6500446F6E6520507269D3
:1007D0006D696E67004D616E75616C207072696D38
:1007E000696E672E2E2E004C656176696E67204714
:1007F0003236003F53706563696669656420582C22
:100800005920636F6F7264696E617465206F7574CF
:10081000206F6620626F756E64732E0A003F285247
:100820002965706561742076616C7565206E6F74E2
:1008300020706C61757369626C653B206D757374B3
:10084000206265206174206C6561737420312E0A0A
:10085000003F537065636966696564206E6F7A7ADC
:100860006C652074656D7065726174757265206E5B
:100870006F7420706C61757369626C652E0A003F3D
:100880005370656369666965642066696C616D654E
:100890006E742073697A65206E6F7420706C617558
:1008A0007369626C652E0A003F53706563696669FF
:1008B0006564207072696D65206C656E6774682070
:1008C0006E6F7420706C61757369626C652E0A00BE
:1008D0003F537065636966696564206E6F7A7A6CF0
:1008E000652073697A65206E6F7420706C61757312
:1008F00069626C652E0A003F5265747261637469A7
:100900006F6E204D756C7469706C696572206D75C1
:100910007374206265207370656369666965642E0F
:100920000A003F53706563696669656420526574A7
:1009300072616374696F6E204D756C7469706C6957
:100940006572206E6F7420706C61757369626C657E
:100950002E0A003F537065636966696564206C61A7
:1009600079657220686569676874206E6F7420709D
:100970006C61757369626C652E0A0043292E0A004A
:100980003F537065636966696564206265642074BD
:10099000656D7065726174757265206E6F7420701C
:1009A0006C61757369626C65202834302D004732A4
:1009B00036207374617274696E672E2E2E0A004F92
:1009C00046460A0046616465204865696768742088
:1009D00000426564204C6576656C696E6720004650
:1009E00061696C656420746F20656E61626C65205E
:1009F000426564204C6576656C696E670A00496ED5
:100A000076616C6964206D6573682E0A0076616C8E
:100A100069640A53746F7261676520736C6F743A0E
:100A20002000696E004D65736820697320003F5592
:100A30007365203020746F20003F496E76616C69C9
:100A4000642073746F7261676520736C6F742E0A13
:100A5000003F454550524F4D2073746F726167657A
:100A6000206E6F7420617661696C61626C652E0A1C
:100A7000004D65736820706F696E74206F75742007
:100A80006F662072616E67650A004D3432312069ED
:100A90006E636F727265637420706172616D6574EC
:100AA00065722075736167650A00446576696174D3
:100AB000696F6E0025533A2025730046696E69738D
:100AC000686564210A003A207A3A2000206F662087
:100AD00000476F696E6720746F3A20580043570AC9
:100AE00000206469723A0020616E676C653A0053B9
:100AF00074617274207261646975733A004D3438A0
:100B000020506F696E740025533A2025642F2564A8
:100B100000506F736974696F6E696E6720746865E1
:100B20002070726F62652E2E2E0A003F4C6567732F
:100B3000206F66206D6F76656D656E7420696D70CF
:100B40006C61757369626C652028302D3135292EF2
:100B50000A003F2028582C5929206F7574206F6691
:100B600020626F756E64732E0A0050726F6265208A
:100B70006F7574206F6620626F756E6473003F53EB
:100B8000616D706C652073697A65206E6F7420707A
:100B90006C61757369626C652028342D3530292E9F
:100BA0000A004D3438205A2D50726F62652052650C
:100BB000706561746162696C6974792054657374DD
:100BC0000A003F2856296572626F7365206C65764E
:100BD000656C20696D706C61757369626C65202845
:100BE000302D34292E0A005374616E6461726420C2
:100BF000446576696174696F6E3A20002052616EB7
:100C000067653A2000204D61783A2000204D696EDA
:100C10003A2000205369676D613A20004D65616E8E
:100C20003A20005741524E494E4721204C6F7720C1
:100C30005A204A65726B206D6179206C6561642071
:100C4000746F20756E77616E746564207061757362
:100C500065732E0A0020204D61783A200020002084
:100C6000204D696E3A2000536F667420656E647380
:100C7000746F70733A20004D32342053256C642019
:100C800054256C64004739322E39204525730047BE
:100C90003120462564004739322E39205A25730009
:100CA0004731205A30204632303000473120582515
:100CB0007320592573204633303030004D343230A4
:100CC00020532569205A2573004D31303620502598
:100CD0006920532569004D32303020442573004788
:100CE000323852305859004739322E392045302099
:100CF0005A300A47315A2573004D31303920532577
:100D000069004D31393020532569004D343230208F
:100D10005330205A300020496E76616C696420653A
:100D200078747275646572200047322F47332062F1
:100D3000616420706172616D65746572730A00533D
:100D40006C6565702E2E2E005A2050726F626520E1
:100D500050617374204265640A005A2050726F62B9
:100D60006520506173742042656400205A3A200067
:100D700020593A200042656420583A20004D65739E
:100D80006820706F696E74206F7574206F662072B2
:100D9000616E67650A004D302053746F70004D31ED
:100DA0002053746F7000436C69636B20746F205222
:100DB0006573756D652E2E2E004E6F204D6F766516
:100DC0002E00456E642066696C65206C6973740A38
:100DD00000426567696E2066696C65206C69737492
:100DE0000A004E6F206D656469610A005265737573
:100DF0006D696E6720534400286E6F2066696C65CC
:100E0000290043757272656E742066696C653A20BC
:100E1000005072696E742074696D653A20000A533F
:100E2000746174733A2046696C616D656E742075E7
:100E30007365643A20002C204C6F6E6765737420D4
:100E40006A6F623A2000546F74616C2074696D653A
:100E50003A200053746174733A20002C2046616973
:100E60006C65643A20002C2046696E69736865647D
:100E70003A20005072696E74733A200053746174A2
:100E8000733A2000436F6F6C696E672E2E2E0048F8
:100E9000656174696E672E2E2E0045202553006F04
:100EA0006B006F666600780773076C076507570766
:100EB00044454255473A004D313133205300426595
:100EC0006420436F6F6C696E672E2E2E004265643E
:100ED0002048656174696E672E2E2E00537550652B
:100EE000522043522D3230204F46462E002F2F00E5
:100EF0004D31343520533C696E6465783E206F7502
:100F000074206F662072616E67652028302D31294C
:100F10000A00205200416363656C65726174696FF9
:100F20006E3A2050004D32303620580046523A007A
:100F300020466C6F773A20003A2000205365727685
:100F40006F2000206F7574206F662072616E676578
:100F50000A00536572766F200020643A0020693AD7
:100F60000020703A00496E76616C6964206578747F
:100F700072756465720A0020643A0020693A0020A4
:100F8000703A004C434420436F6E74726173743A3C
:100F9000200064697300656E0043290A0061626C79
:100FA000656420286D696E2074656D702000436F44
:100FB0006C64206578747275646573206172652055
:100FC000004F666673657473204170706C69656468
:100FD000004572723A20546F6F206661722100548E
:100FE0006F6F206661722066726F6D207265666534
:100FF00072656E636520706F696E740A00454550B6
:10100000524F4D204F4B0A002E0A002028302D3120
:101010003029002076616C7565206F7574206F66CD
:101020002072616E676500416476616E6365204B76
:101030003D004F4646004F4E00506F7765722D6C55
:101040006F7373207265636F7665727920004D3817
:101050003400446F6E65207072696E74696E67202B
:1010600066696C650A004D3737004D3331004361C6
:10107000703A004D4541545041434B00434F4F4C53
:1010800045525F54454D50455241545552450043D9
:1010900048414D4245525F54454D5045524154558B
:1010A000524500424142595354455050494E470021
:1010B00041524353004D4F54494F4E5F4D4F4445AD
:1010C0005300544845524D414C5F50524F54454394
:1010D00054494F4E004C4F4E475F46494C454E4198
:1010E0004D45004155544F5245504F52545F534463
:1010F0005F5354415455530053445F57524954452C
:10110000005245504541540053444341524400501D
:10111000524F4D50545F535550504F525400454D0F
:10112000455247454E43595F504152534552004343
:101130004153455F4C494748545F425249474854E0
:101140004E45535300544F47474C455F4C49474821
:10115000545300534F4654574152455F504F5745E3
:1011600052004255494C445F50455243454E54004D
:101170004C4556454C494E475F44415441005A5FE7
:1011800050524F42450052554E4F55540041555410
:101190004F4C4556454C005052494E545F4A4F42C1
:1011A0000050524F4752455353004155544F5245FA
:1011B000504F52545F54454D5000564F4C554D457D
:1011C0005452494300454550524F4D0042494E410B
:1011D00052595F46494C455F5452414E5346455221
:1011E0000053455249414C5F584F4E5F584F464659
:1011F000004649524D574152455F4E414D453A4D8B
:1012000061726C696E20322E302E375F4457372E54
:101210003320544D33442032534D4442552028410D
:10122000707220323420323032312032313A303153
:101230003A30362920534F555243455F434F44457A
:101240005F55524C3A68747470733A2F2F67697403
:101250006875622E636F6D2F496E73616E69747964
:101260004175746F6D6174696F6E2F4D61726C6939
:101270006E2F747265652F437265616C6974794471
:1012800077696E5F322E302050524F544F434F4C8F
:101290005F56455253494F4E3A312E30204D41430F
:1012A00048494E455F545950453A53755065522050
:1012B00043522D32302045585452554445525F43D5
:1012C0004F554E543A3120555549443A636564654B
:1012D000326132662D343161322D343734382D3954
:1012E0006231322D633535633632663336376666A2
:1012F0000A0050726F6265204F6666736574205AEB
:101300000050726F6265204F6666736574205A00E4
:10131000290A0020746F20003F5A206F7574206FD7
:10132000662072616E6765202800290A0020746FAC
:1013300020003F59206F7574206F662072616E67C0
:101340006520282D00290A0020746F20003F5820B6
:101350006F7574206F662072616E676520282D009E
:1013600050726F6265204F66667365742058004343
:10137000616E6E6F74206F70656E20737562646944
:101380007220002569730025696D20256973002589
:1013900069682025696D2025697300256964202509
:1013A00069682025696D20256973002569792025E4
:1013B0006964202569682025696D202569730023EB
:1013C000646566696E652044454641554C545F002E
:1013D000626564004B6420004B6920004B70200064
:1013E000504944204175746F74756E652066696E4E
:1013F0006973686564212050757420746865206C79
:10140000617374204B702C204B6920616E64204BFB
:101410006420636F6E7374616E74732066726F6D97
:101420002062656C6F7720696E746F20436F6E6603
:10143000696775726174696F6E2E680A005049445D
:10144000204175746F74756E65206661696C6564A2
:10145000212074696D656F75740A005049442041FC
:1014600075746F74756E65206661696C65642120A2
:1014700054656D706572617475726520746F6F204C
:10148000686967680A00204B643A2000204B693A7B
:101490002000204B703A200020436C617373696315
:1014A00020504944200A00204E6F206F76657273E9
:1014B000686F6F740A002054753A2000204B753A0B
:1014C0002000206D61783A2000206D696E3A20007E
:1014D00020643A200020626961733A200050494438
:1014E000204175746F74756E652073746172740A2F
:1014F00000504944204175746F74756E65206661B3
:10150000696C6564212054656D70657261747572D3
:101510006520746F6F20686967680A00504944202D
:101520004175746F74756E6500504944204175743F
:101530006F74756E65206661696C65642120426117
:1015400064206865617465722069640A004572727E
:101550003A207574663820666F6E74206E6F742042
:10156000696E697469616C697A65642E004572728E
:101570003A207574663820666F6E74206E6F742022
:10158000696E697469616C697A65642E004572726E
:101590003A207574663820666F6E74206E6F742002
:1015A000696E697469616C697A65642E0000FE0079
:1015B00003FF8007C7C00701E00000E00000F00063
:1015C00000700400700E00701F00703F80F00E006D
:1015D000E00F01E007C7C003FF8000FE0000FE002F
:1015E00003FF8007C7C00F01E00E00E03F80F01F3F
:1015F00000700E00700400700000700000F0000029
:10160000E00701E007C7C003FF8000FE000E000EE8
:10161000000E000E000E000E000E000E007FC03FF8
:10162000801F000E00040004000E001F003F807F9A
:10163000C00E000E000E000E000E000E000E000E7A
:1016400000FFFFFF7F80FFC0FFC0FFC07F807F8063
:10165000FFC0FFC0FFC03F001E000C00FFE0FFD135
:1016600040A0C8A6A22FF80023AC00AF10FFFEFFD9
:1016700005FFD0FFE0FFC1FFD1E240A0C8A6A22F26
:10168000F800238127AC00AFFFD0FF64FFD1A5FF96
:10169000D0FF64FF64FFD1A4FFD0FF16FFFE4265B8
:1016A0006400456E636C6F73757265002568753AEA
:1016B00025303268750025303268753A2530326839
:1016C0007500202020202020200020202020001F26
:1016D000E0201020102010102010202010201030AA
:1016E000300840048003001FE03FF03FF03FF01F50
:1016F000E01FE03FF03FF03FF00FC0078003003FE6
:10170000FFF038007030FC3020FC102078102030C2
:10171000102C00D02E31D02F7BD02F7BD02E31D06B
:101720002C00D020301020781020FC1030FC3038F5
:1017300000703FFFF03FFFF03800703186302387A4
:10174000102787902F87D02F03D0203010207810BB
:101750002078102030102F03D02F87D02787902398
:1017600087103186303800703FFFF01FFFF81FFFF1
:10177000F8041040020820020820041040082080CD
:101780001041001041000820800410400000001F9C
:10179000FFF81FFFF8FFFFFF8000018E00E19F01AF
:1017A000F19381399F81F99F81F99FB9F98F28F1D0
:1017B0008038018000019FFFF99174999B06A99BD5
:1017C00054A99B56A99B54999FFFF9FFFFFF53759E
:1017D0005065522043522D32302052656164792E7B
:1017E000005072696E74696E672E2E2E006E6F74D3
:1017F000696669636174696F6E200063616E636519
:101800006C005072696E742041626F72746564007E
:101810004469736D6973730055492041626F727436
:101820006564004D323520500A4D323400507269E3
:101830006E742050617573656400526573756D65D3
:101840000055492050617573650050617573696E6C
:10185000672E2E2E00726573756D65004D32340053
:1018600050726F6265205A204F6666736574004C33
:101870006F6164206D6D00556E6C6F6164206D6DDD
:101880000046696C2E204469612E004520696E2057
:101890006D6D5E3300416476616E6365204B004D73
:1018A0003330332055312045256920532569000008
:1018B0000C0F00FE07022503BB017FFE08FE08FE99
:1018C00005080806000040F0C888889878100508C8
:1018D00008060000C0F88888888888F8050505068D
:1018E00000012030F830200508080600002070F8BC
:1018F00020202020E00509090600FF2070A8A8B8D4
:1019000088887020070505070001D86C366CD8055B
:1019100009090600FFF8A88888888888A8F8050AB9
:101920000A0600FE205050505088A8A88870030373
:101930000306000340A040FFFFFFFFFFFFFFFFFF84
:10194000FFFFFFFFFFFFFFFFFFFFFFFFFF000000A4
:101950000605FF0107070602008080808080008066
:10196000030303060105A0A0A0050606060000501B
:10197000F85050F8500509090600FF2070A8A07023
:1019800028A87020050707060000C8C81020409846
:101990009805070706000040A0A040A89068010332
:1019A000030602058080800309090601FF204040EC
:1019B0008080804040200309090601FF80404020CC
:1019C000202040408005070706000020A8702070F6
:1019D000A8200505050600012020F82020020303A9
:1019E0000601FFC04080050101060003F802020263
:1019F000060100C0C00507070600000810102040BF
:101A00004080050707060000708898A8C888700302
:101A1000070706010040C040404040E005070706B8
:101A20000000708808102040F8050707060000F83D
:101A30000810300888700507070600001030509025
:101A4000F81010050707060000F880F008088870F5
:101A5000050707060000304080F0888870050707FA
:101A6000060000F8081010202020050707060000D7
:101A7000708888708888700507070600007088885D
:101A800078081060020505060100C0C000C0C00251
:101A900006060601FFC0C000C04080030505060120
:101AA000012040804020050303060002F800F803EF
:101AB000050506010180402040800507070600005B
:101AC000708810202000200507070600007088B8E5
:101AD000A8B88070050707060000708888F8888815
:101AE00088050707060000F04848704848F00507D9
:101AF0000706000070888080808870050707060050
:101B000000F04848484848F0050707060000F880FC
:101B100080F08080F8050707060000F88080F080DC
:101B2000808005070706000070888080988870050F
:101B30000707060000888888F88888880307070652
:101B40000100E04040404040E00507070600003843
:101B50001010101090600507070600008890A0C0C4
:101B6000A09088050707060000808080808080F8AC
:101B700005070706000088D8A88888888805070711
:101B80000600008888C8A89888880507070600000E
:101B900070888888888870050707060000F08888A4
:101BA000F080808005070706000070888888A8906C
:101BB00068050707060000F08888F0A090880507F0
:101BC0000706000070888070088870050707060007
:101BD00000F8202020202020050707060000888824
:101BE00088888888700507070600008888888850DC
:101BF000502005070706000088888888A8A8500597
:101C000007070600008888502050888805070706C7
:101C1000000088885020202020050707060000F8D3
:101C20000810204080F80309090601FFE080808049
:101C300080808080E005070706000080404020107B
:101C400010080309090601FFE020202020202020A1
:101C5000E00503030600052050880501010600FE8B
:101C6000F803030306010580402005050506000072
:101C700070087888780507070600008080F088885B
:101C800088F005050506000070808088700507074C
:101C90000600000808788888887805050506000091
:101CA0007088F08070050707060000304840E0406B
:101CB00040400507070600FE708888887808700590
:101CC00007070600008080F08888888803070706D9
:101CD00001004000C0404040E00409090601FE1038
:101CE000003010101010906005070706000080807B
:101CF0008890E09088030707060100C040404040FC
:101D000040E0050505060000D0A8A8A8A80505051F
:101D1000060000B0C88888880505050600007088A0
:101D20008888700507070600FEF0888888F08080A4
:101D30000507070600FE78888888780808050505E5
:101D4000060000B0C8808080050505060000788088
:101D50007008F00507070600002020F82020201852
:101D600005050506000088888898680505050600B1
:101D70000088888850200505050600008888A8A8E6
:101D80005005050506000088502050880507070605
:101D900000FE88888850204080050505060000F870
:101DA000102040F80309090601FF20404040804010
:101DB0004040200109090602FF80808080808080E9
:101DC00080800309090601FF8040404020404040D8
:101DD0008005030306000248A890FF554E4C4F4172
:101DE000442046494C414D454E54004C4F414420FF
:101DF00046494C414D454E540046494C414D454E97
:101E000054204348414E4745005049442041757491
:101E10006F74756E65202A005049442D44202A00B5
:101E20005049442D49202A005049442D50202A0071
:101E300020082046616374002008204D617800204E
:101E400008204D696E004F6666004F6E0041757444
:101E50006F74656D70005654726176204D696E0026
:101E6000566D696E00566D6178204500566D61783B
:101E7000205A00566D6178205900566D61782058BF
:101E800000416D6178204500416D6178205A004124
:101E90006D6178205900416D6178205800412D54C2
:101EA000726176656C00412D5265747261637400D5
:101EB000416363656C0056652D4A65726B00565A26
:101EC0002D4A65726B0056592D4A65726B00565843
:101ED0002D4A65726B0050726F6265205A204F6602
:101EE000667365740050726F62652059204F666694
:101EF0007365740050726F62652058204F66667378
:101F0000657400452073746570732F6D6D005A20E1
:101F100053746570732F6D6D005920537465707321
:101F20002F6D6D00582053746570732F6D6D0041D7
:101F30006476616E6365642053657474696E67735B
:101F4000003F0043616E63656C00496E6974004D2B
:101F500034323800496E697469616C697A6520456C
:101F60004550524F4D0046696C616D656E7400546A
:101F7000656D706572617475726500537465707318
:101F80002F6D6D0050726F6265204F6666736574C9
:101F900073004A65726B00416363656C65726174BE
:101FA000696F6E0056656C6F636974790053657470
:101FB00020486F6D65204F66667365747300436FCC
:101FC0006E66696775726174696F6E003F004E6579
:101FD000787420506F696E7400446F6E65004E65B2
:101FE0007874003F0043616E63656C204F626A65E0
:101FF0006374004E4F005945530043616E63656C36
:10200000204F626A656374203D004D61696E005324
:10201000746F770053572D4D6F6465004465706C85
:102020006F790053656C662D546573740052657347
:10203000657400426564004E6F7A7A6C6500466193
:102040006E20537065656400436F6E6669677572D4
:102050006174696F6E004C6F6164205365747469BC
:102060006E67730053746F72652053657474696E84
:10207000677300526573746F72652044656661759D
:102080006C74730050726568656174202420436F1E
:102090006E66004F6666004F6E00506F7765722067
:1020A0004F7574616765004C434420436F6E7472D2
:1020B00061737400424C546F7563680050726F62B4
:1020C00065205A204F666673657400416476616EC0
:1020D0006365642053657474696E6773004D61694C
:1020E0006E004D37303220542564004D363030209C
:1020F000423020542564004D373032203B256400A7
:102100004D37303120542564004D373032004D3783
:102110003031004D363030204230004D61696E0064
:10212000436F6E74696E7565005075726765206DDA
:102130006F726500524553554D45204F5054494FDD
:102140004E533A005052494E542050415553454445
:102150000020204E6F7A7A6C653A20005061726BD5
:10216000696E672E2E2E0000005761697420666F1D
:10217000720066696C616D656E74206368616E677C
:102180006500746F20737461727400576169742004
:10219000666F720066696C616D656E7420756E6C39
:1021A0006F616400004E6F7A7A6C652068656174B7
:1021B000696E6700506C6561736520776169742E84
:1021C0002E2E0000507265737320627574746F6EEA
:1021D00000746F2068656174206E6F7A7A6C650098
:1021E00000496E736572742066696C616D656E740A
:1021F00000616E6420707265737320627574746F11
:102200006E00746F20636F6E74696E756500576140
:10221000697420666F720066696C616D656E74200A
:102220006C6F616400005072657373204275747442
:102230006F6E00746F20726573756D6520707269C2
:102240006E7400005761697420666F722070726945
:102250006E7400746F20726573756D652E2E2E007E
:10226000005761697420666F720066696C616D6504
:102270006E7420707572676500003E2000256C64E6
:102280002E25696D00457874727564656420546FFD
:1022900074616C003E20004C6F6E67657374204A59
:1022A0006F622054696D65003E2000546F74616C4C
:1022B000205072696E742054696D6500436F6D70B3
:1022C0006C65746564003A20005072696E74204336
:1022D0006F756E74003A200031353000350042458C
:1022E000443A204154432031303447542D32005277
:1022F000756E617761792057617463683A204F4E3B
:10230000004D61782054656D7000343530004D69A2
:102310006E2054656D7000350045313A20536C696C
:102320006365456E6720343530C2B0430050535565
:102330000047656E657269630050726F746F636FFA
:102340006C00312E3000426175640032353030301F
:102350003000437265616C69747933442052414D99
:10236000505300556E696669656420426564204C6F
:102370006576656C696E6700457874727564657220
:102380007300310074696E796D616368696E65739D
:1023900033642E636F6D0053755065522043522D88
:1023A000323000323032312D30342D313800322E7F
:1023B000302E375F4457372E33004D61726C696E93
:1023C000005072696E7465722053746174730054A6
:1023D0006865726D6973746F727300426F617264C5
:1023E00020496E666F005072696E74657220496E86
:1023F000666F004D61696E004D31303030005374AE
:102400006F70205072696E7400526573756D65202F
:102410005072696E7400506F776572204F757461E9
:102420006765004D3139305335350A4732380A4730
:10243000323950310A47323950330A473239533131
:102440000A47323953300A47323946302E300A476C
:102450003239410A4D313034533231350A4732383E
:102460000A4D313039533231350A47315831353020
:102470005931353046353030300A47315A300A4DFF
:102480003530300A4D3430300A4D31313720536504
:1024900074205A204F6666736574004D3130365390
:1024A0003132380A4D3330334338533231354530C9
:1024B000550A4D3530300A4D3131372050494420CE
:1024C00054756E6520446F6E65004D31393053355B
:1024D000350A4D313034533231350A4732380A47E4
:1024E00032394C310A47312058313030593130308F
:1024F00046353030300A47315A30004D3530300AD9
:102500004D3131372053657474696E67732053748D
:102510006F726564005072657020666F72205A2079
:1025200041646A757374005049442054756E6500A7
:1025300053746F72652053657474696E67730053CA
:1025400065747570004D61696E003F004261636B98
:102550000053746F70005072696E742066726F6DF4
:10256000204D65646961004368616E6765204D6553
:10257000646961004D32310041626F7574205072A0
:10258000696E746572004368616E67652046696CA8
:10259000616D656E74004C6576656C696E6720547C
:1025A0006F6F6C7300436F6E6669677572617469F3
:1025B0006F6E0054656D7065726174757265004D63
:1025C0006F74696F6E00486F737420537461727416
:1025D00000526573756D65205072696E74004361B9
:1025E0006E63656C204F626A6563740054756E6536
:1025F0000053746F70205072696E7400506175736F
:1026000065205072696E74004E6F204D656469617B
:1026100000496E666F2053637265656E003F00531C
:1026200074617274205072696E740043616E6365E8
:102630006C005072696E740043616E6E6F74206539
:102640006E746572207375626469723A2000022E9E
:102650002E004D61696E002100486F74656E642024
:10266000746F6F20636F6C64004261636B00507223
:102670006F63656564004F6666004F6E00536F665A
:102680007420456E6473746F7073004D6F74696F5E
:102690006E0044697361626C652053746570706587
:1026A0007273004D3834004D34382050726F6265BB
:1026B0002054657374004732384F0A4D3438205027
:1026C0003130004C6576656C20436F726E657273B5
:1026D00000556E696669656420426564204C6576C4
:1026E000656C696E6700486F6D65205A0047323827
:1026F0005A00486F6D652059004732385900486FBD
:102700006D6520580047323858004175746F204875
:102710006F6D65004D61696E00507265686561742A
:10272000202420456E640050726568656174202421
:10273000204265640054656D7065726174757265E0
:1027400000436F6F6C646F776E00507265686561EF
:102750007420240046616E205370656564207E00FD
:10276000426564004E6F7A7A6C65004D61696E0057
:1027700050726F6265205A204F666673657400411F
:102780006476616E6365204B00466C6F770046612E
:102790006E205370656564207E00426564004E6F54
:1027A0007A7A6C65005370656564004D61696E00EE
:1027B0005A2056616C7565004732380A4D31393000
:1027C000205325690A4D313039205325690A473293
:1027D00039205031004265642054656D7000486FA7
:1027E00074656E642054656D70002E256900473253
:1027F000395036432D0048656967687420416D6F14
:10280000756E740041646A757374204D6573682039
:102810004865696768740046696E652054756E6521
:1028200020436C6F73657374004732395034540021
:1028300046696E652054756E6520416C6C004732A8
:102840003950345239393954004732380A47323610
:1028500043504825694225690056616C696461747A
:102860006520437573746F6D204D65736800473242
:10287000380A473236435049310056616C69646109
:102880007465204D65736820282429004732380A72
:1028900047323643504930004732394A2569004CA7
:1028A0006576656C204D65736800536964652050DA
:1028B0006F696E74730047726964204D6573682098
:1028C0004C6576656C696E6700332D506F696E7468
:1028D000204C6576656C696E67004732394A300076
:1028E000473239503352432E2569004D616E756170
:1028F0006C2046696C6C2D696E004732395032424B
:10290000543000536D6172742046696C6C2D696E91
:1029100000473239503354300046696C6C2D696E73
:1029200020416D6F756E74004D65736820696E7619
:10293000616C6964617465642E0A00496E666F207B
:1029400053637265656E00496E76616C696461748B
:102950006520436C6F7365737400473239490049D1
:102960006E76616C696461746520416C6C00436FC4
:102970006E74696E756520426564204D65736800EC
:102980004732395031430046696C6C2D696E204DD9
:10299000657368004275696C6420436F6C64204DF8
:1029A000657368004732394E5031004275696C6476
:1029B00020437573746F6D204D657368004732381E
:1029C0000A4D31393049310A4D31303949310A47E0
:1029D000323950310A4D31303453300A4D313430B0
:1029E0005330004275696C64204D6573682028245B
:1029F00029004732380A4D31393049300A4D3130DB
:102A00003949300A47323950310A4D313034533068
:102A10000A4D313430533000473239256325690A75
:102A20004D31313720004D657368202569204C6F8A
:102A300061646564004D6573682025692053617683
:102A40006564005361766520426564204D65736856
:102A5000004C6F616420426564204D657368004DD1
:102A6000656D6F727920536C6F74004E6F205374D4
:102A70006F726167650047323950345825735925A4
:102A80007352256900202D2D2D2D2D005A3A005905
:102A90003A00486F6D696E672058595A00473238BE
:102AA000004F6666205072696E74657220426163E1
:102AB0006B757000473239532D31004F7574707546
:102AC0007420666F722043535600473239543100E8
:102AD0004F757470757420666F7220486F73740040
:102AE0004732395430004D657368204C6576656C0B
:102AF000696E670045646974204D657368005661AE
:102B00006C6964617465204D657368004D616E7514
:102B1000616C6C79204275696C64204D6573680046
:102B2000473239493939390A4732395032425430FB
:102B3000004275696C64204D65736800372E205320
:102B400061766520426564204D65736800362E20ED
:102B500046696E652054756E6520416C6C00473285
:102B6000395034523939395400352E2056616C6948
:102B700064617465204D65736800342E2046696E6B
:102B8000652054756E6520416C6C004732395034B5
:102B9000523939395400332E2056616C696461749E
:102BA00065204D65736800322E20536D617274206C
:102BB00046696C6C2D696E004732395033543000D1
:102BC000312E204275696C6420436F6C64204D6522
:102BD0007368004732394E503100556E6966696539
:102BE0006420426564204C6576656C696E670046BA
:102BF00061646520486569676874004F7574707515
:102C0000742055424C20496E666F00473239570098
:102C100055424C20546F6F6C73004F75747075740F
:102C2000204D657368204D6170004D6573682053B9
:102C3000746F72616765004D6573682045646974DF
:102C400000537465702D42792D5374657020554280
:102C50004C0041637469766174652055424C0047AD
:102C60003239410044656163746976617465205549
:102C7000424C0047323944004D6F74696F6E004812
:102C80006F6D696E67204661696C6564006F706581
:102C90006E00545249474745524544003A20007A55
:102CA0005F6D696E00795F6D696E00785F6D696E4A
:102CB000005265706F7274696E6720656E6473741C
:102CC0006F70207374617475730A0020746F6F20C5
:102CD0006C6F6E6720657874727573696F6E2070A3
:102CE000726576656E7465640A0020636F6C64209B
:102CF000657874727573696F6E2070726576656E33
:102D00007465640A00486F6D65202573257325730B
:102D1000204669727374005761726E696E673A205B
:102D2000486F6D696E672042756D702044697669E1
:102D3000736F72203C20310A000202040000000080
:102D4000000000000000000000007043000070431D
:102D500000007A43000000410000004100000040F4
:102D6000FFFFFF000000010000000100008000558F
:102D70005555000000400033333300AAAA2A004909
:102D800092240000002000C7711C0099991900D1FD
:102D9000451700555515003BB11300244912001189
:102DA000111100000010000F0F0F00E3380E004358
:102DB000790D00CCCC0C00C3300C00E8A20B0064F1
:102DC000210B00AAAA0A00703D0A009DD809004202
:102DD0007B090092240900DCD308008888080010D1
:102DE00042080000000800F0C1070087870700754F
:102DF000500700711C07003EEB0600A1BC060069ED
:102E000090060066660600703E0600611806001710
:102E1000F4050074D105005BB00500B290050062B6
:102E20007205005555050078390500B81E050005E6
:102E30000505004EEC040087D40400A1BD040090F9
:102E4000A7040049920400C17D0400EE690400C794
:102E5000560400444404005C32040008210400418C
:102E6000100400000004003FF00300F8E003002617
:102E7000D20300C3C30300CCB503003AA803000A81
:102E80009B0300388E0300C08103009F750300D0B0
:102E9000690300505E03001D530300344803009192
:102EA0003D03003333030016290300381F03009746
:102EB000150300300C0300030303000BFA02004962
:102EC000F10200BAE802005CE002002DD802002DF9
:102ED000D0020059C80200B0C0020031B90200DAC5
:102EE000B10200AAAA0200A0A30200BC9C0200FA40
:102EF0009502005C8F0200DF88020082820200459A
:102F00007C02002776020027700200436A02007CE0
:102F1000640200D05E02003F590200C8530200FF65
:102F2000FDFCFAF8F6F4F2F0EEECEAE9E7E5E3E1AD
:102F3000E0DEDCDAD9D7D5D4D2D0CFCDCBCAC8C762
:102F4000C5C3C2C0BFBDBCBAB9B7B6B4B3B2B0AFE7
:102F5000ADACAAA9A8A6A5A4A2A1A09E9D9C9A9941
:102F6000989795949392908F8E8D8B8A8988878677
:102F700084838281807F7E7D7B7A79787776757491
:102F8000737271706F6E6D6C6B6A69686766656489
:102F9000636261605F5E5D5C5B5A59585857565575
:102FA0005453525150504F4E4D4C4B4A4A4948474A
:102FB0004646454443424241403F3E3E3D3C3B3B0A
:102FC0003A39383837363535343332323130302FBC
:102FD0002E2E2D2C2B2B2A29292827272625252460
:102FE000232322212120201F1E1E1D1C1C1B1B1AF7
:102FF0001919181817161615151413131212111182
:10300000100F0F0E0E0D0D0C0C0B0A0A0909080803
:103010000707060605050404030302020100000079
:103020000070430000704300007A4300000000007D
:103030000000000000000053657474696E6773201F
:1030400053746F72656400454550524F4D20496E70
:10305000697469616C697A65640A003F556E6162E2
:103060006C6520746F2073617665206D65736820D0
:10307000646174612E0A003F556E61626C65207454
:103080006F206C6F6164206D65736820646174618A
:103090002E0A00556E696669656420426564204C9D
:1030A0006576656C696E67003B20003A0A00202057
:1030B0004D36303320002055004C0046696C616D60
:1030C000656E74206C6F61642F756E6C6F61642027
:1030D0006C656E677468733A0020204D393030207B
:1030E0004B004C696E65617220416476616E636568
:1030F0003A0020204D3835312058005A2D50726F3B
:103100006265204F66667365740020204D3431334C
:10311000205300506F7765722D4C6F73732052658A
:10312000636F766572793A0020204D323530204346
:10313000004C434420436F6E74726173743A0020F4
:10314000440020490020204D3330342050002044DA
:103150000020490020204D33303120500050494498
:103160002073657474696E67733A002046002048C6
:103170000020204D3134352053004D617465726953
:10318000616C2068656174757020706172616D6535
:10319000746572733A00206D65736865732E0A0A50
:1031A00000454550524F4D2063616E20686F6C643E
:1031B0002000416374697665204D65736820536C07
:1031C0006F743A200020204D3432302053002020EC
:1031D0004D323036205800486F6D65206F6666733B
:1031E00065743A0020580020530020204D323035BD
:1031F000204200416476616E6365643A20423C6D12
:10320000696E5F7365676D656E745F74696D655F28
:1032100075733E20533C6D696E5F666565647261CF
:1032200074653E20543C6D696E5F74726176656CA6
:103230005F66656564726174653E20583C6D6178B7
:103240005F785F6A65726B3E20593C6D61785F798B
:103250005F6A65726B3E205A3C6D61785F7A5F6A87
:1032600065726B3E20453C6D61785F655F6A657293
:103270006B3E0020540020520020204D323034207C
:103280005000416363656C65726174696F6E2028DC
:10329000756E6974732F7332293A20503C707269CD
:1032A0006E745F616363656C3E20523C726574723C
:1032B0006163745F616363656C3E20543C7472614A
:1032C00076656C5F616363656C3E0020204D323033
:1032D000312058004D6178696D756D2041636365DB
:1032E0006C65726174696F6E2028756E6974732FD6
:1032F0007332293A0020204D3230332058004D617E
:1033000078696D756D20666565647261746573209A
:1033100028756E6974732F73293A0053746570733E
:103320002070657220756E69743A00204400202078
:103330004D3230302053002044697361626C656403
:103340000A0046696C616D656E74207365747469FA
:103350006E67733A0020204D3134392043203B20E2
:10336000556E69747320696E2043656C736975735B
:103370000A0020286D6D29002020473231202020AE
:10338000203B20556E69747320696E206D6D003F7F
:103390004D65736820746F6F2062696720666F7275
:1033A00020454550524F4D2E0A0000803B4400807E
:1033B0003B4400002041000096420000A042000073
:1033C000A0420000C8430000BE42D0070000D00762
:1033D0000000640000004B00000024F4D43050C30F
:1033E0008E20C2A24017828B7011127A910D816CCF
:1033F000D90AA861E108C7586607615143061E4B08
:103400005D05C145A7041A411104093D98037139AE
:1034100031034036DB0265339102D4305402802EF2
:103420001D02632CEE01752AC501B028A0011027EA
:1034300081018F2564012B244B01E0223401AC2152
:103440001F018D200D01801FFC00841EED00971DC3
:10345000DF00B81CD200E61BC600201BBC00641AAB
:10346000B200B219A8000A19A0006A189900D11771
:10347000910040178B00B516840031167E00B315FD
:1034800079003A157300C7146F0058146A00EE13E0
:1034900066008813630025135E00C7125B006C1280
:1034A000570015125400C111510070114F00211125
:1034B0004B00D61049008D10470046104400021002
:1034C0004200C00F4000800F3E00420F3C00060F3C
:1034D0003B00CB0E3800930E37005C0E3500270EF4
:1034E0003400F30D3200C10D3100900D3000600D3D
:1034F0002E00320D2D00050D2C00D90C2B00AE0C2A
:103500002900850C29005C0C2700350C27000E0CC7
:103510002600E80B2400C40B2400A00B23007D0B25
:1035200023005A0B2100390B2100180B2000F80A48
:103530001F00D90A1E00BB0A1E009D0A1D00800A3A
:103540001D00630A1C00470A1B002C0A1B00110AFD
:103550001A00F7091A00DD091900C4091900AB099E
:103560001900920917007B091800630917004C091C
:10357000160036091600200916000A091500F5087C
:103580001500E0081400CC081400B8081400A408C2
:103590001400900813007D0812006B0813005808EF
:1035A0001200460812003408110023081100120806
:1035B000110001081100F0071000E0071000D0070B
:1035C0001000C0071000B0070F00A10710009107FE
:1035D0000E0083070F0074070F0065070E005707E2
:1035E0000E0049070E003B070D002E070E002007B6
:1035F0000D0013070D0006070D00F9060C00ED067F
:103600000D00E0060C00D4060C00C8060C00BC0639
:103610000C00B0060C00A4060B0099060C008D06E9
:103620000B0082060B0077060B006C060B00610690
:103630000A0057060B004C060A0042060A0038062C
:103640000A002E060A0024060A001A060A001006BE
:10365000090007060A00FD050900F4050900EB054D
:103660000900E2050900D9050900D0050900C705D0
:103670000900BE050900B5050800AD050800A5054F
:1036800009009C050800940508008C0508008405C5
:1036900008007C050800740508006C050700650536
:1036A00008005D050700560508004E0507004705A0
:1036B00007004005080038050700310507002A0506
:1036C0000700230507001C050600160507000F0567
:1036D00007000805060002050700FB040600F504C4
:1036E0000700EE040600E8040600E2040700DB041D
:1036F0000600D5040600CF040600C9040600C30472
:103700000600BD040600B7040600B1040500AC04C1
:103710000600A6040600A00405009B04060095040C
:103720000500900406008A04050085040500800455
:1037300006007A04050075040500700405006B049A
:10374000050066040500610405005C0405005704DB
:103750000500520405004D0405004804050043041B
:1037600005003E0404003A04050035040500300459
:1037700004002C04050027040400230405001E0493
:1037800004001A04040016040500110404000D04CA
:103790000400090405000404040000040400FC0300
:1037A0000400F8030400F4030400F0030400EC0335
:1037B0000400E8030400E4030400E0030400DC0365
:1037C0000400D8030400D4030400D0030400CC0395
:1037D0000400C8030300C503030024F404D9201B1C
:1037E000C40C5C0E9804C4095F0265077101F405FE
:1037F000F900FB04B30048048700C10369005803C3
:10380000550003034500BE023A0084023100530212
:103810002A002902250004022000E4011C00C8013E
:103820001900AF0117009801140084011300710101
:1038300010006101100051010E0043010D0036011E
:103840000B002B010B0020010B00150109000C01DE
:10385000090003010800FB000800F3000800EB006A
:103860000700E4000600DE000600D8000600D200D3
:103870000600CC000500C7000500C2000500BD0021
:103880000400B9000400B5000400B1000400AD005C
:103890000400A9000400A5000300A20003009F008B
:1038A00004009B00030098000300950002009300B1
:1038B0000300900003008D0002008B0003008800CD
:1038C00002008600020084000300810002007F00E5
:1038D00002007D0002007B000200790002007700F8
:1038E0000100760002007400020072000100710005
:1038F00002006F0002006D0001006C0002006A000F
:103900000100690002006700010066000100650017
:10391000010064000200620001006100010060001B
:1039200001005F0002005D0001005C0001005B001F
:1039300001005A0001005900010058000100570021
:103940000100560001005500010054000100530021
:10395000000053000100520001005100010050001E
:1039600001004F0001004E0000004E0001004D001C
:1039700001004C0001004B0000004B0001004A0018
:103980000100490001004800000048000100470014
:10399000010046000000460001004500000045000F
:1039A0000100440001004300000043000100420008
:1039B0000000420001004100000041000100400001
:1039C00001003F0000003F0001003E0000003E00FB
:1039D00001003D0000003D0001003C0000003C00F3
:1039E00000003C0001003B0000003B0001003A00E9
:1039F00000003A00010039000000390001003800E1
:103A000000003800000038000100370000003700D7
:103A100001003600000036000000360001003500CD
:103A200000003500000035000100340000003400C3
:103A300000003400010033000000330000003300B8
:103A400001003200000032000000320001003100AD
:103A500000003100000031000100300000003000A3
:103A60000000300001002F0000002F0000002F0098
:103A700000002F0001002E0000002E0000002E008C
:103A800001002D0000002D0000002D0000002D0081
:103A900001002C0000002C0000002C0000002C0075
:103AA00001002B0000002B0000002B0000002B0069
:103AB00001002A0000002A0000002A0000002A005D
:103AC0000100290000002900000029000000290051
:103AD0000000290001002800000028000000280044
:103AE0000000280000002800010027000000270037
:103AF000000027000000270000002700010026002A
:103B0000000026000000260000002600000026001D
:103B10000100250000002500000025000000250010
:103B20000000250000002500010024000000240002
:103B300000002400000024000000240001002300F5
:103B400000002300000023000000230000002300E9
:103B500000002300000023000100220000002200DA
:103B600000002200000022000000220000002200CD
:103B700001002100000021000000210000002100C0
:103B800000002100000021000000210001002000B1
:103B900000002000000020000000200000002000A5
:103BA00000002000000020000000200001001F0095
:103BB00000001F0000001F0000001F0000001F0089
:103BC00000001F0000001F0001001E0000001E007A
:103BD00000001E0000001E000000232C0000B82280
:103BE0000000561800003A0F0000B8080000B104A9
:103BF0000000710200003E01000020436F756E74EA
:103C000020583A0042656400453100626564002C2A
:103C10002073797374656D2073746F70706564219F
:103C2000204865617465725F49443A2000486561C7
:103C300074696E67204661696C65640048656174EB
:103C4000696E67206661696C6564004D31313220B0
:103C500053687574646F776E001000C90210012CF0
:103C6000014001220170011801B0010E01F00104B0
:103C7000015002FA00B002F0003003E600D003DC8D
:103C8000009004D2007005C800A006BE000008B471
:103C900000B009AA00D00BA000600E960060118C45
:103CA000000015820020197800C01D6E00A022645B
:103CB00000B0275A00902C500000314600E0343C00
:103CC0000010383200903A2800603C1E00A03D14DD
:103CD00000803E0A00203F0000544845524D414CB0
:103CE0002052554E4157415900546865726D616CC0
:103CF0002052756E61776179004572723A204D41AC
:103D00005854454D50004D415854454D5020747203
:103D100069676765726564004572723A204D494E65
:103D200054454D50004D494E54454D5020747269D4
:103D300067676572656400202F002042403A0020CA
:103D4000403A0020573A0020573A00496E76616C9D
:103D500069642065787472756465720A007C3C3E03
:103D60005E2B3D3F2F5B5D3B2C2A225C0043616E46
:103D70006E6F74206F70656E207375626469722057
:103D800000534420496E6974204661696C005344B5
:103D90002063617264206F6B0A006F70656E526FF2
:103DA0006F74206661696C65640A00766F6C756D6E
:103DB000652E696E6974206661696C65640A004EDF
:103DC0006F20534420636172640A000A4D3234004C
:103DD0004D3233202573002E0A006F70656E206609
:103DE00061696C65642C2046696C653A20004669FF
:103DF0006C652073656C65637465640A00205369A3
:103E00007A653A200046696C65206F70656E65645E
:103E10003A2000454E4420535542524F5554494E86
:103E2000450A002220706F73002220706172656E57
:103E3000743A2200535542524F5554494E4520433F
:103E4000414C4C207461726765743A22005375626C
:103E500063616C6C204F766572666C6F7700457895
:103E6000636565646564206D617820535542524FE7
:103E70005554494E452064657074683A002E0A0016
:103E800044656C6574696F6E206661696C65642C4D
:103E90002046696C653A200046696C652064656C53
:103EA000657465643A00363726033C3D380E2E3083
:103EB0003E121A1C180AFF4309070844000124F4A3
:103EC00004D9201BC40C5C0E9804C4095F0265076A
:103ED0007101F405F900FB04B30048048700C10335
:103EE00069005803550003034500BE023A008402EE
:103EF000310053022A002902250004022000E401B7
:103F00001C00C8011900AF011700980114008401BA
:103F10001300710110006101100051010E004301F6
:103F20000D0036010B002B010B0020010B001501C9
:103F300009000C01090003010800FB000800F30060
:103F40000800EB000700E4000600DE000600D800D1
:103F50000600D2000600CC000500C7000500C20024
:103F60000500BD000400B9000400B5000400B10064
:103F70000400AD000400A9000400A5000300A20095
:103F800003009F0004009B000300980003009500BD
:103F9000020093000300900003008D0002008B00DC
:103FA00003008800020086000200840003008100F4
:103FB00002007F0002007D0002007B000200790009
:103FC0000200770001007600020074000200720017
:103FD0000100710002006F0002006D0001006C0022
:103FE00002006A000100690002006700010066002B
:103FF0000100650001006400020062000100610030
:104000000100600001005F0002005D0001005C0033
:1040100001005B0001005A00010059000100580036
:104020000100570001005600010055000100540036
:104030000100530000005300010052000100510034
:104040000100500001004F0001004E0000004E0032
:1040500001004D0001004C0001004B0000004B002E
:1040600001004A000100490001004800000048002A
:104070000100470001004600000046000100450025
:10408000000045000100440001004300000043001F
:104090000100420000004200010041000000410018
:1040A0000100400001003F0000003F0001003E0011
:1040B00000003E0001003D0000003D0001003C000A
:1040C00000003C0000003C0001003B0000003B0001
:1040D00001003A0000003A000100390000003900F8
:1040E00001003800000038000000380001003700EF
:1040F00000003700010036000000360000003600E6
:1041000001003500000035000000350001003400DA
:1041100000003400000034000100330000003300D0
:1041200000003300010032000000320000003200C5
:1041300001003100000031000000310001003000BA
:10414000000030000000300001002F0000002F00B0
:1041500000002F0000002F0001002E0000002E00A4
:1041600000002E0001002D0000002D0000002D0099
:1041700000002D0001002C0000002C0000002C008D
:1041800000002C0001002B0000002B0000002B0081
:1041900000002B0001002A0000002A0000002A0075
:1041A00000002A0001002900000029000000290069
:1041B000000029000000290001002800000028005C
:1041C000000028000000280000002800010027004F
:1041D0000000270000002700000027000000270043
:1041E0000100260000002600000026000000260036
:1041F0000000260001002500000025000000250029
:10420000000025000000250000002500010024001A
:10421000000024000000240000002400000024000E
:104220000100230000002300000023000000230001
:1042300000002300000023000000230001002200F2
:1042400000002200000022000000220000002200E6
:1042500000002200010021000000210000002100D8
:1042600000002100000021000000210000002100CA
:1042700001002000000020000000200000002000BD
:1042800000002000000020000000200000002000AE
:1042900001001F0000001F0000001F0000001F00A1
:1042A00000001F0000001F0000001F0001001E0092
:1042B00000001E0000001E0000001E00000024F48C
:1042C000D43050C38E20C2A24017828B7011127A54
:1042D000910D816CD90AA861E108C7586607615140
:1042E00043061E4B5D05C145A7041A411104093D53
:1042F0009803713931034036DB0265339102D430C3
:104300005402802E1D02632CEE01752AC501B028CF
:10431000A001102781018F2564012B244B01E0228D
:104320003401AC211F018D200D01801FFC00841E73
:10433000ED00971DDF00B81CD200E61BC600201B55
:10434000BC00641AB200B219A8000A19A0006A18C9
:104350009900D117910040178B00B51684003116D3
:104360007E00B31579003A157300C7146F00581416
:104370006A00EE1366008813630025135E00C712FF
:104380005B006C12570015125400C11151007011DE
:104390004F0021114B00D61049008D1047004610E8
:1043A000440002104200C00F4000800F3E00420F48
:1043B0003C00060F3B00CB0E3800930E37005C0E1E
:1043C0003500270E3400F30D3200C10D3100900D81
:1043D0003000600D2E00320D2D00050D2C00D90C83
:1043E0002B00AE0C2900850C29005C0C2700350C35
:1043F00027000E0C2600E80B2400C40B2400A00BA1
:1044000023007D0B23005A0B2100390B2100180BD0
:104410002000F80A1F00D90A1E00BB0A1E009D0AD0
:104420001D00800A1D00630A1C00470A1B002C0A9D
:104430001B00110A1A00F7091A00DD091900C40946
:104440001900AB091900920917007B0918006309CC
:1044500017004C09160036091600200916000A0933
:104460001500F5081500E0081400CC081400B80881
:104470001400A4081400900813007D0812006B08B3
:1044800013005808120046081200340811002308CF
:1044900011001208110001081100F0071000E007D8
:1044A0001000D0071000C0071000B0070F00A107D0
:1044B000100091070E0083070F0074070F006507B7
:1044C0000E0057070E0049070E003B070D002E0790
:1044D0000E0020070D0013070D0006070D00F9065A
:1044E0000C00ED060D00E0060C00D4060C00C8061A
:1044F0000C00BC060C00B0060C00A4060B009906CC
:104500000C008D060B0082060B0077060B006C0674
:104510000B0061060A0057060B004C060A00420613
:104520000A0038060A002E060A0024060A001A06A7
:104530000A001006090007060A00FD050900F40537
:104540000900EB050900E2050900D9050900D005BD
:104550000900C7050900BE050900B5050800AD053D
:104560000800A50509009C050800940508008C05B5
:104570000800840508007C050800740508006C0527
:104580000700650508005D050700560508004E0593
:1045900007004705070040050800380507003105FA
:1045A00007002A050700230507001C05060016055D
:1045B00007000F0507000805060002050700FB04B9
:1045C0000600F5040700EE040600E8040600E20415
:1045D0000700DB040600D5040600CF040600C9046A
:1045E0000600C3040600BD040600B7040600B104BB
:1045F0000500AC040600A6040600A00405009B0408
:10460000060095040500900406008A040500850450
:104610000500800406007A04050075040500700496
:1046200005006B04050066040500610405005C04D8
:10463000050057040500520405004D040500480418
:104640000500430405003E0404003A040500350457
:104650000500300404002C04050027040400230492
:1046600005001E0404001A040400160405001104C9
:1046700004000D04040009040500040404000004FF
:104680000400FC030400F8030400F4030400F00336
:104690000400EC030400E8030400E4030400E00366
:1046A0000400DC030400D8030400D4030400D00396
:1046B0000400CC030400C8030300C5030300726FA9
:1046C000746174696F6E206D61747269783A0A0062
:1046D00024F404D9201BC40C5C0E9804C4095F02A6
:1046E00065077101F405F900FB04B3004804870075
:1046F000C10369005803550003034500BE023A0098
:104700008402310053022A002902250004022000FD
:10471000E4011C00C8011900AF0117009801140042
:1047200084011300710110006101100051010E009D
:1047300043010D0036010B002B010B0020010B0083
:10474000150109000C01090003010800FB00080025
:10475000F3000800EB000700E4000600DE0006009E
:10476000D8000600D2000600CC000500C7000500F6
:10477000C2000500BD000400B9000400B50004003B
:10478000B1000400AD000400A9000400A50003006E
:10479000A20003009F0004009B0003009800030098
:1047A0009500020093000300900003008D000200BA
:1047B0008B000300880002008600020084000300D2
:1047C000810002007F0002007D0002007B000200E9
:1047D00079000200770001007600020074000200F8
:1047E00072000100710002006F0002006D00010004
:1047F0006C0002006A00010069000200670001000D
:104800006600010065000100640002006200010012
:1048100061000100600001005F0002005D00010016
:104820005C0001005B0001005A000100590001001A
:10483000580001005700010056000100550001001A
:104840005400010053000000530001005200010019
:1048500051000100500001004F0001004E00000017
:104860004E0001004D0001004C0001004B00000013
:104870004B0001004A00010049000100480000000F
:10488000480001004700010046000000460001000A
:104890004500000045000100440001004300000005
:1048A00043000100420000004200010041000000FE
:1048B00041000100400001003F0000003F000100F6
:1048C0003E0000003E0001003D0000003D000100F0
:1048D0003C0000003C0000003C0001003B000000E8
:1048E0003B0001003A0000003A00010039000000DE
:1048F00039000100380000003800000038000100D5
:1049000037000000370001003600000036000000CC
:1049100036000100350000003500000035000100C0
:1049200034000000340000003400010033000000B7
:1049300033000000330001003200000032000000AC
:1049400032000100310000003100000031000100A0
:104950003000000030000000300001002F00000097
:104960002F0000002F0000002F0001002E0000008B
:104970002E0000002E0001002D0000002D00000080
:104980002D0000002D0001002C0000002C00000074
:104990002C0000002C0001002B0000002B00000068
:1049A0002B0000002B0001002A0000002A0000005C
:1049B0002A0000002A000100290000002900000050
:1049C0002900000029000000290001002800000043
:1049D0002800000028000000280000002800010036
:1049E000270000002700000027000000270000002B
:1049F000270001002600000026000000260000001D
:104A0000260000002600010025000000250000000F
:104A10002500000025000000250000002500010001
:104A200024000000240000002400000024000000F6
:104A300024000100230000002300000023000000E8
:104A400023000000230000002300000023000100D9
:104A500022000000220000002200000022000000CE
:104A600022000000220001002100000021000000BF
:104A700021000000210000002100000021000000B2
:104A800021000100200000002000000020000000A4
:104A90002000000020000000200000002000000096
:104AA000200001001F0000001F0000001F00000088
:104AB0001F0000001F0000001F0000001F00010079
:104AC0001E0000001E0000001E0000001E0000006E
:104AD00024F4D43050C38E20C2A24017828B7011B0
:104AE000127A910D816CD90AA861E108C75866074E
:104AF000615143061E4B5D05C145A7041A411104CF
:104B0000093D9803713931034036DB026533910268
:104B1000D4305402802E1D02632CEE01752AC5018B
:104B2000B028A001102781018F2564012B244B019F
:104B3000E0223401AC211F018D200D01801FFC00FB
:104B4000841EED00971DDF00B81CD200E61BC600D6
:104B5000201BBC00641AB200B219A8000A19A000F8
:104B60006A189900D117910040178B00B516840080
:104B700031167E00B31579003A157300C7146F0023
:104B800058146A00EE1366008813630025135E0054
:104B9000C7125B006C12570015125400C11151006E
:104BA00070114F0021114B00D61049008D104700A5
:104BB0004610440002104200C00F4000800F3E002B
:104BC000420F3C00060F3B00CB0E3800930E37001F
:104BD0005C0E3500270E3400F30D3200C10D31009C
:104BE000900D3000600D2E00320D2D00050D2C00B3
:104BF000D90C2B00AE0C2900850C29005C0C270079
:104C0000350C27000E0C2600E80B2400C40B2400F2
:104C1000A00B23007D0B23005A0B2100390B210030
:104C2000180B2000F80A1F00D90A1E00BB0A1E003C
:104C30009D0A1D00800A1D00630A1C00470A1B0014
:104C40002C0A1B00110A1A00F7091A00DD091900C5
:104C5000C4091900AB091900920917007B09180053
:104C6000630917004C0916003609160020091600C2
:104C70000A091500F5081500E0081400CC08140016
:104C8000B8081400A4081400900813007D0812004E
:104C90006B0813005808120046081200340811006F
:104CA000230811001208110001081100F00710007C
:104CB000E0071000D0071000C0071000B0070F0079
:104CC000A107100091070E0083070F0074070F0063
:104CD00065070E0057070E0049070E003B070D0041
:104CE0002E070E0020070D0013070D0006070D000C
:104CF000F9060C00ED060D00E0060C00D4060C00D1
:104D0000C8060C00BC060C00B0060C00A4060B0084
:104D100099060C008D060B0082060B0077060B002F
:104D20006C060B0061060A0057060B004C060A00D1
:104D300042060A0038060A002E060A0024060A0067
:104D40001A060A001006090007060A00FD050900F8
:104D5000F4050900EB050900E2050900D905090081
:104D6000D0050900C7050900BE050900B505080002
:104D7000AD050800A50509009C050800940508007C
:104D80008C050800840508007C05080074050800EF
:104D90006C050700650508005D050700560508005D
:104DA0004E050700470507004005080038050700C5
:104DB000310507002A050700230507001C0506002A
:104DC000160507000F050700080506000205070085
:104DD000FB040600F5040700EE040600E8040600E4
:104DE000E2040700DB040600D5040600CF04060039
:104DF000C9040600C3040600BD040600B70406008B
:104E0000B1040500AC040600A6040600A0040500D9
:104E10009B04060095040500900406008A04050022
:104E200085040500800406007A0405007504050069
:104E3000700405006B0405006604050061040500AC
:104E40005C04050057040500520405004D040500EC
:104E500048040500430405003E0404003A0405002C
:104E600035040500300404002C0405002704040068
:104E7000230405001E0404001A040400160405009F
:104E8000110404000D0404000904050004040400D6
:104E900000040400FC030400F8030400F40304000D
:104EA000F0030400EC030400E8030400E40304003E
:104EB000E0030400DC030400D8030400D40304006E
:104EC000D0030400CC030400C8030300C50303009F
:104ED00024F404D9201BC40C5C0E9804C4095F029E
:104EE00065077101F405F900FB04B300480487006D
:104EF000C10369005803550003034500BE023A0090
:104F00008402310053022A002902250004022000F5
:104F1000E4011C00C8011900AF011700980114003A
:104F200084011300710110006101100051010E0095
:104F300043010D0036010B002B010B0020010B007B
:104F4000150109000C01090003010800FB0008001D
:104F5000F3000800EB000700E4000600DE00060096
:104F6000D8000600D2000600CC000500C7000500EE
:104F7000C2000500BD000400B9000400B500040033
:104F8000B1000400AD000400A9000400A500030066
:104F9000A20003009F0004009B0003009800030090
:104FA0009500020093000300900003008D000200B2
:104FB0008B000300880002008600020084000300CA
:104FC000810002007F0002007D0002007B000200E1
:104FD00079000200770001007600020074000200F0
:104FE00072000100710002006F0002006D000100FC
:104FF0006C0002006A000100690002006700010005
:10500000660001006500010064000200620001000A
:1050100061000100600001005F0002005D0001000E
:105020005C0001005B0001005A0001005900010012
:105030005800010057000100560001005500010012
:105040005400010053000000530001005200010011
:1050500051000100500001004F0001004E0000000F
:105060004E0001004D0001004C0001004B0000000B
:105070004B0001004A000100490001004800000007
:105080004800010047000100460000004600010002
:1050900045000000450001004400010043000000FD
:1050A00043000100420000004200010041000000F6
:1050B00041000100400001003F0000003F000100EE
:1050C0003E0000003E0001003D0000003D000100E8
:1050D0003C0000003C0000003C0001003B000000E0
:1050E0003B0001003A0000003A00010039000000D6
:1050F00039000100380000003800000038000100CD
:1051000037000000370001003600000036000000C4
:1051100036000100350000003500000035000100B8
:1051200034000000340000003400010033000000AF
:1051300033000000330001003200000032000000A4
:105140003200010031000000310000003100010098
:105150003000000030000000300001002F0000008F
:105160002F0000002F0000002F0001002E00000083
:105170002E0000002E0001002D0000002D00000078
:105180002D0000002D0001002C0000002C0000006C
:105190002C0000002C0001002B0000002B00000060
:1051A0002B0000002B0001002A0000002A00000054
:1051B0002A0000002A000100290000002900000048
:1051C000290000002900000029000100280000003B
:1051D000280000002800000028000000280001002E
:1051E0002700000027000000270000002700000023
:1051F0002700010026000000260000002600000015
:105200002600000026000100250000002500000007
:1052100025000000250000002500000025000100F9
:1052200024000000240000002400000024000000EE
:1052300024000100230000002300000023000000E0
:1052400023000000230000002300000023000100D1
:1052500022000000220000002200000022000000C6
:1052600022000000220001002100000021000000B7
:1052700021000000210000002100000021000000AA
:10528000210001002000000020000000200000009C
:10529000200000002000000020000000200000008E
:1052A000200001001F0000001F0000001F00000080
:1052B0001F0000001F0000001F0000001F00010071
:1052C0001E0000001E0000001E0000001E00000066
:1052D00024F4D43050C38E20C2A24017828B7011A8
:1052E000127A910D816CD90AA861E108C758660746
:1052F000615143061E4B5D05C145A7041A411104C7
:10530000093D9803713931034036DB026533910260
:10531000D4305402802E1D02632CEE01752AC50183
:10532000B028A001102781018F2564012B244B0197
:10533000E0223401AC211F018D200D01801FFC00F3
:10534000841EED00971DDF00B81CD200E61BC600CE
:10535000201BBC00641AB200B219A8000A19A000F0
:105360006A189900D117910040178B00B516840078
:1053700031167E00B31579003A157300C7146F001B
:1053800058146A00EE1366008813630025135E004C
:10539000C7125B006C12570015125400C111510066
:1053A00070114F0021114B00D61049008D1047009D
:1053B0004610440002104200C00F4000800F3E0023
:1053C000420F3C00060F3B00CB0E3800930E370017
:1053D0005C0E3500270E3400F30D3200C10D310094
:1053E000900D3000600D2E00320D2D00050D2C00AB
:1053F000D90C2B00AE0C2900850C29005C0C270071
:10540000350C27000E0C2600E80B2400C40B2400EA
:10541000A00B23007D0B23005A0B2100390B210028
:10542000180B2000F80A1F00D90A1E00BB0A1E0034
:105430009D0A1D00800A1D00630A1C00470A1B000C
:105440002C0A1B00110A1A00F7091A00DD091900BD
:10545000C4091900AB091900920917007B0918004B
:10546000630917004C0916003609160020091600BA
:105470000A091500F5081500E0081400CC0814000E
:10548000B8081400A4081400900813007D08120046
:105490006B08130058081200460812003408110067
:1054A000230811001208110001081100F007100074
:1054B000E0071000D0071000C0071000B0070F0071
:1054C000A107100091070E0083070F0074070F005B
:1054D00065070E0057070E0049070E003B070D0039
:1054E0002E070E0020070D0013070D0006070D0004
:1054F000F9060C00ED060D00E0060C00D4060C00C9
:10550000C8060C00BC060C00B0060C00A4060B007C
:1055100099060C008D060B0082060B0077060B0027
:105520006C060B0061060A0057060B004C060A00C9
:1055300042060A0038060A002E060A0024060A005F
:105540001A060A001006090007060A00FD050900F0
:10555000F4050900EB050900E2050900D905090079
:10556000D0050900C7050900BE050900B5050800FA
:10557000AD050800A50509009C0508009405080074
:105580008C050800840508007C05080074050800E7
:105590006C050700650508005D0507005605080055
:1055A0004E050700470507004005080038050700BD
:1055B000310507002A050700230507001C05060022
:1055C000160507000F05070008050600020507007D
:1055D000FB040600F5040700EE040600E8040600DC
:1055E000E2040700DB040600D5040600CF04060031
:1055F000C9040600C3040600BD040600B704060083
:10560000B1040500AC040600A6040600A0040500D1
:105610009B04060095040500900406008A0405001A
:1056200085040500800406007A0405007504050061
:10563000700405006B0405006604050061040500A4
:105640005C04050057040500520405004D040500E4
:1056500048040500430405003E0404003A04050024
:1056600035040500300404002C0405002704040060
:10567000230405001E0404001A0404001604050097
:10568000110404000D0404000904050004040400CE
:1056900000040400FC030400F8030400F403040005
:1056A000F0030400EC030400E8030400E403040036
:1056B000E0030400DC030400D8030400D403040066
:1056C000D0030400CC030400C8030300C503030097
:1056D0001000C90210012C014001220170011801C3
:1056E000B0010E01F00104015002FA00B002F00016
:1056F0003003E600D003DC009004D2007005C8003F
:10570000A006BE000008B400B009AA00D00BA0009B
:10571000600E960060118C00001582002019780040
:10572000C01D6E00A0226400B0275A00902C5000CB
:1057300000314600E0343C0010383200903A280036
:10574000603C1E00A03D1400803E0A00203F000087
:105750006001F4017001EA019001E001B001D6019D
:10576000D001CC010002C2013002B8016002AE01DA
:105770009002A401D0029A012003900170038601D7
:10578000C0037C0130047201A004680120055E01A1
:10579000B005540160064A0120074001F0073601B8
:1057A000F0082C01100A2201500B1801C00C0E0148
:1057B000500E04013010FA002012F0005014E600E0
:1057C000C016DC007019D200501CC800501FBE006B
:1057D0007022B400B025AA00F028A000202C96006A
:1057E000302F8C0010328200A0347800F0366E002A
:1057F000E0386400803A5A00403B5500E03B5000DE
:10580000F03C4600C03D3C00603E3200E03E2800D7
:10581000303F1E00503F1900703F1400A03F0A00A7
:10582000C03F0000D03FF6FFE03FECFF5A5F6D6FD6
:1058300076655F636F6D700A0047323858004732F3
:105840003859004732385A004732384F0A4D3438F9
:1058500020503130004D38340047323950345239FD
:1058600039395400473239503454004732380A47E6
:10587000323643504930004732380A4732364350B7
:105880004931004732394A300047323950335430B9
:10589000004732395032425430004732380A4D31D5
:1058A000393049300A4D31303949300A47323950A0
:1058B000310A4D31303453300A4D313430533000D9
:1058C0004732380A4D31393049310A4D3130394982
:1058D000310A47323950310A4D31303453300A4D94
:1058E0003134305330004732394E5031004732396D
:1058F000503143004732394900473239543000476C
:105900003239543100473239532D31004732394949
:105910003939390A47323950324254300047323926
:105920004E503100473239503354300047323950ED
:1059300034523939395400473239503452393939AF
:105940005400473239440047323941004732395711
:1059500000417869732000206D696E3A00206D6106
:10596000783A00416363656C65726174696F6E209B
:105970006C696D697465642E0A0046415354005386
:105980004C4F570005000006010004000601000608
:1059900005000000060004004572726F72207772E5
:1059A0006974696E6720746F20454550524F4D21D0
:1059B0000A0053544F505045442E20005072696ED7
:1059C0007465722073746F707065642064756520EF
:1059D000746F206572726F72732E2046697820741E
:1059E0006865206572726F7220616E6420757365E0
:1059F000204D39393920746F207265737461727467
:105A00002E202854656D7065726174757265206909
:105A1000732072657365742E205365742069742039
:105A200061667465722072657374617274696E6701
:105A3000290A004E6F20436865636B73756D20778C
:105A4000697468206C696E65206E756D6265722C74
:105A5000204C617374204C696E653A20004E6F20B3
:105A6000436865636B73756D2077697468206C6932
:105A70006E65206E756D6265722C204C61737420AA
:105A80004C696E653A2000636865636B73756D20C1
:105A90006D69736D617463682C204C617374204C64
:105AA000696E653A20004C696E65204E756D6265C1
:105AB00072206973206E6F74204C617374204C697E
:105AC0006E65204E756D6265722B312C204C6173B2
:105AD00074204C696E653A20004D313130005365B9
:105AE0007269616C20737461747573206D69736D74
:105AF000617463680A00776169740A005344207214
:105B0000656164206572726F720A00486F74656E19
:105B1000642049646C652054696D656F7574004834
:105B20006F74656E642049646C652054696D656F9F
:105B300075740A002121204B494C4C206361757318
:105B40006564206279204B494C4C20627574746FF7
:105B50006E2F70696E0A002121204B494C4C206346
:105B6000617573656420627920746F6F206D756351
:105B70006820696E6163746976652074696D65205B
:105B80002D2063757272656E7420636F6D6D616E2A
:105B9000643A20004D656469612052656D6F7665D9
:105BA00064004D6564696120496E73657274656453
:105BB000004D313030305300627573793A20706196
:105BC0007573656420666F7220696E7075740A0063
:105BD000627573793A2070617573656420666F72BF
:105BE00020757365720A00627573793A2070726F5E
:105BF00063657373696E670A00506C656173652035
:105C00005265736574005052494E544552204841C4
:105C10004C5445440025533A20255300706F776556
:105C2000726F6666004B494C4C45442E2000507202
:105C3000696E7465722068616C7465642E206B698E
:105C40006C6C28292063616C6C6564210A005354D4
:105C50004F505045442E20005072696E746572207A
:105C600073746F707065642064756520746F20654F
:105C700072726F72732E2046697820746865206591
:105C800072726F7220616E6420757365204D3939B0
:105C90003920746F20726573746172742E202854D9
:105CA000656D7065726174757265206973207265C7
:105CB0007365742E20536574206974206166746561
:105CC000722072657374617274696E67290A006567
:105CD00063686F3A004572726F723A00204A002082
:105CE000204D3432312049002020473239204939B3
:105CF00039390A006163746976650A00696E0000CB
:105D00002053797374656D2076312E303120002058
:105D100020207C0A004E414E0020202E2020200012
:105D2000207C004C43443A0A004353563A0A002070
:105D3000666F7220003A0A0A000A42656420546FB6
:105D4000706F677261706879205265706F7274004D
:105D500050726F62696E67204661696C65640A0003
:105D600050726F62696E67204661696C65640020DD
:105D70005A3A200020593A200042656420583A20BF
:105D8000004732384C3000446F6E652E0A003F49A0
:105D90006E76616C69642073746F726167652073DD
:105DA0006C6F742E0A3F557365203020746F20008D
:105DB0003F454550524F4D2073746F7261676520A7
:105DC0006E6F7420617661696C61626C652E0A0089
:105DD000446F6E652E0A003F496E76616C696420DF
:105DE00073746F7261676520736C6F742E0A3F5510
:105DF0007365203020746F20003F454550524F4D51
:105E00002073746F72616765206E6F7420617661B4
:105E1000696C61626C652E0A00473239205032206D
:105E200066696E69736865642E0A005859206F753B
:105E30007473696465207072696E7461626C652048
:105E40007261646975732E0A003F4572726F722029
:105E5000696E20427573696E657373204361726465
:105E6000206D6561737572656D656E742E0A004DE7
:105E7000616E75616C6C792070726F62696E6720FB
:105E8000756E726561636861626C6520706F696EC2
:105E900074732E0A00292E0A0A0050726F62696E0E
:105EA000672061726F756E642028004D65736820ED
:105EB000696E76616C6964617465642E2050726FDE
:105EC00062696E67206D6573682E0A004D657368A0
:105ED000207A65726F65642E0A0044656661756C90
:105EE000742073746F7261676520736C6F742030F7
:105EF0002073656C65637465642E0A004C6F616481
:105F0000696E6720746573745F7061747465726E16
:105F10002076616C7565732E0A0A00496E76616C95
:105F2000696420746573745F7061747465726E2047
:105F300076616C75652E20282D3120746F203229F2
:105F40000A0A0020696E76616C6964617465642E6A
:105F50000A0A004C6F636174696F6E7300456E745A
:105F6000697265204D657368005374616E64617277
:105F70006420446576696174696F6E3A20004D65EE
:105F8000616E204D657368204865696768743A20C2
:105F90000023206F662073616D706C65733A20007A
:105FA0000A4D657368206F6E6C7920706172746938
:105FB000616C6C7920706F70756C617465642E0A09
:105FC0000A0050726F62696E6720506F696E7400CC
:105FD00025532025692F2569002E0A002F005072B5
:105FE0006F62696E67206D65736820706F696E748B
:105FF000200020616E642074616B652061206D65F6
:1060000061737572656D656E742E0A006D6D207416
:106010006869636B2E0A00427573696E657373203D
:1060200043617264206973200052656D6F7665204C
:1060300026204D6561737572652042656400526566
:106040006D6F7665207368696D00506C61636520C3
:106050007368696D20756E646572206E6F7A7A6CF4
:1060600065000A4D657368206F6E6C7920706172EF
:106070007469616C6C7920706F70756C61746564A3
:106080002E0A004D65736820506F696E74204D654F
:106090006173757265642061743A20004D656173A7
:1060A00075726500506C616365205368696D2026C8
:1060B000204D656173757265004D6F76696E67205E
:1060C000746F206E657874004D657368204564694F
:1060D00074696E672053746F7070656400446F6EEE
:1060E000652045646974696E67204D6573680A00B0
:1060F000446F6E652045646974696E67204D6573F1
:10610000680046696E652054756E696E67204D653E
:1061100073680028582C5929206F75747369646559
:10612000207072696E7461626C6520726164697559
:10613000732E0A004F6666736574206F7574206F46
:106140006620626F756E64732E20283020746F2075
:1061500031306D6D290A0A00496E76616C696420E0
:106160006D617020747970652E0A0A003F284629F7
:106170006164652068656967687420666F72204293
:106180006564204C6576656C20436F72726563743C
:10619000696F6E206E6F7420706C61757369626CCC
:1061A000652E0A0A003F43616E277420616374699B
:1061B0007661746520616E642064656163746976DC
:1061C000617465206174207468652073616D652059
:1061D00074696D652E0A0A00426F74682058202683
:1061E0002059206C6F636174696F6E73206D7573D5
:1061F00074206265207370656369666965642E0A40
:106200000A003F496E76616C696420677269642098
:1062100073697A6520284A29207370656369666905
:1062200065642028322D39292E0A0A003F2850297A
:10623000686173652076616C756520696E76616C46
:1062400069642028302D36292E0A0A003F28562955
:106250006572626F7365206C6576656C20696D7020
:106260006C61757369626C652028302D34292E0AA3
:106270000A003F285229657065746974696F6E2041
:10628000636F756E7420696E76616C696420283165
:106290002B292E0A0A00446F696E672047323900A5
:1062A00093598E59895984595D0A0062656420703A
:1062B0006C616E65206E6F726D616C203D205B00BD
:1062C000436F756C64206E6F7420636F6D706C65C6
:1062D0007465204C53462100436F72726563746588
:1062E000645F5A3D0025532025692F2569000A0A5D
:1062F000002F0054696C74696E67206D65736820A7
:10630000706F696E7420003F4572726F72207072F8
:106310006F62696E6720706F696E742E2041626FC4
:106320007274696E67206F7065726174696F6E2E2A
:106330000A00436F727265637465645F5A3D00259D
:106340005320332F330054696C74696E67206D6578
:1063500073682028332F33290A00436F72726563F4
:106360007465645F5A3D00255320322F3300546911
:106370006C74696E67206D6573682028322F33292D
:106380000A00436F727265637465645F5A3D00541E
:10639000696C74696E6720506F696E7400255320B4
:1063A000312F330054696C74696E67206D657368B2
:1063B0002028312F33290A00646F6E650A00496E68
:1063C00073756666696369656E7420646174610AD9
:1063D000000000803F66663A426666B842CCCC094F
:1063E0004366663743000065430000803F66663AB7
:1063F000426666B842CCCC09436666374300006506
:10640000434578747261706F6C6174696E67206D5A
:106410006573682E2E2E0021212053544F50206387
:10642000616C6C65642062656361757365206F667D
:1064300020424C546F756368206572726F72202D14
:1064400020726573746172742077697468204D39A5
:1064500039390A0021212053544F502063616C6C5C
:1064600065642062656361757365206F6620424CC8
:10647000546F756368206572726F72202D2072658B
:1064800073746172742077697468204D3939390AE0
:10649000005072696E74696E67204F626A6563743A
:1064A000002553202569002F2F616374696F6E3AB0
:1064B00000737461727400656E6400486F74656E79
:1064C0006420746F6F20636F6C640A0053656E64A0
:1064D000204D31303820746F20726573756D650AF8
:1064E00000496E736572742066696C616D656E74C7
:1064F00020616E642073656E64204D3130380A006F
:1065000052656865617420446F6E65005265686508
:106510006174696E672E2E2E005265686561740085
:106520004865617465722054696D656F75740053B8
:10653000656E64204D31303820746F206865617459
:10654000206E6F7A7A6C650A004E6F7A7A6C6520DD
:106550005061726B656400706175736564005061B1
:1065600075736500726573756D656400526573754A
:106570006D696E67004732362043616E63656C65F6
:10658000640041425300504C4100534420707269F2
:106590006E74696E67206279746520004E6F742096
:1065A0005344207072696E74696E670A002F6175BA
:1065B000746F25632E670057726974696E67207463
:1065C0006F2066696C653A200066726573680064C6
:1065D0006F696E67002066696C653A20004E6F77C0
:1065E000200002FD55555555555FFFFFFFFFFFFF8A
:1065F000FFFFFFFE00000000003FFFFFFFFFFFFF67
:10660000FFFFFFFD000007FFFFFFFFFFFFFFFFFF92
:10661000FFFFFFFE07C00555555555555FFFFFFFAE
:10662000FFFFFFFC0A200600000000003FFFFFFF05
:10663000FFFFFFFE141005000007FFFFFFFFFFFF35
:10664000FFFFFFFC28080607C00555555555555F47
:10665000FFFFFFFE5404040A200600000000003F74
:10666000FFFFFFFC600406141005000007FFFFFF9A
:10667000FFFFFFFE50040428080607C005555555C6
:1066800055555FFC6004065404040A20060000000F
:1066900000003FFE54041C600406141005000000B6
:1066A00000001FFC28082E50040428080607C0001C
:1066B00001F03FFE1410546004065404040A200044
:1066C00002081FFC0A206654041C60040614100013
:1066D00005043FFE07C05428082E50040428080073
:1066E0000A021FFC00002E1410546004065404001B
:1066F00015013FFE00001C0A206654041C600400C3
:1067000018011FFC00000607C05428082E50040082
:1067100014013FFE00000400002E14105460040019
:1067200018011FFCFFFFFE00001C0A206654041C19
:1067300015013FFED5555400000607C05428082A0D
:106740000A021FFC84104600000400002E141051A1
:1067500005043FFEC41044FFFFFE00001C0A206138
:1067600002881FFC841046D5555400000607C0510E
:1067700001F03FFE84104484104600000400002A0B
:1067800000001FFCC41046C41044FFFFFE00001CA4
:1067900000003FFE841044841046D555540000008C
:1067A00000001FFCD555568410448410460000009C
:1067B00000003FFCFFFFFCC41046C41044FFFFFF75
:1067C000FFFF9FFE000006841044841046D55555F7
:1067D0005555BFFD555554D5555684104484104128
:1067E00004109FFFFFFFFCFFFFFCC41046C41041D4
:1067F0000411BFFFFFFFFE00000684104484104117
:1068000004109FFFFFFFFD555554D5555684104188
:1068100004109FFFFFFFFFFFFFFCFFFFFCC41041C0
:106820000411BFFFFFFFFFFFFFFE000006841041C1
:1068300004109FFFFFFFFFFFFFFD555554D5555531
:106840005555BFFFFFFFFFFFFFFFFFFFFCFFFFFFEF
:10685000FFFF9FFFFFFFFFFFFFFFFFFFFE000000A6
:1068600000003FFFFFFFFFFFFFFFFFFFFD555555F6
:1068700055555FFFFFFFFFFFFFFFFFFFFFFFFFFF1C
:10688000FFFFFFFFFFFFFFFFFFFFFFFFFFFFFFFF18
:10689000FFFFFFFFFFFFFFFFFFFFFFFFFFFFFFFF08
:1068A000FFFFFFFFFFFFFFFFFFFFFFFFFFFFFFFFF8
:1068B000FFFFFFE02EFB7DFBFBCFC1DFBB3EC0E156
:1068C000FE3C1FFDEE7B39F9F3CF9EDFBB3EDFDEE2
:1068D000FCDDE7FDEE3BBBF9EBD7BF5FBB5EDFDE68
:1068E000FDEDF7FDEEBBD3FAEBB73FDFBB4EDFDFCD
:1068F000FFCDF3FDEEDBC7FAEBBB7FC03B6EC0E321
:10690000FF1DF3FDEECBEFFADBBB7FDFBB66DFF8ED
:10691000FFCDF3FDEEEBEFFB5B033F5FBB76DFFEEE
:106920007FEDF3FDEEF3EFFB5B79BEDFBB7ADFDEDD
:106930007DEDF7FDEEF3EFFBBAFD9EDFBB7CDFDE06
:10694000FDCDE7FDEEFBEFFBBAFDC1DFBB7EC0E096
:10695000FE1C1F6D61726C696E66772E6F72670028
:10696000322E302E375F4457372E33001FFFFFFF84
:10697000FFFFFF600000000001FF4000000000007A
:10698000FF8000000000007F83CF00000C303F87B5
:10699000FF80000C301F867980000C000F8C30C700
:1069A000838C30E78C30CFC7CC31F38C30DCECEC0F
:1069B00033B98C30D86C6C33198C30D06C0C3319E3
:1069C0008C30D86C0C33198C30DC6C0E3B198C304D
:1069D000CF7C079F198C30C77C038F1940000000C3
:1069E000000002600000000000061FFFFFFFFFFF25
:1069F000F86001F4017001EA019001E001B001D6F4
:106A000001D001CC010002C2013002B8016002AE27
:106A1000019002A401D0029A012003900170038624
:106A200001C0037C0130047201A004680120055EEE
:106A300001B005540160064A0120074001F0073605
:106A400001F0082C01100A2201500B1801C00C0E95
:106A500001500E04013010FA002012F0005014E62C
:106A600000C016DC007019D200501CC800501FBEB8
:106A7000007022B400B025AA00F028A000202C96B7
:106A800000302F8C0010328200A0347800F0366E77
:106A900000E0386400803A5A00403B5500E03B502B
:106AA00000F03C4600C03D3C00603E3200E03E2825
:106AB00000303F1E00503F1900703F1400A03F0AF5
:106AC00000C03F0000D03FF6FFE03FECFF20205029
:106AD0006C616E6E65724275666665724279746548
:106AE000733A20002046726565204D656D6F72799E
:106AF0003A2000436F6D70696C65643A2041707292
:106B000020323420323032310A00204C617374203C
:106B1000557064617465643A20323032312D3034FE
:106B20002D3138207C20417574686F723A20546989
:106B30006E794D616368696E657333440A00322E65
:106B4000302E375F4457372E330A004D61726C691F
:106B50006E0020536F6674776172652052657365AD
:106B6000740A00205761746368646F67205265730C
:106B700065740A002042726F776E206F7574205220
:106B8000657365740A002045787465726E616C20C7
:106B900052657365740A00506F77657255700A000C
:106BA00073746172740A004732385859004D31309D
:106BB0003031006572726F722077726974696E6726
:106BC00020746F2066696C650A00446F6E652073DF
:106BD0006176696E672066696C652E0A004D3239F0
:106BE00000456E6473746F70730025532025632015
:106BF000256320256320256300205A3A0020593A56
:106C00000020583A00656E6473746F707320686971
:106C1000743A200000000A0B02090C0D0E0807034D
:106C2000040100000000000000000000000000005F
:106C30000000000000000000000000000000000054
:106C40001211100000000000000000000000000011
:106C500000000000000000000000004D6F7665207D
:106C600025736D6D004D6F766520302E316D6D0092
:106C70004D6F766520316D6D004D6F76652031303A
:106C80006D6D004D6F7665204178697300457874AD
:106C90007275646572004D6F7665205A004D6F768F
:106CA000652059004D6F76652058008665826543E2
:106CB00068616E67652046696C616D656E7400552C
:106CC0006E6C6F61642046696C616D656E74004C1A
:106CD0006F61642046696C616D656E740050726509
:106CE0006865617420437573746F6D0050726568D8
:106CF0006561742024004261636B0070726F6D7077
:106D0000745F0073686F7700627574746F6E0062F1
:106D10006567696E0050757267654D6F72650050EA
:106D2000617573656400436F6E74696E7565004CC0
:106D30006F61642046696C616D656E742054004912
:106D40006E736572742066696C616D656E74206126
:106D50006E642073656E64204D3130380A00220A5B
:106D600000556E6B6E6F776E20636F6D6D616E6434
:106D70003A2022002042002050006F6B0020450086
:106D8000205A00205900204D393220580020453A21
:106D900000205A3A0020593A00583A0020746F6F88
:106DA000206C6F6E6720657874727573696F6E20E2
:106DB00070726576656E7465640A0020636F6C643A
:106DC00020657874727573696F6E20707265766570
:106DD0006E7465640A00526573656E643A20006ED5
:106DE0006F74696669636174696F6E2000000022C8
:106DF00000250028002B002E003100340002010085
:106E000000050108010B0100002100240027002AD1
:106E1000002D003000330001010000040107010AC9
:106E20000105050505070508080808020202020A0F
:106E30000A0808040404040101010101010101031D
:106E400003030303030303040707070C0C0C0C0CD8
:106E50000C0C0C0202020206060606060606060BCB
:106E60000B0B0B0B0B0B0B01021020200808102042
:106E700040102040800201020108040201010204C6
:106E80000810204080804020100804020180040285
:106E900001804020100804020108040201010204DC
:106EA0000810204080010204081020408000D30117
:106EB0002F0211241FBECFEFD1E2DEBFCDBF00E015
:106EC0000CBF17E0A0E0B2E0E8E9F3E903E00BBF94
:106ED00002C007900D92AE32B107D9F72DE1AEE2B4
:106EE000B7E001C01D92A732B207E1F717E3C8E58A
:106EF000D7E300E006C021970109802FFE010F941F
:106F0000D6C4C735D10780E00807A9F70F94C8B2E7
:106F10000D94BAC90C9400002CEA35EC47E25EE30C
:106F200060910B0970910C0980910D0990910E09E7
:106F30000F94D9C56093061A7093071A8093081AA4
:106F40009093091A08952CEA35EC47E25EE36091CC
:106F50000F097091100980911109909112090F94F5
:106F600053BE6093021A7093031A8093041A90938D
:106F7000051A0895FC0184910895FC01808108950B
:106F8000FC01A081B1811C92A281B3818C918F5FA1
:106F90008C930280F381E02D90818CE0989F800D8E
:106FA0001124E1EDFAE113AE84AF089590E080E0A2
:106FB000089590E080E00895282F9091910C8330FF
:106FC00021F495FD0FC094FD0FC0892F90E0B0E033
:106FD000A0E004C0B695A795979587952A95D2F716
:106FE0008170089581E0089580E008950F931F93C4
:106FF000E62FF0E0EE59F74F008110E030E020E09E
:10700000082E04C036952795179507950A94D2F750
:1070100000FD07C0FA018083618381E01F910F9119
:10702000089580E0FBCF0F931F93CF938C01C62F61
:107030008EE690E10F94BB4FC8010F94BB4F8AE3DB
:107040000F94304F80E38C0F0F94304F8AE0CF9134
:107050001F910F910D94304F81EF91E10F94BB4F31
:1070600060E081EE91E10E94133860E08CEC91E1E8
:107070000E94133861E085EC91E10E94133861E0D1
:107080008AEB91E10E94133861E08AEA91E10E9463
:10709000133860E081EA91E10E94133861E087E9EA
:1070A00091E10E94133861E08DE891E10E9413386C
:1070B00060E086E891E10E94133861E08EE791E19B
:1070C0000E94133861E080E791E10E94133861E08B
:1070D00082E691E10E94133860E083E591E10E942D
:1070E000133860E085E491E10E94133860E08FE29C
:1070F00091E10E94133861E08EE191E10E94133822
:1071000061E08FE091E10E94133861E088E091E155
:107110000E94133860E081E091E10E94133861E041
:1071200088EF90E10E94133861E083EE90E10E94C5
:10713000133861E085ED90E10E94133861E082EC44
:1071400090E10E94133860E085EB90E10E941338D3
:1071500061E080EB90E10E94133861E083EA90E106
:107160000E94133860E08FE890E10E94133860E0DD
:107170008CE790E10E94133860E08FE19BE10E9470
:10718000D937682F617083E790E10C941338EF9240
:10719000FF920F931F93CF93DF93EC018B017A0142
:1071A0008A859B858617970731F0888199810F948E
:1071B00056AA1B870A87B701888199810F94999CE9
:1071C0002E813F81820F932F911D9F838E8390E0AC
:1071D00080E0DF91CF911F910F91FF90EF90089584
:1071E0009F92AF92BF92CF92DF92EF92FF920F9356
:1071F0001F93CF93DF93EC018B01942EA52E8A85EC
:107200009B858617970731F0888199810F9456AA3C
:107210001B870A8788859985019649F5BC800A8174
:107220008E81080FC880D980D6015596ED91FC91CA
:10723000C6011995B80EE92CFA2C10E0F70121913E
:107240007F01211127C08E819F81810F911D9F8316
:107250008E8390E080E0DF91CF911F910F91FF909E
:10726000EF90DF90CF90BF90AF909F9008950E81E8
:107270001F81692D7A2D888199810F94999C800FA7
:10728000912F911D288539852817390738F681E017
:1072900090E0E1CF4B2D602FC6010F94AEAA080FEE
:1072A000180FCCCFDF92EF92FF920F931F93CF93E3
:1072B000DF93EC01D62E1CAD0BAD7C0184E0E80E13
:1072C000F11CE98DFA8DC7011995412F480F2D2D1D
:1072D000602FC7010F94AEAA9BAD890F8BAF81E0E1
:1072E00090E0DF91CF911F910F91FF90EF90DF9091
:1072F0000895AF92BF92DF92EF92FF920F931F9388
:10730000CF93DF938C01EB01D42E79018FE04817E6
:1073100009F486C0A5E14A17B1F1BAE04B130EC0DB
:10732000EC81FD8130E020E042E061E0C801199588
:1073300041E756E1BE01C8010F9459AB0A80DB81D9
:10734000C02DF2E3DF1609F4E2C0FD1508F491C088
:1073500085E1D81609F4E0C0A7E1DA1609F4EFC018
:10736000B4E1DB127BC0EE81FF818D8190E0880F5C
:10737000991F8E0F9F1F11928E179F07E1F7CE0165
:107380000F9476A86BC0AA80BB804CE556E1C8017B
:107390000F9459ABF5014481440F406BBE01C80105
:1073A0000F9441AB41E0BE01C8010F9449ABD50138
:1073B00016962D913C911797EC81FD8115964C9175
:1073C00066E0C801199540E0BE01C8010F9451ABB9
:1073D0004CE556E1BE01C8010F9459ABF50144815B
:1073E000440F4F5F406BBE01C8010F9441AB41E0B9
:1073F000BE01C8010F9449ABD50115964C91159764
:1074000016962D913C91240F311DEC81FD8166E093
:10741000C801199540E0BE01C8010F9451AB8ECF51
:1074200041E0C8010F9451AB40E0BE01C8010F9488
:1074300049AB41E8BE01C8010F9441ABF70140815F
:1074400050E05595479555954795BE01C8010F9455
:1074500041AB40E0BE01C8010F9451AB81E0DF9128
:10746000CF911F910F91FF90EF90DF90BF90AF9061
:107470000895E6E4DE1609F471C0F7E4DF1609F4B6
:1074800071C08BE3D812EACFD70111969C91119766
:1074900013968C9138E0390F813031F0833011F040
:1074A000392F02C0392F985021E04B81491708F439
:1074B00020E041E0391708F040E091E05A813517AB
:1074C00008F490E0322F342B932311F4242331F26B
:1074D000F701128100E0D12C843048F490E0FC01E7
:1074E000EB53FD4FD0808F539D4FDC010C9117FF64
:1074F00004C0B701CE010F947DA8F70180818D0DE6
:1075000080838181800F8183110F89F7A7CFB70115
:10751000CE010F947DA8A2CFCE010F9460A888233E
:1075200009F49DCFEE81FF818D8190E0880F991F36
:107530008E0F9F1F11928E179F07E1F78FCFD701F4
:107540001C928A8111968C9311978D81815012968D
:107550008C9312978B8113968C9380CF8D81F7013A
:1075600080837CCF8981D7018C9378CFCF92DF92B3
:10757000EF92FF920F931F93CF93DF93CDB7DEB7B8
:107580002C970FB6F894DEBF0FBECDBFF0900C1B4A
:10759000E0900D1B2091740821111DC04DE655E1AE
:1075A0006E2D8F2D0F941AAB90E080E0F80EF092C4
:1075B0000C1BE0920D1B99272C960FB6F894DEBF9A
:1075C0000FBECDBFDF91CF911F910F91FF90EF9034
:1075D000DF90CF900895C090D91AD090DA1A25ED97
:1075E0003AE13A8329832F2D30E03C832B832E2DE3
:1075F00030E03E832D8318861F827A8769871C8638
:107600001B8600EF18E39E012F5F3F4F4AEB57E3C5
:10761000BC01C6010F949482B60185ED9AE10F94E6
:1076200056AA8F819885C2CFCF93C62F0F94B542AB
:10763000882319F0CF910D940F428C2FCF9108958C
:10764000CF93DF93EB010F94B542882319F00F9489
:10765000FF41EB01CE01DF91CF9108950F931F936E
:10766000CF93DF9300D01F92CDB7DEB79C010CE61D
:107670001CE090E1E7E8FDE0D80101900D929A95B9
:10768000E1F7F9012081318142815381F801608560
:107690007185828593850F94DFC4F80160877187B7
:1076A0008287938780E090E0A0EAB0E489839A83A0
:1076B000AB83BC83CE0101960F94A4140F900F905E
:1076C0000F900F90DF91CF911F910F910895CF935D
:1076D00084E50F94B542C0E08823D9F00F940F429F
:1076E000C82F1816B4F40F94DC5B8DE40F94304F60
:1076F00080916D0890916E080F940DAD6C2FCC0F9A
:10770000770B86E19DE00F9499528AE00F94304FF9
:10771000CFEF8C2FCF91089583E50F94B542882346
:10772000E9F00F94AFA260937C0C70937D0C809372
:107730007E0C90937F0C0F94374220E030E04AE7B4
:1077400054E40F9453BE0F9452C660930802709392
:10775000090280930A0290930B02089580915807C2
:1077600084FD13C080915A0787FD0FC080915B078D
:10777000837059F40E9439F780911F09882321F002
:1077800010921F091092200908950E9428F788E599
:107790000F946742882331F05F9A8091E40B8E7FCB
:1077A0008093E40B89E50F946742882331F08A9A2D
:1077B0008091E40B8D7F8093E40B8AE50F94674200
:1077C000882359F08091080180958170809306018B
:1077D0008091E40B8B7F8093E40B85E40F946742E8
:1077E000882351F20F94974CC7CF80912E07909128
:1077F0002F07009731F04AE050E070E060E00D9410
:10780000CBBB60E070E0CB01089580915807827196
:1078100049F480915A078C7829F480915B07837032
:1078200009F475C082E40F946742882351F00E94E6
:10783000F53B6093991470939A1480939B149093E2
:107840009C1483E50F946742882351F00F943742CC
:107850006093C9147093CA148093CB149093CC1482
:1078600084E50F946742882351F00F943742609368
:10787000CD147093CE148093CF149093D01488E5D8
:107880000F946742882351F00F9437426093AC0DF8
:107890007093AD0D8093AE0D9093AF0D89E50F946D
:1078A0006742882351F00F9437426093B00D709374
:1078B000B10D8093B20D9093B30D8AE50F9467429A
:1078C0008823B1F00F9437426093B40D7093B50DD7
:1078D0008093B60D9093B70D2DEC3CEC4CEC5DE332
:1078E0000F94EDBD181624F083E29CE00F94BB4F7B
:1078F00085E40F946742882351F00F9437426093D8
:10790000B80D7093B90D8093BA0D9093BB0D089587
:107910000F931F93CF93DF9300D000D01F921F923D
:10792000CDB7DEB7FC018B0183A5811112C081E0C8
:1079300083A784819581A681B781B05889839A8372
:10794000AB83BC83BE016F5F7F4F8CE69CE00F94DE
:107950001E401D821E821F82188620E030E040E01B
:107960005FE360918F0D7091900D8091910D9091DA
:10797000920D0F94DFC469837A838B839C839E016D
:107980002B5F3F4FAE014F5F5F4F6BE87DE087E8B5
:107990009DE00F94F93E1D821E821F82188620E012
:1079A00030E040E05FE3F801608571858285938572
:1079B0000F94DFC469837A838B839C83B8016C5FE7
:1079C0007F4F9E012B5F3F4FAE014F5F5F4FC8015E
:1079D0000F94F93E28960FB6F894DEBF0FBECDBFC8
:1079E000DF91CF911F910F9108952F923F924F9267
:1079F0005F926F927F928F929F92AF92BF92CF923F
:107A0000DF92EF92FF920F931F93CF93DF93CDB747
:107A1000DEB7A2970FB6F894DEBF0FBECDBF8C01C4
:107A20001B015E834D834090870D5090880D6090C0
:107A3000890D70908A0D80908B0D90908C0DA09088
:107A40008D0DB0908E0DDB018D919D910D90BC91AF
:107A5000A02D8F87988BA98BBA8B9C01AD01C30198
:107A6000B2010F94DEC46B017C01D10114968D919B
:107A70009D910D90BC91A02D8B8B9C8BAD8BBE8B63
:107A80009C01AD01C501B4010F94DEC46F8B788FEA
:107A9000898F9A8FAD81BE818D919D910D90BC9102
:107AA000A02D8F839887A987BA879C01AD01C30158
:107AB000B2010F94DEC46B8F7C8F8D8F9E8FAD8152
:107AC000BE8114968D919D910D90BC91A02D8B87B8
:107AD0009C87AD87BE879C01AD01C501B4010F94A1
:107AE000DEC46F8F78A389A39AA3A7019601C7016B
:107AF000B6010F9453BE6B017C012F89388D498DDF
:107B00005A8DCA01B9010F9453BE9B01AC01C70144
:107B1000B6010F94DFC44B015C012F853889498978
:107B20005A896F81788589859A850F94DEC42B01E7
:107B30003C012B893C894D895E896B857C858D85CF
:107B40009E850F94DEC46B017C01A3019201C301E9
:107B5000B2010F9453BE2B013C01A7019601C7014E
:107B6000B6010F9453BE9B01AC01C301B2010F9447
:107B7000DFC40F94DDC76B017C012B8D3C8D4D8DD7
:107B80005E8DCA01B9010F9453BE2B013C012F8DAC
:107B900038A149A15AA1CA01B9010F9453BE9B0152
:107BA000AC01C301B2010F94DFC49B01AC01C5015C
:107BB000B4010F943FC71816B4F520E030E0A901D6
:107BC000C701B6010F943FC787FF2AC0C701B6019E
:107BD000905820E030E040EA50E40F943FC7181678
:107BE00014F5A1016D817E81C8010E94F53CA29629
:107BF0000FB6F894DEBF0FBECDBFDF91CF911F91BE
:107C00000F91FF90EF90DF90CF90BF90AF909F903B
:107C10008F907F906F905F904F903F902F9008953E
:107C2000C701B601D6CF20E030E040E050E4C50106
:107C3000B4010F943FC7181624F4B101C8010E9483
:107C4000883C19821A821B821C82BE016F5F7F4FA3
:107C5000C1010F941E402DEC3CEC4CEC5CE3C701E1
:107C6000B6010F9453BE9B01AC01F8016081718194
:107C7000828193810F9453BE69837A838B839C8323
:107C8000C8010F94E59ABE016F5F7F4F8D819E8181
:107C90000F941E40ACCF3F924F925F926F927F92B3
:107CA0008F929F92AF92BF92CF92DF92EF92FF920C
:107CB0000F931F93CF93DF93CDB7DEB768970FB6BF
:107CC000F894DEBF0FBECDBF7C01DB018C91342E5A
:107CD000380E95E0931508F40EC11196EC91022F21
:107CE0000E0F063008F007C1F0E0EE59F74F408064
:107CF000512C712C612C082E04C0769467945794F3
:107D000047940A94D2F740FEF6C0E02FF0E0EE5917
:107D1000F74F4080512C712C612C032C04C07694B9
:107D20006794579447940A94D2F740FEE4C0122F08
:107D3000A42E6B010F94BC442B013C016A2D660FED
:107D4000770B072E000C880B990B0F94F4BD4B0199
:107D50005C01AC019B01C301B2010F94DFC46D87CC
:107D60007E878F87988B832D0F94BC44A501940147
:107D70000F94DEC469837A838B839C83F6018181AF
:107D80000F9426442B013C01612F660F770B072EC1
:107D9000000C880B990B0F94F4BD4B015C01AC01F6
:107DA0009B01C301B2010F94DFC4698B7A8B8B8B6B
:107DB0009C8B802F0F942644A50194010F94DEC460
:107DC0006D837E838F839887F70180859185A28557
:107DD000B38589879A87AB87BC878D8B9E8BAF8B4A
:107DE000B88F4FEE50E061E070E0CE0141960E9406
:107DF000A6EF4FEE50E061E070E0CE0105960E94E4
:107E0000A6EF4FEE50E061E070E0CE010D960E94CB
:107E1000A6EF4FEE50E061E070E0CE0101960E94C7
:107E2000A6EF49885A886B887C8827E137EB41EDBB
:107E300058EBC301B2010F943FC787FD5CC027E038
:107E400030E040E753E4C301B2010F94EDBD1816D2
:107E50000CF451C04D845E846F84788827E137EB41
:107E600041ED58EBC301B2010F943FC787FD43C0FA
:107E700027E030E040E753E4C301B2010F94EDBDC9
:107E80001816CCF14D805E806F80788427E137EB47
:107E900041ED58EBC301B2010F943FC787FD2BC0E2
:107EA00027E030E040E753E4C301B2010F94EDBD99
:107EB00018160CF149805A806B807C8027E137EBE3
:107EC00041ED58EBC301B2010F943FC787FD13C0CA
:107ED00027E030E040E753E4C301B2010F94EDBD69
:107EE00018164CF0AE014F5F5F4FBE01635F7F4FCE
:107EF000C7010E94F53C68960FB6F894DEBF0FBE2E
:107F0000CDBFDF91CF911F910F91FF90EF90DF9048
:107F1000CF90BF90AF909F908F907F906F905F9029
:107F20004F903F9008954F925F926F927F928F9201
:107F30009F92AF92BF92CF92DF92EF92FF921F93E8
:107F4000CF93DF9300D01F92CDB7DEB719821A828C
:107F50001B821C82CE0101964C0187E8C82E8DE061
:107F6000D82E9CE6E92E9CE0F92E2BE7A22E2DE0E0
:107F7000B22E10E088E5810F0F94B542F401819391
:107F80004F01882341F00F9437422B013C0180912F
:107F90008714882359F0F60180819181A281B381F1
:107FA000F70180839183A283B38314C0812F0E9441
:107FB000DC37882309F4D0C0F60120813181428169
:107FC0005381C301B2010F94DFC4F7016083718351
:107FD000828393831F5FF4E0CF0ED11C84E0E80E10
:107FE000F11C94E0A90EB11C133021F685E40F9426
:107FF000B5428C83882309F4B9C00F9437426B01D2
:108000007C0183E00E94DC37882371F02091930D7E
:108010003091940D4091950D5091960DC701B60188
:108020000F94DFC46B017C01C092780CD092790C64
:10803000E0927A0CF0927B0C8091D309882359F15D
:1080400080911B1B82FF27C08C81882321F18981AD
:10805000811103C08A818823F1F02DEC3CEC4CE4C3
:108060005DE36091D20C7091D30C8091D40C90910F
:10807000D50C0F94DFC49B01AC0160918F0D709102
:10808000900D8091910D9091920D0F943FC718160D
:1080900014F40F945BAD40E050E0BA0186E40F9415
:1080A000C24220E030E0A9010F943FC7181684F4C3
:1080B0000F94374220E030E040E752E40F94D9C5F6
:1080C00060938702709388028093890290938A025A
:1080D0008091881483FD2CC080918714811128C061
:1080E0008091D00B882321F12091930D3091940D34
:1080F0004091950D5091960D6091780C7091790C8E
:1081000080917A0C90917B0C0F94DEC42091DD0B52
:108110003091DE0B4091DF0B5091E00B0F94DFC4E8
:108120006093DD0B7093DE0B8093DF0B9093E00B7D
:108130000F900F900F900F90DF91CF911F91FF90B4
:10814000EF90DF90CF90BF90AF909F908F907F90F7
:108150006F905F904F900895F501208131814281A9
:108160005381C301B2010F94DEC42FCF8091930DD0
:108170009091940DA091950DB091960D8093780CEF
:108180009093790CA0937A0CB0937B0C55CFCF923F
:10819000DF92EF92FF920F931F93CF93DF93CDB7B0
:1081A000DEB7A0970FB6F894DEBF0FBECDBF0E941A
:1081B000673B87FDD1C0482F61E081E00E9465C721
:1081C00085E40F946742882309F4D5C00F943742A1
:1081D0006B017C0120E030E0A9010F943FC787FFCD
:1081E00004C0F7FAF094F7F8F094F7FAF094F7F87F
:1081F000F094C98ADA8AEB8AFC8A8CE0E5E9F2E03D
:10820000DE01119601900D928A95E1F78AE50F94AF
:10821000B542882351F040E050E0BA018AE50F945E
:10822000C24269877A878B879C8788E50F94B5421D
:10823000882351F040E050E0BA0188E50F94C24233
:1082400069837A838B839C8389E50F94B542882365
:1082500051F040E050E0BA0189E50F94C2426D83CD
:108260007E838F83988785E50F946742882309F47E
:1082700089C00F9437426B017C0120E030E0A901F6
:10828000C701B6010F943FC787FF04C0F7FAF09407
:10829000F7F8F094F7FAF094F7F8F094CD8ADE8AC4
:1082A000EF8AF88E198E1A8E1B8E1C8E8CE40F941A
:1082B0006742882309F46FC00F9437426B017C0139
:1082C00020E030E0A901C701B6010F943FC787FF46
:1082D00004C0F7FAF094F7F8F094CD8EDE8EEF8EAE
:1082E000F8A262E070E082E40F94EE42F82E8091F2
:1082F000EC09811131C021E0AE014B5E5F4FBE0140
:108300006F5F7F4FCE0141960F945467882321F110
:108310006F2D81E00F94687E82E50F94B54288232B
:1083200009F442C00F94334240E050E060EA71E447
:108330004D875E876F87788B2091EC09222361F04F
:108340008C012F2DAE01435F5F4FBE01635E7F4FF7
:10835000CE0149960F944565A0960FB6F894DEBFFE
:108360000FBECDBFDF91CF911F910F91FF90EF9086
:10837000DF90CF900895C12CD12C80E8E82E80E4C6
:10838000F82E33CFC090CB09D090CC09E090CD0926
:10839000F090CE0972CFC090CF09D090D009E09074
:1083A000D109F090D2098CCF90E080E0BDCFCF9280
:1083B000DF92EF92FF920F931F93CF93DF93CDB78E
:1083C000DEB76C970FB6F894DEBF0FBECDBF8CE45E
:1083D0000F946742882309F4C3C00F9437426B019E
:1083E0007C0120E030E0A9010F943FC787FF04C063
:1083F000F7FAF094F7F8F094F7FAF094F7F8F094AD
:10840000C98EDA8EEB8EFC8E8CE0E5E9F2E0DE01BF
:10841000119601900D928A95E1F788E50F94B54287
:108420008823A1F040E050E0BA0188E50F94C242F1
:1084300020917B0D30917C0D40917D0D50917E0DF2
:108440000F94DEC469837A838B839C8389E50F94C0
:10845000B5428823A1F040E050E0BA0189E50F94CD
:10846000C24220917B0D30917C0D40917D0D509149
:108470007E0D0F94DEC46D837E838F8398878AE59B
:108480000F94B542882351F040E050E0BA018AE5EC
:108490000F94C24269877A878B879C87F0901B1B59
:1084A000F2FAFF24F0F840E061E080E00E9465C746
:1084B00060E080E50F94D942E82E1D861E861F8657
:1084C000188A8091EC0981113CC02E2DAE01435FCA
:1084D0005F4FBE016F5F7F4FCE0149960F94546787
:1084E000882379F18091D30981110F945BADFF202E
:1084F00011F0EE2031F160E080E00F94687E898D0C
:108500009A8DAB8DBC8DB0588D8B9E8BAF8BB88FF9
:10851000198A1A8A1B8A1C8A1D861E861F86188A3B
:108520008091EC09882369F010E000E020E0AE01C2
:108530004B5E5F4FBE016F5E7F4FCE010D960F9475
:1085400045656C960FB6F894DEBF0FBECDBFDF91C8
:10855000CF911F910F91FF90EF90DF90CF900895F2
:10856000C12CD12C80E8E82E80E4F82E45CFAF92C4
:10857000BF92CF92DF92EF920F931F93CF93DF932F
:108580005B01EA016901882309F463C08CE19CE086
:108590000F94BB4FF501608171818281938146E028
:1085A0000F94232EE1100BC083E19CE00F94BB4F8E
:1085B000688179818A819B8146E00F94232E8CE02B
:1085C0009CE00F94BB4FF6016081718182819381A1
:1085D00043E00F94232E85E09CE00F94BB4FF801FD
:1085E000608171818281938143E00F94232E8CEF0F
:1085F0009BE00F94BB4FF601208131814281538172
:10860000F80160817181828193810F94DEC443E01F
:108610000F94232EEE20F9F08AE00F94304F87EE6E
:108620009BE00F94BB4F688179818A819B8146E0F2
:108630000F94232E8AE00F94304F8AE0DF91CF9180
:108640001F910F91EF90DF90CF90BF90AF900D945E
:10865000304FE110E4CFDF91CF911F910F91EF9058
:10866000DF90CF90BF90AF900895CF93DF93CDB7B9
:10867000DEB720E2488559856F818E810F94729B09
:10868000DF91CF9108954FE350E0BC0189EE9BE06C
:108690000D94A0C963E972E084E690E00E94B6B050
:1086A0006AEB72E084E690E00C94B6B081110C9411
:1086B0004A4368EB71E084E190E00C94B6B00E940C
:1086C000E6F20C9456430F94A8390C9456430F9439
:1086D000F61C0C944A43282F1092500C8091400CA9
:1086E0009091410CA091420CB091430CB7FF08C08F
:1086F0001092400C1092410C1092420C1092430CBC
:1087000080911E09882331F08091400C8093440CA5
:1087100010923F0C80913E0C1816FCF4082E000CB1
:10872000990B821B91092091440C022E000C330BF3
:108730002817390794F097FF02C090E080E08093FB
:10874000440C092E000CAA0BBB0B8093400C909399
:10875000410CA093420CB093430C8091440C6623CF
:10876000A9F09091450C891714F48093450C209141
:10877000450C022E000C330B2C5F3F4F482F082E68
:10878000000C550B241735071CF484508093450CBE
:1087900008958F929F92AF92BF92EF92FF920F93A4
:1087A0001F93CF93DF93EC018B01E42EF22E809187
:1087B000CF1A9091D01A8C179D0709F440C02091D0
:1087C000030927FD109203092DEBC93ED20709F0DA
:1087D00041C0845F9C4571F40F94AFA26E517B4FF2
:1087E0008F4F9F4F60930509709306098093070987
:1087F00090930809D093D01AC093CF1A30E020E0AC
:108800000093400C1093410C2093420C3093430C86
:10881000E092450CF0923E0CC45FDC4531F41092BE
:1088200020091092040910921F0982E080937F02B0
:1088300081E080933F0C10921B0910921309DF9185
:10884000CF911F910F91FF90EF90BF90AF909F90AD
:108850008F9008952CE5C43FD20761F6895E9D4B49
:1088600019F0C4EFDCE5C6CF0F94AFA280900509E4
:1088700090900609A0900709B09008096819790935
:108880008A099B0997FFEDCF8091E40B87708730B1
:1088900041F7C9EED8E5AECF20E040E070E060E0FF
:1088A00084EF9CE50C94C9430F931F93CF93DF9300
:1088B000CDB7DEB76E970FB6F894DEBF0FBECDBF53
:1088C000282F082E000C330B90911C0240911D02A2
:1088D0008F3F39F0F901EE0FFF1FE25EFD4F9081EF
:1088E00041814F939F933F938F938FE998E19F939B
:1088F0008F938E010F5F1F4F1F930F930F9484BDB3
:10890000C8010E9443430E944C440FB6F894DEBF56
:108910000FBECDBF6E960FB6F894DEBF0FBECDBFB3
:10892000DF91CF911F910F910895CF930F94F61C73
:108930000E94E6F2C82F882319F080E00F9451328C
:108940008C2F0E945643CF910C944C44AF92BF920F
:10895000CF92DF92EF92FF920F931F93CF93DF930B
:10896000CDB7DEB764970FB6F894DEBF0FBECDBFAC
:108970000E94673BD82E87FDB5C08AE50F94B542AB
:10898000882309F4C0C040E050E0BA018AE50F94A2
:10899000C2427B018C014D2D63E085E00E9465C7DA
:1089A00020918F0D3091900D4091910D5091920D2D
:1089B00060E070E08AE793E40F94DEC45B016C0131
:1089C0009701A8010F943FC7181614F0750186018E
:1089D00020E030E0A901B701C8010F943FC7181685
:1089E00024F4E12CF12C00E010E0B701C8010F9451
:1089F0004BC6072E000C880B990B0F94F4BD6D83AA
:108A00007E838F83988720E030E0A9010F94EDBD2D
:108A1000882321F0CE0105960E942E3B80E090E055
:108A2000A0EAB1E489879A87AB87BC871D861E863A
:108A30001F86188A8CE40F946742882309F468C063
:108A40000F9437426B017C0120E030E0A901C7019F
:108A5000B6010F943FC787FF04C0F7FAF094F7F808
:108A6000F094C98ADA8AEB8AFC8A2091FB1930914A
:108A7000FC192430310574F08091F9199091FA199C
:108A8000821B930B97FF03C091958195910901E09B
:108A900004970CF400E063E080E00F94DA64811145
:108AA00040C083E08093210210921A090E944C4436
:108AB0006D817E818F8198858B019C01305809835F
:108AC0001A832B833C8320E030E0A9010F94EDBD95
:108AD000882321F0CE0101960E942E3B10921A09A4
:108AE0000E944C4464960FB6F894DEBF0FBECDBF13
:108AF000DF91CF911F910F91FF90EF90DF90CF907A
:108B0000BF90AF900895E12CF12C00E211E443CF27
:108B1000C090CF09D090D009E090D109F090D2094F
:108B200093CF83E0E82E22E0AE01475F5F4FBE01A6
:108B30006F5E7F4FCE010D960F94FC98B9CF809158
:108B4000991A90919A1A891B8F7011F40D94854C83
:108B500081E00895E0910409EE2389F0E150E0936B
:108B6000040988E0E89FF0011124EC53F74F62817B
:108B7000738127814681808191810C94C9430C9433
:108B80004C44E0910409E63010F581E08E0F8093AB
:108B900004094091400C5091410C6091420C70913D
:108BA000430C9091450C80913E0C28E0E29FF0012F
:108BB0001124EC53F74F2091CF1A3091D01A318302
:108BC00020834283538364837583968387830895C8
:108BD0002F923F924F925F926F927F928F929F92CD
:108BE000AF92BF92CF92DF92EF92FF920F931F93BB
:108BF000CF93DF9300D000D0CDB7DEB71C017A83CE
:108C000069832B833C834D835E832701380181E098
:108C100080933F0C0E94C14583E080937F02309295
:108C200002092092010989819A8190930009809319
:108C3000FF088B819C81AD81BE818093FB0890935E
:108C4000FC08A093FD08B093FE084092F7085092EC
:108C5000F8086092F9087092FA08F12CE12CC092A1
:108C6000400CD092410CE092420CF092430CB09236
:108C7000D01AA092CF1A9092F6088092F5088C8DA7
:108C80008093F40826960FB6F894DEBF0FBECDBFD2
:108C9000DF91CF911F910F91FF90EF90DF90CF90D8
:108CA000BF90AF909F908F907F906F905F904F900C
:108CB0003F902F900895CF93DF93CDB7DEB78E818D
:108CC0009091DF17891778F08093DF179E01275F57
:108CD0003F4F4F81588564E570E08AE897E10F9433
:108CE000B4BD10928917DF91CF9108950F931F9310
:108CF000CF93DF938C0167FF03C01092DF1760E012
:108D00002091DF17862F062E000C990B28171906C5
:108D100009F05CF56093DF1760E08DEE97E10F944A
:108D2000C94FC8010F94BB4F8AE00F94304FC80160
:108D30000F94FDBC800F911FEC01C01BD10BC535FA
:108D4000D1053CF00197FC012491207C2038D1F31F
:108D5000F3CFDD27AE01B8018AE897E10F941EBD7D
:108D6000C657D84E188210928917DF91CF911F9164
:108D70000F910895CF938091BC08811109C08AE4B6
:108D800098E190930A098093090981E08093BC08D7
:108D90000E94C14520E040E070E060E087E598E592
:108DA0000E94C943C1E0C09320090E9428F7109295
:108DB00020090E94AA45C09320094AE358E161E4D2
:108DC00078E184E00F94059A60E08DE298E10E94DA
:108DD000764640E061E080E00E9465C783E298E16A
:108DE0009093E80B8093E70BCF9108951092840C39
:108DF00010927E0280911B1B806480931B1B61E09C
:108E00008BEF97E10F94C94F40E158E168E178E1B9
:108E100085E00F94059A60E082E098E10E94764632
:108E20000C944C44CF93C82F0F94C04C81111AC09E
:108E300080911B1B82FF0CC080914717811105C0D8
:108E40008FE59CE0CF910D94948687E497E1FACF6B
:108E500080913609813061F08EEC97E1CC2321F0CE
:108E6000CF9108958DE298E16FEFCF910C94764603
:108E700081EE97E1F9CF80E00E9412471092840CB6
:108E800010927E020F94B24C882351F080911B1BEC
:108E900082FD06C08CE598E19093E80B8093E70B88
:108EA00061E085E598E10F94C94F0D943E230F933F
:108EB0001F930F94AFA20091B8081091B9082091A8
:108EC000BA083091BB08601B710B820B930B97FDA6
:108ED0000CC086B186FB882780F991E08927349BF6
:108EE0008260329B8460809361078091610781700A
:108EF0009091610791FD82609091B708981721F1D8
:108F00008130E1F120F1823051F1833069F19091AB
:108F100060079923B9F09091B608992399F0909140
:108F2000B60820911C0930911D09290F311D97FDAC
:108F30003A9530931D0920931C091092B60891E0D0
:108F400090937F028093B7081F910F9108959130FD
:108F500079F09230E1F69091B60891500CC09923C7
:108F600039F09330C1F3D3CF9130A9F3923079F631
:108F70009091B6089F5F9093B608C9CF992359F393
:108F8000933029F6F5CFCF92DF92EF92FF92CF93F5
:108F9000C82F0F94AFA26B017C0124EA30E74DE7A4
:108FA0005FE360912D0270912E0280912F029091CB
:108FB00030020F94EDBD87FD18C08AEF90E0A0E06D
:108FC000B0E08C0D9D1DAE1DBF1D8093AA0890932F
:108FD000AB08A093AC08B093AD08C0931B02CF912F
:108FE000FF90EF90DF90CF90089580E090E0DC015B
:108FF000E8CFCF9393E090937F02811110926107A5
:109000000F94AFA26C507E4F8F4F9F4F6093B80864
:109010007093B9088093BA089093BB0868E873E12D
:1090200082E090E00E94B6B0C6E0C15049F00F94D3
:10903000B02862E070E080E090E00F947CA2F5CF71
:10904000CF910895CF92DF92EF92FF920F931F93EB
:109050000F94AFA200917B0810917C0820917D08AD
:1090600030917E086B017C01C01AD10AE20AF30A32
:109070009701860137FD11C020917A082095209331
:109080007A086A547C4F8F4F9F4F60937B08709390
:109090007C0880937D0890937E0881E090917A0807
:1090A000911101C080E01F910F91FF90EF90DF9030
:1090B000CF9008950F940144882339F062E370E063
:1090C00080E090E00F94554CF5CF62E370E080E0D3
:1090D00090E00D94554C2F923F924F925F926F9279
:1090E0007F928F929F92AF92BF92CF92DF92EF9238
:1090F000FF920F931F93CF93DF93CDB7DEB7C9577E
:10910000D1090FB6F894DEBF0FBECDBF8EEA99E04D
:109110000F94BB4F87E00F94BE39811190C084E556
:109120000F94B542882329F00F94334281110E9495
:1091300091EE80E090E0A0E8BFE389839A83AB835F
:10914000BC838D839E83AF83B8878DEC9CECACE4AD
:10915000BEE389879A87AB87BC8780E090E0A0E276
:10916000B1E48D879E87AF87B88B8CE390E09A8BB4
:10917000898B8DEC90E09C8B8B8B8DEC9CECACEC1C
:10918000BEE38D8B9E8BAF8BB88F80E090E0A0EE1E
:10919000BFE3898F9A8FAB8FBC8F1BA61CA64AE9B1
:1091A00059E969E97EE38FE40F94C2426D8F7E8FA7
:1091B0008F8F98A360E083E40F94D94289A360E085
:1091C0008BE40F94D9428AA389E40F94B542312CE1
:1091D00010E000E08823C9F00F940F4290E01816C9
:1091E000190614F481E090E033243394380E232DD3
:1091F0002150330BC90126E0289FF001299FF00D73
:109200001124E55DF34F0281138182E40F94B5428E
:10921000882319F00F9433428C010115110559F17F
:10922000C80188978536910520F16CE870E080E8E8
:1092300099E00F9499528BE799E00F94BB4FC75870
:10924000DF4F0FB6F894DEBF0FBECDBFDF91CF91D9
:109250001F910F91FF90EF90DF90CF90BF90AF9054
:109260009F908F907F906F905F904F903F902F9046
:1092700008951A8B098B8CE40F94B5428823E1F092
:109280000F9437424B015C0189869A86AB86BC8677
:1092900020E030E0A9010F943FC787FD0AC020E01D
:1092A00030E040E050E4C501B4010F94EDBD181664
:1092B0001CF483E599E0C1CF81E50F9467428823D0
:1092C00031F180912E0790912F07892BE9F00F94AF
:1092D00037424B015C018D829E82AF82B8862DECB5
:1092E0003CEC4CE45DE30F943FC787FD0AC020E0EF
:1092F00030E040E751E4C501B4010F94EDBD18160C
:1093000034F482E299E099CF87EF98E096CF83E535
:109310000F94B5428823E9F00F9437424B015C016A
:109320008D8A9E8AAF8AB88E2DEC3CEC4CEC5DE3C6
:109330000F943FC787FD0AC020E030E040E050E4D2
:10934000C501B4010F94EDBD18161CF480ED98E032
:1093500074CF80E50F946742882341F080912E07F7
:1093600090912F07892B29F58FEF8BA786E40F9417
:10937000B542882309F43DC00F9437424B015C018C
:10938000898E9A8EAB8EBC8E20E030E040E85FE3A1
:109390000F943FC787FD0AC020E030E040E850E46A
:1093A000C501B4010F94EDBD18161CF58FE798E0C8
:1093B00044CF8BA58F5F8BA70F9437424B015C0185
:1093C0008D869E86AF86B88A20E030E0A9010F9492
:1093D0003FC787FD0BC020E030E048EC51E4C501F9
:1093E000B4010F94EDBD18160CF0C0CF88EA98E0D8
:1093F00024CF898C9A8CAB8CBC8C4D885E886F880E
:10940000788CA5019401C501B4010F9453BE9B0152
:10941000AC0160E070E084E490E40F94D9C5298148
:109420003A814B815C810F9453BE6B017C01A30197
:109430009201C301B2010F9453BEA50194010F9490
:1094400053BE2CEE31E548EB5DE30F94D9C59B018B
:10945000AC01C701B6010F9453BE69837A838B8335
:109460009C8310E000E0332069F0A32DA150BB0BDA
:1094700026E02A9FF0012B9FF00D1124E55DF34FAC
:109480000081118188E40F94B542882319F00F946C
:1094900033428C010115110559F0C801855A910913
:1094A0008F30914018F081E598E0C7CE1C8B0B8B74
:1094B00085E50F9467428823C9F00F94AFA2611528
:1094C00071058105910511F00F9436B980912E0731
:1094D00090912F07892BC9F00F9437426093680849
:1094E0007093690880936A0890936B0865E270E056
:1094F00082E50F94EE42E1969FAF8EAFE19718168A
:10950000190644F08DE198E098CE60E070E088E4C0
:1095100092E4E4CF89E50F94B542882381F10F945A
:10952000374220917F0D3091800D4091810D5091F7
:10953000820D0F94DEC46B017C0188E50F94B54267
:10954000882331F10F94374220917B0D30917C0DAF
:1095500040917D0D50917E0D0F94DEC46BA37CA3D2
:109560008DA39EA3CFA2D8A6E9A6FAA6CE01839684
:109570000F94E848811115C083EF97E05ECEC0904C
:109580008B0DD0908C0DE0908D0DF0908E0DD5CF81
:109590006091870D7091880D8091890D90918A0D51
:1095A000DDCF84E40F94674211E081270F94D14A04
:1095B00080E090E0A0EAB0E48DA79EA7AFA7B8AB8B
:1095C00060E0CE018D960F9412162091B00CEA96B1
:1095D0002FAFEA971092B00C0E94C3DD80EA97E0AB
:1095E0000F94BB4F89899A894A970CF094C063E61F
:1095F0008DE797E00E94764681E00E94F9478B89CB
:109600009C890E94AAF641E061E080E00F94C1309D
:10961000882309F494C080E00E94124781E00E94F0
:10962000F9471092930D1092940D1092950D10928F
:10963000960D83E99DE00F94CE081BA5112309F434
:10964000E2C020E030E040E751E46091B91470914D
:10965000BA148091BB149091BC140F94D9C5219673
:109660006CAF7DAF8EAF9FAF21971F3F09F024C332
:1096700081E08093600763E685ED97E00E9476467F
:1096800068E873E182E090E00E94B6B080E1E7E82C
:10969000FDE0ACE6BCE001900D928A95E1F7CE01C9
:1096A00001960F94E59AC12CD12C76010F940144B8
:1096B00081119DC068E873E182E090E00E94B6B03D
:1096C00020E030E040E85EE36091780C7091790C26
:1096D00080917A0C90917B0C0F94DFC46093780C8E
:1096E0007093790C80937A0C90937B0C20E030E09F
:1096F00040E85EE3C701B6010F94DFC46B017C0153
:1097000020E030E84BE354E40F943FC787FD5FC08F
:109710001092600714C063E680E997E00E947646E5
:1097200081E00E94F9471093600789899A890F9414
:10973000274061E081E00F943A2F811158CF6FEFFD
:1097400087EE97E00E9476468CA5811112C081E0D9
:109750008CA78D819E81AF81B885B0588DA79EA7BB
:10976000AFA7B8ABBE01635D7F4F8CE69CE00F9462
:109770001E4080E090E0A0EAB0E48093740C9093E7
:10978000750CA093760CB093770C1DA61EA61FA691
:1097900018AABE01635D7F4F8CE69CE00F941E40CB
:1097A000EA96BFADEA97B093B00C0E94C3DD109269
:1097B00060078AA1811143CD10929E0C10929D0CDE
:1097C0000E945BDE90E080E00E94AAF638CDCE01D8
:1097D000CD960F94A41480E1E7E8FDE0ACE6BCE090
:1097E00001900D928A95E1F70E9428F75FCF0E94C1
:1097F0005A4863E688EC97E00E94764681E00E9432
:10980000F94710926007E2E6F8E086E0DF011D927A
:109810008A95E9F780E1E7E8FDE0ACE6BCE001907D
:109820000D928A95E1F789859A85AB85BC858093F1
:10983000740C9093750CA093760CB093770C1DA6C6
:109840001EA61FA618AABE01635D7F4F8CE69CE092
:109850000F941E40BE01635E7F4F8CE69CE00F9428
:109860001E4081E08093600789A1882309F47BC2B0
:1098700088E0E7E8FDE0DE019D9601900D928A9573
:10988000E1F78FEF8DAF8EAFAE01435C5F4F66EFB8
:1098900077E3CE018D960F94AA49BE01635C7F4F9A
:1098A00082E698E00F94E84186E0FE01FD96DE0135
:1098B000A75ABF4F01900D928A95E1F786E0FE010D
:1098C000E75AFF4FDE01A15ABF4F01900D928A95D2
:1098D000E1F786E0FE01E15AFF4FDE01AB59BF4FD1
:1098E00001900D928A95E1F7CE018B599F4F0F940D
:1098F0001A44882309F4C8C1A6968FADA6970F9481
:10990000BC44762E872E982EA92E862F982DA92D11
:10991000BA2D65968CAF9DAFAEAFBFAF6597A796DA
:109920008FADA7970F9426446B017C016996CCAE4E
:10993000DDAEEEAEFFAE6997CE018F5A9F4F0F940A
:10994000E848882309F4A4C1A6966FACA697A79609
:10995000BFACA79720E030E040EA50E4672D782DB7
:10996000892D9A2D0F94DFC4162F072F382E292EFC
:10997000862F902FA32DB22D21968CAF9DAFAEAF29
:10998000BFAF21972596CCAEDDAEEEAEFFAE2597EC
:10999000611012C2B110EBC120E030E040EA50E4A7
:1099A000C701B6010F94DFC46B017C01BB2009F431
:1099B0008BC224E0172D082D392C2A2C2B150CF4E2
:1099C000F2C122ED422E23E5522E2BE7622E21E436
:1099D000722E21968CAC9DACAEACBFAC2197259677
:1099E0008CAD9DADAEADBFAD2597E9968CAF9DAF6B
:1099F000AEAFBFAFE9979C01AD0169966CAD7DAD8F
:109A00008EAD9FAD69970F94DEC4E5966CAF7DAFC8
:109A10008EAF9FAFE597A501940165966CAD7DADC6
:109A20008EAD9FAD65970F94DEC42D966CAF7DAF64
:109A30008EAF9FAF2D97E5968CAD9DADAEADBFAD12
:109A4000E59761968CAF9DAFAEAFBFAF6197A501B3
:109A500094016091870D7091880D8091890D90918E
:109A60008A0D0F94DEC4E5966CAF7DAF8EAF9FAFCD
:109A7000E597E9962CAD3DAD4EAD5FADE9976091B0
:109A80008B0D70918C0D80918D0D90918E0D0F949A
:109A9000DEC44B015C01812F902FA32DB22D8DA729
:109AA0009EA7AFA7B8ABC9AADAAAEBAAFCAAC98439
:109AB000DA84EB84FC84CDAADEAAEFAAF8AE2DEC02
:109AC0003CEC4CEC5CE3C301B2010F9453BE298122
:109AD0003A814B815C810F9453BE2091930D30915C
:109AE000940D4091950D5091960D0F94DFC469AF80
:109AF0007AAF8BAF9CAFE5962CAD3DAD4EAD5FAD73
:109B0000E597CA01B9010F9453BE2B013C01A50191
:109B10009401C501B4010F9453BE9B01AC01C30174
:109B2000B2010F94DFC420E030E040E050E40F9435
:109B30003FC71816ACF420E030E040E05FE3C70117
:109B4000B6010F94DFC429966CAF7DAF8EAF9FAF87
:109B50002997BE01635C7F4FCE0101960E94883C2D
:109B600089859A85AB85BC8529968CAF9DAFAEAFB4
:109B7000BFAF2997AF961CAE1DAE1EAE1FAEAF97FE
:109B8000BE0165597F4FCE01CD960F941E40CE0188
:109B900001960F94E59AE090B114F090B214009100
:109BA000B3141091B414A090AD14B090AE14C09042
:109BB000AF14D090B0149501A601B701C8010F945D
:109BC0003FC7181614F475018601809087029090A3
:109BD0008802A0908902B0908A022DEC3CEC4CECFB
:109BE0005DE3B701C8010F9453BE60938702709381
:109BF00088028093890290938A0240E0BE01675BED
:109C00007F4FCE018D960F942EA380E1E7E8FDE013
:109C1000ACE6BCE001900D928A95E1F78092870254
:109C200090928802A0928902B0928A020F9407440F
:109C3000811185CD20E04FEFBE016B597F4FCE01E2
:109C400001960E944B3E20E041E0BE016B597F4FE0
:109C5000CE0101960E944B3E2FEF40E0BE016B59B2
:109C60007F4FCE0101960E944B3E21E040E0BE01B5
:109C70006B597F4FCE0101960E944B3E0E9428F700
:109C80000F94074481115BCD8091D3148093D41439
:109C9000E196AEADBFADE1971197E196BFAFAEAF24
:109CA000E197AB2B09F44BCDCE018B599F4F0F940D
:109CB0001A448111D9CD43CD63E685EB97E00E942C
:109CC000764681E00E94F94780E1E7E8FDE0ACE6F6
:109CD000BCE001900D928A95E1F72D853E854F8578
:109CE00058896091780C7091790C80917A0C9091E0
:109CF0007B0C0F94DFC46093780C7093790C809385
:109D00007A0C90937B0CCE01CD960F94A4142D85E4
:109D10003E854F8558896091780C7091790C8091BF
:109D20007A0C90917B0C0F94DEC46093780C709346
:109D3000790C80937A0C90937B0C8CA5811163CD68
:109D400081E08CA78D819E81AF81B885B0588DA7A9
:109D50009EA7AFA7B8ABBE01635D7F4F8CE69CE0CA
:109D60000F941E4050CD88E0FE01B39684CD872D20
:109D7000982DA92DBA2D21968CAF9DAFAEAFBFAF58
:109D8000219720E030E040EA50E4C701B6010F948B
:109D9000DEC425966CAF7DAF8EAF9FAF2597B4E044
:109DA000BB150CF0F9CD92ED492E93E5592E9BEFA2
:109DB000692E90E4792E0DCE34E036150CF056C0A5
:109DC00062961FAD629763960FAD639764963FAC42
:109DD000649765962FAC65973B15FCF420E030E066
:109DE00040EA50E4672D782D892D9A2D0F94DEC41A
:109DF00021966CAF7DAF8EAF9FAF219720E030E012
:109E000040EA50E4C701B6010F94DEC46B017C0147
:109E100084E08B150CF0D5CDC6CF872D982DA92DBC
:109E2000BA2D21968CAF9DAFAEAFBFAF219720E08A
:109E300030E040EA50E4C701B6010F94DFC4259634
:109E40006CAF7DAF8EAF9FAF2597B110D7CF20E01D
:109E500030E040EA50E4612F702F832D922D0F9453
:109E6000DEC4162F072F382E292E9DCFB1100FC01C
:109E700020E030E040E251E4612F702F832D922DDD
:109E80000F94DEC4162F072F382E292E9ACD94E07A
:109E900082ED482E83E5582E8BEF682E81E4782ED4
:109EA0009B150CF096CD20E030E040E251E4612FAC
:109EB000702F832D922D0F94DEC421966CAF7DAF51
:109EC0008EAF9FAF21977DCD172D082D392C2A2CD1
:109ED0006ACFFC0180E09491992331F0907C903816
:109EE00009F08F5F3196F7CF0895FC0180E09191E2
:109EF000992329F0907C9038D1F38F5FF8CF0895A3
:109F0000AF92BF92CF92DF92EF92FF920F931F9387
:109F1000CF93DF93EC015B018A01FB01199587FD6B
:109F200016C0C82ED12CF12CE12C2196F801C0824C
:109F3000D182E282F382CE01DF91CF911F910F9106
:109F4000FF90EF90DF90CF90BF90AF900895982F43
:109F5000907E903CA9F48F7190E0B0E0A0E06C019D
:109F60007D0156E0CC0CDD1CEE1CFF1C5A95D1F790
:109F7000CE010196F50119958F73C82A2296D6CF86
:109F8000982F907F903E11F58F7090E0B0E0A0E0A8
:109F90006C017D0136E0CC0CDD1CEE1CFF1C3A95FB
:109FA000D1F7CE010196F50119958F73C82A46E0C5
:109FB000CC0CDD1CEE1CFF1C4A95D1F7CE0102969D
:109FC000F50119958F73C82A2396B0CF982F987FE3
:109FD000903F79F5877090E0B0E0A0E06C017D01E2
:109FE00086E0CC0CDD1CEE1CFF1C8A95D1F7CE015F
:109FF0000196F50119958F73C82A96E0CC0CDD1CEB
:10A00000EE1CFF1C9A95D1F7CE010296F501199529
:10A010008F73C82A26E0CC0CDD1CEE1CFF1C2A9591
:10A02000D1F7CE010396F50119958F73C82A2496AE
:10A030007DCF982F907C903841F4807C803869F4F3
:10A040002196CE01F5011995F8CF8E7F8D3F28F02E
:10A050002196CE01F5011995F8CFC12CD12C7601AE
:10A0600065CF8F929F92AF92BF92CF92DF92EF9285
:10A07000FF920F93FC01C080D180E280F38080903A
:10A08000760890907708A0907808B0907908A5019C
:10A090009401C701B6010F94EDBD8823E9F020E0DB
:10A0A00030E0A901C701B6010F94EDBD882309F482
:10A0B00084C0A5019401C701B6010F94EDBD87FDD1
:10A0C0007EC081E080937508C0927608D0927708B0
:10A0D000E0927808F09279088091091B813198F418
:10A0E00080910B1B833078F08091750844E0481B09
:10A0F00054E4E52E56E1F52E0CE022E062E485ED15
:10A100009AE10F94C2AB8091091B853180F4809154
:10A110000B1B843160F041E4E42E46E1F42E01E0B3
:10A1200023E044E16CE385ED9AE10F94C2AB8091AA
:10A13000091B8F33C0F580910B1B8F32A0F18091EA
:10A14000750840E3481B87E2E82E86E1F82E0DE013
:10A1500022E06AE585ED9AE10F94C2AB8091750823
:10A1600041E3481B9DE0E92E96E1F92E22E065E0EF
:10A1700085ED9AE10F94C2AB2DEDE22E25E1F22E92
:10A1800000E123E04FE262E185ED9AE10F94C2AB7A
:10A190003DEAE32E35E1F32E23E04FE267E685ED5D
:10A1A0009AE10F94C2AB0F91FF90EF90DF90CF90A8
:10A1B000BF90AF909F908F90089580E083CF8FEFF6
:10A1C00081CF9CE0899F802D112491E0980F90937E
:10A1D00019092CE0280F2093590C30E02E5F3F4FD7
:10A1E0004091091B4217130619F014F080E00895FE
:10A1F00020910B1B9217D0F7662341F08E5F0F94CE
:10A2000070A98091590C8E5F0F9470A98091590CA0
:10A210009091091B891750F320910B1B90911909FC
:10A22000291720F310920C1B80930D1B81E00895D9
:10A2300020917208022E000C330B8217130641F096
:10A24000809372086FEA78E185ED9AE10D9456AA41
:10A2500008951F93CF93DF931F92CDB7DEB78F3F43
:10A26000910519F014F08FEF90E08837910514F400
:10A2700088E790E09093560280935502182F8091C2
:10A280000E1B811105C081E080930E1B0F9497A8CF
:10A290006091D71A7091D81A19839E012F5F3F4F92
:10A2A0004FE085ED9AE10F9493A80F90DF91CF9145
:10A2B0001F910895CF938091730881114FC0109220
:10A2C0000C1B10920D1B10920E1B1092DA1A10929A
:10A2D000D91A1092DC1A1092DB1A1092DE1A81E061
:10A2E0008093DD1A82E28093DF1A1092E41A1092B2
:10A2F000E31AE8EFFAE126E03BE18FEF81932E17B6
:10A300003F07E1F7C1E0C093F51A29E932E0309345
:10A31000EB1A2093EA1AC093EC1A1092ED1A1092DD
:10A32000EE1A90E49093EF1A1092F01A2FEE32E0AA
:10A330003093071B2093061B23E132E03093D81A99
:10A340002093D71A99E19093FA1A9BE19093F91A06
:10A350008093F81A0F9497A8C093730880915502C0
:10A36000909156020E94295181E0809374088DEAF1
:10A3700095E19093EC198093EB191092EE191092DD
:10A38000ED19CF9108950E945A513E98469A3C98F3
:10A39000449A3A98429A0E9457471092B6080895F4
:10A3A000CF92DF92EF92FF920F931F93CF93DF93A1
:10A3B000CDB7DEB72C970FB6F894DEBF0FBECDBF7A
:10A3C0006F3F71058105910509F0D0F481ED9AE1A7
:10A3D0000E945239E091D91AF091DA1A319684919B
:10A3E00090E02C960FB6F894DEBF0FBECDBFDF9184
:10A3F000CF911F910F91FF90EF90DF90CF90089534
:10A40000F0900C1BE0900D1B2091740821110FC0DF
:10A410004DE855E16E2D8F2D0F941AAB90E080E042
:10A42000F80EF0920C1BE0920D1B9927DACFC0902A
:10A43000D91AD090DA1A25ED3AE13A8329832F2DE3
:10A4400030E03C832B832E2D30E03E832D83188615
:10A450001F822FEF3FEF3A8729871C861B8600EF6C
:10A4600018E39E012F5F3F4FAB01BC01C6010F9463
:10A47000D081B60185ED9AE10F9456AA8F81988517
:10A48000CFCF4F925F926F927F928F929F92BF92A7
:10A49000CF92DF92EF92FF920F931F93CF93DF93B0
:10A4A00000D000D01F921F92CDB7DEB77C016A01A9
:10A4B0004901FB0190818CE0989F800D1124982F19
:10A4C000F7012081822F880F820F880F80930C1B49
:10A4D00090930D1B4115510571F1FA82E9827C833D
:10A4E0006B83011121C0AE014B5F5F4FB401C60108
:10A4F0000E94804F6C016D817E818F8198856115EE
:10A50000710581059105B9F00E94D051F701808154
:10A510008F5F8083853138F3CE0101960E94C0376A
:10A52000E2CFB12C860129C08A01B12C26C0452872
:10A5300046284728B1F728960FB6F894DEBF0FBE1D
:10A54000CDBFDF91CF911F910F91FF90EF90DF90E2
:10A55000CF90BF909F908F907F906F905F904F9023
:10A560000895B39407C0B1102EC001151105C9F2AA
:10A570000F5F1F4F01151105A9F2AE014B5F5F4F31
:10A58000B401C6010E94804F6C014D805E806F80D7
:10A5900078844114510461047104A9F0F0E24F166B
:10A5A000510461047104F9F2D301C2018D97A1092C
:10A5B000B1090297A105B10530F04BE244165104F0
:10A5C0006104710471F6F7018081482F4B0D552706
:10A5D000551F4631510534F0853020F0CE010196EB
:10A5E0000E94C03781E0411451046104710409F4F0
:10A5F00080E0B80EF70180818B0D8083BB2009F4C9
:10A6000096CFBA94AE014B5F5F4FB401C8010E9470
:10A61000804F8C016D817E818F8198850E94D05101
:10A62000EDCF2F923F924F925F926F927F928F92D7
:10A630009F92AF92BF92CF92DF92EF92FF920F93D1
:10A640001F93CF93DF9300D0CDB7DEB74C013B0112
:10A650005A01222E3B8328014091400C5091410C1D
:10A660006091420C7091430C4115510561057105D3
:10A6700079F081E0141615060CF080E08093130940
:10A680001092400C1092410C1092420C1092430C0C
:10A690001091130930903D0C10923D0C311005C003
:10A6A00080917F02882309F472C0C2010E94694F21
:10A6B000082F80E0C114D10419F0C6010E94694F2F
:10A6C0001A821982E114F104B1F4402F50E0282FCE
:10A6D00030E0CA01820F931F46976CF485E190E049
:10A6E000841B950B821B930B97FD0196959587957F
:10A6F0008A8381E0898301E02AEB37E3A201BE016E
:10A700006F5F7F4FCE0102960E944152E114F10427
:10A7100091F08A81882321F01A8289818F5F898351
:10A7200000E02DEB37E3A701BE016F5F7F4FCE0145
:10A7300002960E944152C114D10459F000E02AEB64
:10A7400037E3A601BE016F5F7F4FCE0102960E94E4
:10A75000415241E04127B30181E00F94EDA9C401CA
:10A760000E94694F412FB40194E1981B892F0F94E7
:10A77000EDA9332049F0111102C0A22CBB80A11415
:10A78000B104D9F0F501199581E0809320090F906B
:10A790000F900F90DF91CF911F910F91FF90EF904D
:10A7A000DF90CF90BF90AF909F908F907F906F90F1
:10A7B0005F904F903F902F9008950E94AA45E4CF5C
:10A7C000AF92BF92CF92DF92EF92FF920F931F93BF
:10A7D000CF93DF9300D01F92CDB7DEB77C01062F59
:10A7E0006A01122F86E0A82EB12C11160CF040C081
:10A7F000AE014F5F5F4F6AEB77E3C7010E94804F66
:10A800007C0169817A818B819C816115710581054B
:10A81000910571F16D3371058105910509F450C001
:10A820006E3771058105910509F44AC06A327105D8
:10A830008105910569F507FF12C082EA96E10E3F96
:10A8400011F08EE996E126E01202B00111240E9477
:10A85000B63A66E070E00F94C2C4161B61C065E4AE
:10A8600070E080E090E00E94D051115059F510E066
:10A87000812F0F900F900F900F90DF91CF911F912C
:10A880000F91FF90EF90DF90CF90BF90AF90089521
:10A89000643271058105910579F4C114D10461F028
:10A8A00026E01202B0011124C6010E94B63AB50199
:10A8B0000F94C2C4161B99CF0E94D051115095CF4E
:10A8C00007FDBBCF61E089819A81AB81BC81CD97C7
:10A8D000A105B10509F460E0600F6A30ACF01150D9
:10A8E000862F6AE00F94A0C4092F682F880F770B7A
:10A8F000605D7F4F072E000C880B990B0E94D05192
:10A90000112309F4B4CF602F062E000C770B605D85
:10A910007F4F072E000C880B990B0E94D0511150CD
:10A92000112309F4A4CF86E01802B0011124C70155
:10A930000E94B63A66E070E00F94C2C4161B98CF2E
:10A940006FEF7FEF0C94B63ACF93DF93FC0125AD08
:10A95000211104C021E025AF0F9497A8C091D71A08
:10A96000D091D81AE091061BF091071B82E019954F
:10A97000E091061BF091071B81E0199530E020E083
:10A9800044E1BE0185ED9AE10F9493A828E03BE1F4
:10A9900047E1BE0185ED9AE10F9493A8E091061B73
:10A9A000F091071B80E0DF91CF9119944F925F9255
:10A9B0006F927F928F929F92AF92BF92CF92DF92CF
:10A9C000EF92FF920F931F93CF93DF9300D01F92CC
:10A9D000CDB7DEB70F94AFA26B017C0180911B0253
:10A9E0008F3FF1F10F94AFA28090AA089090AB082E
:10A9F000A090AC08B090AD08681979098A099B0944
:10AA000097FD2EC08091991A90919A1A8F5F8F703E
:10AA1000891731F1E0911B0280E090E0A8E4B3E4F3
:10AA2000E43050F424E0E29FF0011124E355FD4F9F
:10AA300080819181A281B38189839A83AB83BC8316
:10AA40008E010F5F1F4F23E93DE04FE85DE06BE8AB
:10AA50007DE087E89DE00F947E978FEF80931B0247
:10AA60000E94574780916007811116C00F940144DE
:10AA7000882391F08091B508811110C091E09093E6
:10AA8000B5088091840C892780933D0C1092840C2A
:10AA900081E00E94F94702C01092B50880915C07DE
:10AAA00090915D07A0915E07B0915F07A7019601A5
:10AAB000281B390B4A0B5B0BDA01C901B7FF05C034
:10AAC00080911B09882309F4EAC1D701C6018C597A
:10AAD0009F4FAF4FBF4F80935C0790935D07A0934C
:10AAE0005E07B0935F076091B608062E000C770BE7
:10AAF00077FF03C07195619571099091B6088091B7
:10AB0000B408981302C0633068F0633069F4809130
:10AB1000B60887FD6BC081E0880F880F8093B60868
:10AB200064E002C01092B6088091B6088093B40821
:10AB3000643008F05DC080913D0C8111DBC08091D4
:10AB4000CF1A9091D01A3CE5843F930709F0F6C0E4
:10AB500080918002882309F4DFC0815080938002B5
:10AB60000E9453FA8090C00D9090C10DA090C20D2C
:10AB7000B090C30D81110F94384CD501C4013AE057
:10AB8000B695A795979587953A95D1F7009751E097
:10AB9000A507B10520F08FEF9FEFA0E0B0E09695FC
:10ABA000879520917F022111F8C030911B09311146
:10ABB000A4C18091CF1A9091D01A845F9C4509F46A
:10ABC00083C18091200981117FC18091B00890914B
:10ABD000B108A091B208B091B308C81AD90AEA0A1C
:10ABE000FB0AF7FC7FC10E944C447CC18FEF94CFDD
:10ABF0008091500C21E030E040E050E0882309F4DF
:10AC000056C080904C0C90904D0CA0904E0CB09083
:10AC10004F0C81149104A104B104E9F170E090E0BB
:10AC200080E00F94F2BD20E030E040E85EE30F9456
:10AC300053BE2B013C01C701B601681979098A0985
:10AC40009B090F94F2BD9B01AC01C301B2010F94AB
:10AC5000D9C520E030E04AE754E40F9453BE4B01DD
:10AC60005C0120E030E042E053E40F943FC724E66B
:10AC700030E040E050E087FF12C020E030E040EAE2
:10AC800052E4C501B4010F943FC72AE030E040E030
:10AC900050E087FF04C021E030E040E050E0C09287
:10ACA0004C0CD0924D0CE0924E0CF0924F0CA091B7
:10ACB000B6080A2E000CBB0B0F947DC424E030E0D4
:10ACC00040E050E00F9453C48091400C9091410CAF
:10ACD000A091420CB091430C820F931FA41FB51F8B
:10ACE0008093400C9093410CA093420CB093430C82
:10ACF0001092B608D701C6018856954CAF4FBF4F8A
:10AD00008093B0089093B108A093B208B093B308B1
:10AD100081E080937F0213CF8CE08093800280914A
:10AD2000AE089091AF08009729F001979093AF0873
:10AD30008093AE0881E080937F0212CF86529C4BB5
:10AD400009F00ECF809180029FEF980F90938002C0
:10AD5000811106CF80915D0C8F5F80935D0C909187
:10AD60005E0C24E0891708F02CE0209380029817ED
:10AD700010F410925D0C81E080937F02D701C60130
:10AD80008856954CAF4FBF4F8093B0089093B10851
:10AD9000A093B208B093B308E3CE009741F040917E
:10ADA000AE085091AF084817590708F002CF8091BC
:10ADB0001B09811112C0223038F0243008F441C040
:10ADC000243011F410927F0281ED9AE10E94A45484
:10ADD00081E080931E0980931B0983E00E94185133
:10ADE00081E08093F51AE091CF1AF091D01A19956D
:10ADF00010921E0980911B09811127C010923D0CF1
:10AE00008091CF1A9091D01A845F9C4509F0D9CED9
:10AE10000F94AFA2DC01CB018C199D09AE09BF09CB
:10AE20008090AE089090AF08B12CA12C881699069E
:10AE3000AA06BB0608F0BDCE9093AF088093AE087B
:10AE4000B8CE81E080937F02BFCF85ED9AE10F9469
:10AE500024AA91E0811101C090E090931B098823FE
:10AE600069F28091CF1A9091D01A845F9C45B9F411
:10AE70000F94AFA2DC01CB018C199D09AE09BF096B
:10AE8000C090AE08D090AF08F12CE12CC816D906BE
:10AE9000EA06FB0620F49093AF088093AE080F906B
:10AEA0000F900F900F90DF91CF911F910F91FF9016
:10AEB000EF90DF90CF90BF90AF909F908F907F905A
:10AEC0006F905F904F90089558E9C50E5AE3D51ED4
:10AED000E11CF11CC092B008D092B108E092B20817
:10AEE000F092B30880911B098111D9CF80917F0224
:10AEF0008130A9F610927F02D2CF009709F46DCF6E
:10AF00004ECFCF92DF92EF92FF920F931F93CF938A
:10AF1000DF93CDB7DEB72C970FB6F894DEBF0FBE28
:10AF2000CDBFF0900C1BE0900D1B209174082111F7
:10AF30001DC04DE455E16E2D8F2D0F941AAB90E09E
:10AF400080E0F80EF0920C1BE0920D1B99272C96D6
:10AF50000FB6F894DEBF0FBECDBFDF91CF911F912A
:10AF60000F91FF90EF90DF90CF900895C090D91A85
:10AF7000D090DA1A25ED3AE13A8329832F2D30E07B
:10AF80003C832B832E2D30E03E832D8318861F8239
:10AF90007A8769871C861B8600EF18E39E012F5F66
:10AFA0003F4F4DEB57E3BC01C6010F949482B601AD
:10AFB00085ED9AE10F9456AA8F819885C2CFBF92F2
:10AFC000CF92DF92EF92FF920F931F93CF93DF9375
:10AFD0008B01F42EE90141FB662760F90E94E150E4
:10AFE000882309F45AC0B12C0115110521F0C801BC
:10AFF0000E94694FB82EE12C209721F0CE010E94CB
:10B00000754FE82E80E8C82ED12CF0FE1EC085E1D9
:10B0100090E08B199109B7FC93958E199109E7FC83
:10B02000939597FD019695958795F82E30E8C32E58
:10B03000D12CFA94F7FC09C060E270E080E090E067
:10B040000E94D051C81AD90AF4CFBB2099F0C6018A
:10B0500066E070E00F94AEC4262F40915B0C5091D7
:10B060005C0C60915A0CC8010E94E05396E0899FE5
:10B0700060011124EE2031F0B601CE010E9481570B
:10B08000C81AD90A87E0C816D10438F060E270E027
:10B0900080E090E00E94D051F3CFDF91CF911F91DB
:10B0A0000F91FF90EF90DF90CF90BF900895809127
:10B0B0007F02882351F06091090970910A0930E0FC
:10B0C00020E041E081E00C94DF5708956FEF7FEFBF
:10B0D0000C948157AF92BF92CF92DF92EF92FF9282
:10B0E0000F931F93CF93DF935C016B010E94694F15
:10B0F000E82EC6010E94754FF12C03E110E0081BF9
:10B100001109C5E20E151F050CF4CFE18C2F90E05C
:10B110009C012E5F3F4F4091091B4217130609F017
:10B12000CCF5099720910B1B281719069CF140912B
:10B130005B0C50915C0C60915A0C10920C1BC093EC
:10B140000D1B25E1C5010E94E053D1E0C114D104DB
:10B15000B1F06AE370E080E090E00E94D0510E15FB
:10B160001F05D4F4C45F8091091BC81740F02091DB
:10B170000B1B4C2F4950550B241715067CF4DF91FF
:10B18000CF911F910F91FF90EF90DF90CF90BF90E4
:10B19000AF900895D0E0DACFDD2389F3802F880FB8
:10B1A000080F000F00930C1BC0930D1B60E270E0B2
:10B1B00080E090E00E94D051C601DF91CF911F91B5
:10B1C0000F91FF90EF90DF90CF90BF90AF900C94D5
:10B1D0006658CF92DF92EF92FF92CF93DF938091E8
:10B1E0003D0C10923D0C882351F010922009DF9104
:10B1F000CF91FF90EF90DF90CF900C94AA4581E023
:10B20000809320098091400C9091410CA091420CB8
:10B21000B091430C0097A105B10509F44BC02AE099
:10B22000289FE001299FD00D11241092400C10920C
:10B23000410C1092420C1092430CBE010D2E000CDA
:10B24000880B990B0F94F4BD2091CE0D3091CF0D4A
:10B250004091D00D5091D10D0F9453BE2091901A72
:10B260003091911A4091921A5091931A0F94DFC421
:10B270006B017C0120E030E040E151EC0F943FC7CE
:10B2800087FD18C020E030E040E151E4C701B6017D
:10B290000F94EDBD181674F0CE010F94E8A2C09281
:10B2A000901AD092911AE092921AF092931A82E038
:10B2B00080937F0280917F02882399F080E99AE150
:10B2C0000F94B39BBC0180E698E10E946A5880E924
:10B2D0009AE1DF91CF91FF90EF90DF90CF900C94A7
:10B2E0003150DF91CF91FF90EF90DF90CF90089594
:10B2F0000F931F93CF93DF93FC01EB018091400CE0
:10B300009091410CA091420CB091430CB7FF08C042
:10B310001092400C1092410C1092420C1092430C6F
:10B320008091F7089091F808A091F908B091FA0877
:10B330004091400C5091410C6091420C7091430C33
:10B3400084179507A607B70744F48093400C9093A1
:10B35000410CA093420CB093430C80917F02882350
:10B36000E1F06091400C7091410C8091420C909101
:10B37000430C0091FB081091FC082091FD083091CE
:10B38000FE08600F711F821F931F1995BC018091E9
:10B390000109909102090E946A5880913D0C811127
:10B3A00008C08091F4088823D1F180917F0288231E
:10B3B000B1F18091FF08909100090097B1F04091A0
:10B3C000400C5091410C6091420C7091430C0091E3
:10B3D000FB081091FC082091FD083091FE08400FF9
:10B3E000511F621F731FFE011995E091F508F0913E
:10B3F000F608309741F08091F408811103C08091E4
:10B400003D0C8111199580913D0C10923D0C8823C3
:10B4100031F0DF91CF911F910F910C94AA45DF91EC
:10B42000CF911F910F9108958F929F92AF92BF92EB
:10B43000CF92DF92EF92FF920F931F93CF93DF9300
:10B44000CDB7DEB72C970FB6F894DEBF0FBECDBFD9
:10B45000982F862F5A017901D02E692F0E94E15032
:10B46000882309F487C010917408C701002381F173
:10B470000E94694FC82E8090D91A9090DA1A111143
:10B4800043C01FEF23E12C1940915B0C50915C0CE1
:10B4900060915A0CC5010E94E053CC2009F46AC0A7
:10B4A000B6E08B9F500111246AE370E080E090E0E9
:10B4B0000E94D05157E0A516B10408F442C060E2E2
:10B4C00070E080E090E00E94D051A81AB90AF2CF53
:10B4D0000E94754FC82E8090D91A9090DA1A1123C5
:10B4E00081F2FE0133968AE0DF011D928A95E9F729
:10B4F00085ED9AE19A83898307EC18E39E012F5F1B
:10B500003F4F4DEB57E312C0FE0133968AE0DF0157
:10B510001D928A95E9F785ED9AE19A83898307EC74
:10B5200018E39E012F5F3F4F4AEB57E3B701C40179
:10B530000F949482B40185ED9AE10F9456AA1F816D
:10B54000A1CF4091590C212F30E0A6E0CA9EC00146
:10B5500011242E5F3F4F281739070CF49C0180E817
:10B56000821B80930C1B40930D1BC701DD20A9F0AB
:10B570000E94A0542C960FB6F894DEBF0FBECDBF2C
:10B58000DF91CF911F910F91FF90EF90DF90CF90BF
:10B59000BF90AF909F908F9008950E946658EACF19
:10B5A0002F923F924F925F926F927F928F929F92D3
:10B5B000AF92BF92CF92DF92EF92FF920F931F93C1
:10B5C000CF93DF9300D000D0CDB7DEB761E081E04C
:10B5D0000E946B438091450C8D83582E8B5F89832D
:10B5E0004424439473E0372EE3EC6E2EEDED7E2E73
:10B5F00082E085198A83942D95199B83852D8195E9
:10B600008C83232C25188D81811181C08091440C5D
:10B61000882309F455C080917F02882359F081E086
:10B620009091440C911180E024E04FE25FE16C8145
:10B630000F94729B8091B00C882309F435C18D81E1
:10B64000833009F05CC18091440C833009F4CDC093
:10B6500080917F0281110EC194E09E838E818F5F65
:10B660009D81891322C08091440C891709F47FC100
:10B6700080917F028823C9F011E08091440C9D8164
:10B68000891310E06091CF097091D0098091D109A0
:10B690009091D2090E94AFC700E09C014FE658E1AB
:10B6A0006D816519812F0E94145A8D818F5F8D8362
:10B6B00099818913A8CF8E818E5F80933E0C0EC036
:10B6C00080913D0C10923D0C882309F4A4CF0E9478
:10B6D000AA4580913F0C882309F49DCF26960FB68A
:10B6E000F894DEBF0FBECDBFDF91CF911F910F91B8
:10B6F000FF90EF90DF90CF90BF90AF909F908F9092
:10B700007F906F905F904F903F902F9008959D8114
:10B710009130A1F58091440C8130F9F080917F0245
:10B72000882309F487CF81E08E838091440C813097
:10B7300009F01E826091BC0D7091BD0D8091BE0D0F
:10B740009091BF0D0E9474C600E09C0145E958E14C
:10B750006B818E810E94145A6DCF80913D0C1092A6
:10B760003D0C8823D9F26CEB7DE085E998E10F94DC
:10B77000919E80913F0C882389F2B0CF9D819230B9
:10B7800009F058CF8091440C8230C1F080917F0243
:10B79000882309F44FCF81E09091440C923009F056
:10B7A00080E09091B00C2AE43EE1911102C026E4C1
:10B7B0003EE101E04BE858E16A81CCCF8091B00CCA
:10B7C00090913D0C10923D0C992301F384258093B8
:10B7D000B00C30927F026114710411F00E94C3DD3D
:10B7E00080913F0C882391F279CF80913D0C10928B
:10B7F0003D0C882309F42CCF0F94CD9C20E030E041
:10B800004AE754E46091AC0C7091AD0C8091AE0CA1
:10B810009091AF0C0F9453BE20E030E0A9010F943B
:10B82000DFC420E030E84BEB54E40F94DEC40F9407
:10B8300052C61F9243EC842E4DED942E5EE4A52E4D
:10B8400056E9B52E6B0116EDE12E16E0F12E00E063
:10B8500010E02CED35E040E050E06CEA7CE081E85F
:10B8600098E10E94E8450F9080913F0C882309F4ED
:10B87000EFCE34CF81E08E838091440C833009F089
:10B880001E826091AC0C7091AD0C8091AE0C9091C9
:10B89000AF0C0E94F0C700E09C0141E858E1622D26
:10B8A0008E810E94145AD8CE83E08E838E819D8132
:10B8B0008913D4CE8091440C9E81891719F180910F
:10B8C0007F02882309F4CACEFD80F51811E080912B
:10B8D000440C9D81891310E06091CB097091CC09D3
:10B8E0008091CD099091CE090E94AFC700E09C01E4
:10B8F00047E758E16F2D812F0E94145AAFCE94E094
:10B900009E83D4CF80913D0C10923D0C8823B9F2D8
:10B910000F94CD9C20E030E0A9016091CB0970919B
:10B92000CC098091CD099091CE090F94DFC40F947A
:10B9300052C61F92912C812C28E4A22E26E9B22E09
:10B940006B011EEEE12E12E0F12E00E010E020E08F
:10B9500030E0A9016BEC79E087E798E10E94E845C7
:10B960000F9080913F0C882309F4A9CFB7CE809126
:10B970003D0C10923D0C882309F47ACE0F94CD9C97
:10B9800020E030E0A9016091CF097091D009809149
:10B99000D1099091D2090F94DFC40F9452C61F921F
:10B9A000912C812C88E4A82E86E9B82E6B011EEE1E
:10B9B000E12E12E0F12E00E010E020E030E0A901DD
:10B9C0006FEC79E08FE698E10E94E8450F90809156
:10B9D0003F0C882309F44CCE81CEE1EDFAE183AF30
:10B9E00064AFCA010C9466584F925F926F927F9237
:10B9F0008F929F92AF92BF92CF92DF92EF92FF927F
:10BA00000F931F93CF93DF9300D01F921F92CDB758
:10BA1000DEB71092500C80913D0C10923D0C8823A3
:10BA2000F9F020E040E070E060E089EE9DEB0E94DC
:10BA3000C9430F900F900F900F900F90DF91CF910F
:10BA40001F910F91FF90EF90DF90CF90BF90AF903C
:10BA50009F908F907F906F905F904F900C945A5171
:10BA600020918102309182024091400C5091410C12
:10BA7000CA01820F931F2436310509F066C447308E
:10BA8000510544F006978A3091050CF06DC48AE0A8
:10BA900090E074C406964A3F5F4FACF380911E0954
:10BAA000882309F4DAC181E04091FB195091FC1917
:10BAB0002091F9193091FA19241735070CF080E01C
:10BAC00040919D0C50919E0C20919B0C30919C0CB0
:10BAD000241735070CF482608093A90820917B0D10
:10BAE00030917C0D40917D0D50917E0D6091870DC0
:10BAF0007091880D8091890D90918A0D0F94DFC40B
:10BB00004B015C0120917F0D3091800D4091810DA2
:10BB10005091820D60918B0D70918C0D80918D0DE7
:10BB200090918E0D0F94DFC469837A838B839C83FD
:10BB30002091830D3091840D4091850D5091860D9B
:10BB400060918F0D7091900D8091910D9091920D5B
:10BB50000F94DFC42B013C0120E030E040E251E4CF
:10BB60000F9453BE20E030E048EC52E40F9453BEF3
:10BB70006B017C0120E030E0A901C301B2010F9408
:10BB8000EDBD20E030E040EA50EC87FD04C020E04D
:10BB900030E040EA50E4C701B6010F94DFC420E072
:10BBA00030E040E251E40F94D9C50F944BC62B010D
:10BBB0003C0180E277FE09C07094609450944094F8
:10BBC000411C511C611C711C8DE28093510C60E280
:10BBD000F0E14F16F7E25F06610471048CF0C301D7
:10BBE000B20120E137E240E050E00F9453C4CA01B3
:10BBF000B9012AE030E040E050E00F9453C4605DAA
:10BC00006093520C60E248EE441643E0540661042F
:10BC100071048CF0C301B20128EE33E040E050E043
:10BC20000F9453C4CA01B9012AE030E040E050E06B
:10BC30000F9453C4605D6093530CC301B20124E6BA
:10BC400030E040E050E00F9453C46AE0C62ED12C9F
:10BC5000E12CF12CCA01B901A70196010F9453C43C
:10BC6000605D6093540CC301B201A70196010F946B
:10BC700053C46D83CA01B901A70196010F9453C43F
:10BC80009D81992309F48AC38EE28093550C605DEF
:10BC90006093560C905D9093570C61E57CE081EACF
:10BCA00098E00F948BC920E030E0A901C501B401F0
:10BCB0000F94EDBD20E030E040E05FEB87FD04C075
:10BCC00020E030E040E05FE3C501B4010F94DFC441
:10BCD0000F944BC6CB010F942D25BC018CE998E045
:10BCE0000F948BC920E030E0A90169817A818B81B2
:10BCF0009C810F94EDBD20E030E040E05FEB87FDDC
:10BD000004C020E030E040E05FE369817A818B810C
:10BD10009C810F94DFC40F944BC6CB010F942D254B
:10BD2000BC0187E998E00F948BC9E0910309EF7794
:10BD3000E983E11127C00F94B24C882319F1809157
:10BD4000131B9091141BA091151BB091161B00970B
:10BD5000A105B105B9F0BC01CD016D597F4F8F4FE1
:10BD60009F4F24E630E040E050E00F9431C46091F2
:10BD7000171B7091181B8091191B90911A1B0F941F
:10BD800031C429830F947C22162FA72EB82E092F99
:10BD9000F62E80911A02F9818F17C9F0F0931A02DA
:10BDA00048E4F49FB001112490E080E00F94F2BDCC
:10BDB0002AE037ED43E25CE30F9453BE0F9452C682
:10BDC0006093960869816111FBC21092910880917D
:10BDD0001902F81609F441C010931902612F7A2D47
:10BDE0008B2D902F20E13EE040E050E00F9431C4D5
:10BDF00069012CE3422E512C612C712C612F7A2D7C
:10BE00008B2D902FA30192010F9431C4CA01B90167
:10BE1000A30192010F9431C4E4E6CE16D10408F0D8
:10BE2000F7C27F936F93DF92CF9286EB96E19F9359
:10BE30008F9381E898E09F938F930F9484BD0FB602
:10BE4000F894DEBF0FBECDBF85E0982F990F990FF4
:10BE5000891B880F8058809380080E94224889831C
:10BE600081E00E9418518091091B863180F48091F5
:10BE70000B1B833060F095E9E92E97E1F92E03E181
:10BE800023E043E068E085ED9AE10F94C2AB809136
:10BE9000A908982F927042E102E081FF02C048E0B9
:10BEA0000CE08091091B843180F480910B1B841776
:10BEB00060F0992309F4C1C281E797E17C0123E096
:10BEC00068E485ED9AE10F94C2AB8091091B84313F
:10BED000C0F480910B1B8230A0F0F981FF2309F49C
:10BEE000AFC28091C40D882309F4AAC285E397E10B
:10BEF0007C0102E123E042E068E685ED9AE10F94DF
:10BF0000C2AB8091091B8C3108F00CC1C090F919AB
:10BF1000D090FA19A090FB19B090FC19843198F4D4
:10BF200080910B1B883078F08091A90880FF8BC22C
:10BF300087EE96E17C010CE022E048E068E285EDC6
:10BF40009AE10F94C2AB8091091B883048F5498172
:10BF5000411104C08091E409811122C0C5010F94F0
:10BF6000D725FC01808193E0803229F4818192E021
:10BF7000803209F491E043E050E0491B51094E0F33
:10BF80005F1F892F880F880F981B892F67E0815DBD
:10BF90000E94ED5C69E070E080E090E00E94D0518A
:10BFA0008091091B8C3130F580910B1B843110F18D
:10BFB000C6010F94D725FC01808193E0803229F4DB
:10BFC000818192E0803209F491E043E050E0491B26
:10BFD00051094E0F5F1F892F880F880F981B892FDB
:10BFE0006CE1815D0E94ED5C69E070E080E090E0D2
:10BFF0000E94D05100919B0C10919C0C8091091BC8
:10C00000883060F56981611104C08091E90981116E
:10C0100025C080919D0C90919E0C0F94D725FC011A
:10C02000808193E0803229F4818192E0803209F4AA
:10C0300091E043E050E0491B51094E0F5F1F892FEB
:10C04000880F880F981B892F67E08E5A0E94ED5C3D
:10C0500069E070E080E090E00E94D0518091091B7F
:10C060008C3130F580910B1B843110F1C8010F9495
:10C07000D725FC01808193E0803229F4818192E010
:10C08000803209F491E043E050E0491B51094E0F22
:10C090005F1F892F880F880F981B892F6CE18E5A9C
:10C0A0000E94ED5C69E070E080E090E00E94D05179
:10C0B0008091091B8C31B0F580910B1B843190F17C
:10C0C0009091C40D292F30E02115310559F1898156
:10C0D0008111BCC18091640287FDB8C1989F900115
:10C0E0001124220F232F221F330B31951AE244E62D
:10C0F000429FC001439F900D112481589F4F6FEFC5
:10C1000070E00F94C2C4CB010F94D725AC016CE151
:10C1100087E60E94ED5C612F110F770B880B990B5E
:10C120000E94D0510F94B24C882369F18091091B71
:10C13000843348F580910B1B8A3228F107E028E010
:10C140004AE26AE285ED9AE10F94D0A905E022E087
:10C150004CE262E385ED9AE10F94D0A96AE08AE2AD
:10C160000F9489A96091D71A7091D81A82E38093AD
:10C17000F11A8BE28093F21A21EF3AE142E385ED66
:10C180009AE10F9493A88091091B853340F4809124
:10C190000B1B813320F06AE486E30F9489A9809118
:10C1A000091B843368F480910B1B823348F002E052
:10C1B0002091960842E367E385ED9AE10F94D0A9B8
:10C1C0008091091B8033D8F480910B1B8832B8F022
:10C1D00080919108882361F041E958E060E387E3AA
:10C1E0000E94ED5C65E270E080E090E00E94D0513A
:10C1F00041E858E060E3809180080E94ED5C809106
:10C20000091B873208F050C080910B1B8F3108F456
:10C210004BC083E080930C1B16E210930D1B68E566
:10C2200070E080E090E00E94D0518BE080930C1B86
:10C2300010930D1B9981992309F40AC18CE998E0A8
:10C240000E94665888E280930C1B16E210930D1B27
:10C2500069E570E080E090E00E94D05180E3809337
:10C260000C1B10930D1BF981FF2309F412C187E900
:10C2700098E00E9466588DE480930C1B16E21093A0
:10C280000D1B6AE570E080E090E00E94D05185E5EA
:10C2900080930C1B10930D1BF981FF2309F41CC123
:10C2A00081EA98E00E9466588091091B833338F533
:10C2B00080910B1B8B3218F183E00E94185183E0B0
:10C2C00080930C1B83E380930D1B66E070E080E09D
:10C2D00090E00E94D05181E00E941851809181022B
:10C2E000909182020F94D725AC0163E38CE00E9409
:10C2F000ED5C65E270E080E090E00E94D0518091BA
:10C30000091B813408F084C180910B1B863308F42B
:10C310007FC110920C1B8EE380930D1B8AE897E17E
:10C320000E94754F182F863108F0FBC08AE897E10C
:10C330000E946658153109F46BC160E270E080E03C
:10C3400090E00E94D0511F5FF5CF243631054CF4A8
:10C350008536910504F58A30910534F48AE090E041
:10C3600009C084369105BCF0883EE3E09E0714F0D6
:10C3700087EE93E02817390709F490CB9093820257
:10C38000809381021092400C1092410C1092420C4A
:10C390001092430C83CB84E690E0F0CF662351F0FB
:10C3A0008EE28093550C605D6093560C80E2809322
:10C3B000570C73CC80E28093560C8093550CF6CFCB
:10C3C0008981843608F164E60F9494C4805D80937B
:10C3D000550C99819A30D0F02AE0892F622F0F9462
:10C3E00094C40F9494C4905D9093560C89816AE034
:10C3F0000F9494C4905D9093570C65E57CE081E9BF
:10C4000098E00F948BC9E3CC80E2E1CF90E2ECCFCF
:10C410007F936F93DF92CF928CEA96E19F938F93F5
:10C4200081E898E09F938F930F9484BD0FB6F894A2
:10C43000DEBF0FBECDBF86E008CD8BE697E13ECDD7
:10C440008FEF96E155CD8FEC96E174CD15E24FCE8E
:10C4500087E00F94E60A80FF13C00CE918E0F801AA
:10C4600061918F01662309F4EDCE6F320CF06FE31A
:10C47000062E000C770B880B990B0E94D051EFCF42
:10C480008091E40B80FDDACE8AEC96E10E94A05404
:10C49000D9CE87E00F94E60A869580FF13C007E99E
:10C4A00018E0F80161918F01662309F4E4CE6F3240
:10C4B0000CF06FE3062E000C770B880B990B0E9493
:10C4C000D051EFCF8091E40B869580FDD0CE8AECE1
:10C4D00096E10E94A054CFCE87E00F94E60A86959D
:10C4E000869580FF13C001EA18E0F80161918F0181
:10C4F000662309F4D9CE6F320CF06FE3062E000CE0
:10C50000770B880B990B0E94D051EFCF8091E40BF1
:10C510008695869580FDC4CE82EC96E10E94A0545B
:10C52000C3CE80917F08F981F817B1F01091891777
:10C53000F0937F088AE897E10E94754F181708F07A
:10C5400064C01F5FE12FF0E0E657F84E8081807CE9
:10C550008038B9F3109389170091891710E00657B6
:10C56000184EC8010E94754F898360E870E0C801C9
:10C570000E9481574981453108F04AC060E270E06D
:10C5800080E090E00E94D0516981643109F440C09C
:10C5900060E270E080E090E00E94D05189818331B8
:10C5A000B9F160E270E080E090E00E94D0519981A2
:10C5B000923171F1292F30E02E5F3F4F4AEF420355
:10C5C000B001439F700D112460587F4F8AE897E1B6
:10C5D0000E94815760E270E080E090E00F900F9041
:10C5E0000F900F900F90DF91CF911F910F91FF90BF
:10C5F000EF90DF90CF90BF90AF909F908F907F9003
:10C600006F905F904F900C94D05110928917A4CFE7
:10C610000F900F900F900F900F90DF91CF911F917F
:10C620000F91FF90EF90DF90CF90BF90AF909F90D1
:10C630008F907F906F905F904F9008952F923F92D0
:10C640004F925F926F927F928F929F92AF92BF9222
:10C65000CF92DF92EF92FF920F931F93CF93DF93CE
:10C66000D62FC72FFC0180809180A280B380C501A6
:10C67000B40120E831E541E050E00F9431C4C90134
:10C680006DE671E00F94AEC46B017C01C501B4018D
:10C6900020E13EE040E050E00F9431C4CA01B9010E
:10C6A00028E130E040E050E00F9431C4362E272ED0
:10C6B000062F172F8CE3482E512C612C712CC501AD
:10C6C000B401A30192010F9431C4B62EA72ECA0162
:10C6D000B901A30192010F9431C4CB01C114D1045B
:10C6E00079F1AF92BF927F936F932F923F92FF9217
:10C6F000EF92DF92CF928BEA93E19F938F93CF9348
:10C70000DF930F9484BD8DB79EB70E960FB6F89445
:10C710009EBF0FBE8DBF8D2F9C2FDF91CF911F919C
:10C720000F91FF90EF90DF90CF90BF90AF909F90D0
:10C730008F907F906F905F904F903F902F900895D3
:10C74000E114F104C9F0AF92BF927F936F932F92DF
:10C750003F92FF92EF928BE993E19F938F93CF9358
:10C76000DF930F9484BDEDB7FEB73C960FB6F894F7
:10C77000FEBF0FBEEDBFCFCF012BB9F0AF92BF927E
:10C780007F936F932F923F928FE893E19F938F93C4
:10C79000CF93DF930F9484BD8DB79EB70A960FB6E3
:10C7A000F8949EBF0FBE8DBFB6CF892BA9F0AF9274
:10C7B000BF927F936F9387E893E19F938F93CF937B
:10C7C000DF930F9484BDEDB7FEB738960FB6F8949B
:10C7D000FEBF0FBEEDBF9FCFAF92BF9283E893E144
:10C7E0009F938F93CF93DF930F9484BD0F900F90FF
:10C7F0000F900F900F900F908ECFAB01BC01409324
:10C80000171B5093181B6093191B70931A1B80E819
:10C810009CE10C94C3E6CF93DF93DB01F9019C917B
:10C820009130C1F0943080F094509C938830D1F4D2
:10C8300080819181009771F0019791838083480FE7
:10C84000591FEA01188206C08C3539F49C5F9C930D
:10C85000943041F4DF91CF9108958B3339F781E023
:10C860008C93F8CF20813181B9016F5F7F4F718345
:10C870006083420F531FEA018883808191818F3545
:10C8800091056CF7E7CF0F931F9381E00091171B81
:10C890001091181B2091191B30911A1B4091131BEA
:10C8A0005091141B6091151B7091161B04171507EE
:10C8B0002607370708F480E01F910F9108954F92E3
:10C8C0005F926F927F928F929F92AF92BF92CF9220
:10C8D000DF92EF92FF920F931F93CF931092710804
:10C8E000109270082FE320936F0810926E08109238
:10C8F0006D0810926C081092580710925907109208
:10C900005A0710925B079C01F90190812F5F3F4FFE
:10C910009032D1F39E34C9F4818190ED980F9A3012
:10C9200020F08D3211F08B3281F432969F012F5F0F
:10C930003F4F808180538A3008F47EC09F012F5F73
:10C940003F4F8081803209F479C0F093880CE093E6
:10C95000870C8F010F5F1F4FC0816AE270E0C80132
:10C960000F9480C9009731F0FC01319780818032AB
:10C97000E1F31182CD3429F0C43519F0C73409F040
:10C980004BC0F80180810F5F1F4F8032D1F380537D
:10C990008A3008F041C0C0936F0890E080E04AE020
:10C9A000DF011196489F9001499F300D1124C90164
:10C9B000C0972081820F911D27FD9A95218130ED2E
:10C9C000320F3A30E8F190936E0880936D082E3262
:10C9D00061F4329630E04AE0DF0131962C9150ED5F
:10C9E000520F5A3078F130936C089D01D9012F5FB6
:10C9F0003F4F4C914032D1F3CD34A1F58E319105AA
:10CA000039F030F58731910519F08C31910551F5E8
:10CA1000B0937108A0937008CF911F910F91FF9070
:10CA2000EF90DF90CF90BF90AF909F908F907F90CE
:10CA30006F905F904F900895F90178CFF9017ECF04
:10CA4000FD01AECF349F200D112430ED320FC4CF45
:10CA50008537910538F087379105D0F2803A23E089
:10CA60009207B1F25091870C70E060E0C12CD12C9C
:10CA70007601C394FD0131964C91442309F492C090
:10CA80004132A1F4CD3491F48032910579F4F093E0
:10CA90007108E093700863E270E0CF010F9480C9E1
:10CAA000009709F4B9CFFC011082B6CF41544A3146
:10CAB00008F073C0DF012D91203209F459C030ED28
:10CAC000320F3A3008F465C02E3209F053C021818C
:10CAD00020532A3008F45DC030E020E06115710574
:10CAE00019F4BF0161507109A42FB0E0260137018C
:10CAF00004C0440C551C661C771C4A95D2F78090E4
:10CB0000580790905907A0905A07B0905B07842867
:10CB10009528A628B7288092580790925907A09286
:10CB20005A07B0925B0721153105A9F1251BA25CBC
:10CB3000B84F2C9320812154DF012A3108F49ACF79
:10CB4000DF012191222309F495CF30ED320F3A30E5
:10CB5000B8F333ED320F323098F32B3289F39D0165
:10CB60002F5F3F4F4C91403209F084CFD901F7CF6E
:10CB7000FD01A0CF2D3219F02B3209F0ADCF21816C
:10CB800030ED320F3A3028F02E3209F0A5CF228155
:10CB90009FCF9F01A9CF20E0CACF6115710551F643
:10CBA000BD01C8CF709371086093700835CFCF93E3
:10CBB000DF93EC018991882319F00F94304FFACF5D
:10CBC0008DE00F94304F8AE0DF91CF910D94304F7C
:10CBD000FC01659175918591949108952F923F92F2
:10CBE0004F925F926F927F928F929F92AF92BF927D
:10CBF000CF92DF92EF92FF920F931F93CF93DF9329
:10CC0000CDB7DEB7C654D1090FB6F894DEBF0FBE5C
:10CC1000CDBF70E060E085E40F94EE42182F8F3FA7
:10CC200009F484C08823E9F089E295E1CA5BDF4F0B
:10CC30000FB6F894DEBF0FBECDBFDF91CF911F912D
:10CC40000F91FF90EF90DF90CF90BF90AF909F90AB
:10CC50008F907F906F905F904F903F902F900D94AA
:10CC6000BB4F24EB30E03A83298383E50F94B54230
:10CC7000882321F00F9433429A83898365E070E022
:10CC800083E40F94EE428AA760E085E50F94D942D1
:10CC900025968FAF259760E08CE195E10E9476465E
:10CCA000A981BA81BD01BB0F880B990B0F94F4BD0C
:10CCB0006D837E838F8327969FAF27970F94AFA2B4
:10CCC000688B798B8A8B9B8B1F3F09F046C420E0D1
:10CCD00030E04CE053E46D817E818F8127969FADDB
:10CCE00027970F943FC718160CF0ABC181EF94E162
:10CCF0000F94BB4F80E0CA5BDF4F0FB6F894DEBFE6
:10CD00000FBECDBFDF91CF911F910F91FF90EF909C
:10CD1000DF90CF90BF90AF909F908F907F906F905B
:10CD20005F904F903F902F900C94124746E450E054
:10CD30005A8349839ACF1FAEAFC12496EEADFFADA3
:10CD40002497808383C2FBEE4F2E512C612C712CD3
:10CD500004C384E190E0A0E0B0E08C8B9D8BAE8BAF
:10CD6000BF8BE4E14E2E512C612C712C04C34C8AF4
:10CD70005D8A6E8A7F8AFFC22496EEADFFAD24974E
:10CD80008083D4C389819A81AB81BC8129A93AA9C6
:10CD90004BA95CA9821B930BA40BB50BB7FD59C023
:10CDA0008FAD0F94C72E8AE00F94304F89819A81FE
:10CDB000AB81BC818053984FAF4FBF4F89AB9AABCB
:10CDC000ABABBCAB9DA9911177C02EA93FA948ADD3
:10CDD00059ADB101802F26969FAD26970F943FC77E
:10CDE00018160CF053C020E030E040E050E4B101F0
:10CDF000802F26969FAD26970F94DFC46EAB7FAB36
:10CE000088AF99AF2CA53DA54EA55FA589819A81D4
:10CE1000AB81BC81280F391F4A1F5B1F2AAF3BAF74
:10CE20004CAF5DAF20E030E040EC50E46D817E819E
:10CE30008F8127969FAD27970F94DEC49101402FD5
:10CE400026965FAD26970F94EDBD881F8827881F13
:10CE50008DAB88899989AA89BB89C816D906EA0643
:10CE6000FB0610F4D701C60129813A814B815C8110
:10CE7000281B390B4A0B5B0BDA01C90181389F442F
:10CE8000A241B105A8F18DE394E10EC289819A8196
:10CE9000AB81BC812AAD3BAD4CAD5DAD821B930B2C
:10CEA000A40BB50B4DE25CE36CE37CE3B7FDD1CFA3
:10CEB000812F0E94E8EFCDCF20E030E040EF51E439
:10CEC0006D817E818F8127969FAD27970F94DEC459
:10CED0009B01AC01B101802F26969FAD26970F9440
:10CEE000EDBD87FFB6CF49ED5CE369EE7CE3E0CFB3
:10CEF0004AA55BA5888D998D481759070CF09EC0EF
:10CF000003970CF49BC080EE93E10F94BB4F1F3F3F
:10CF100009F076C0A0EDB3E1BA83A9838FEB93E16A
:10CF20000F94BB4F89819A810F94BB4F48855985D7
:10CF30006A857B858CED93E10F9478528AE00F949B
:10CF4000304F8FEB93E10F94BB4F89819A810F94FF
:10CF5000BB4F49A15AA16BA17CA188ED93E10F942D
:10CF600078528AE00F94304F8FEB93E10F94BB4FD0
:10CF700089819A810F94BB4FB501A40184ED93E19F
:10CF80000F9478528AE00F94304F2596FFAD259785
:10CF9000FF2391F12CEA35EC47E25EE369A17AA127
:10CFA0008BA19CA10F9453BE6B017C012CEA35EC44
:10CFB00047E25EE3C501B4010F94D9C528853985E0
:10CFC0004A855B851F3F09F52093A00C3093A10C87
:10CFD0004093A20C5093A30CC092A40CD092A50C29
:10CFE000E092A60CF092A70C6093A80C7093A90C89
:10CFF0008093AA0C9093AB0C81E0809366027ACE6A
:10D00000EAE5FCE6FA83E98389CF2093FE193093A1
:10D01000FF194093001A5093011AC092021AD0923D
:10D02000031AE092041AF092051A6093061A70939C
:10D03000071A8093081A9093091ADECF0E94D654DB
:10D0400080C08DED94E10F94BB4F0E94DBEE8FE723
:10D0500080939F0C24EB30E0A8EEB3E00F9485C4DE
:10D060006CA77DA78EA79FA7288939894A895B89E4
:10D07000260F371F481F591F2AAF3BAF4CAF5DAF7C
:10D080001092660281E080937E0232E0310F3EAF63
:10D09000323008F450CE1FAFC888D988EA88FB88A0
:10D0A000C9AADAAAEBAAFCAA812C912C540189A264
:10D0B0009AA2ABA2BCA288869986AA86BB868FE775
:10D0C00090E0A0E0B0E08C8B9D8BAE8BBF8B1C867C
:10D0D00090E49A8FACE1AB8FB6E4BC8F1D8E1E8EB0
:10D0E0001F8E18A23FE7432E512C612C712C1DAAD4
:10D0F0008EAA9FAAA8AEB9AE1EA21FA218A619A6F4
:10D10000E1E0EDA3198E188E212C312C00E026963B
:10D110001FAE2697F5E11F02C00111249C012B5080
:10D12000364E22963FAF2EAF2297285F3F4F249670
:10D130003FAF2EAF24974AA5042E000C550B5BA7DA
:10D140004AA780917E02882309F4B0C00F94AFA251
:10D1500069837A838B839C835091EA0958AB55236A
:10D1600009F48BC00E948EEF60919B0C70919C0C17
:10D170001F3F39F02296AEADBFAD229714966D9148
:10D180007C91072E000C880B990B0F94F4BD1B01AA
:10D19000082F26969FAF26972D8D3E8D4F8D58A137
:10D1A00026969FAD26970F943FC718163CF42D8EF8
:10D1B0003E8E0F8F2696BFAD2697B8A32C853A8D4D
:10D1C0004B8D5C8DB101802F26969FAD26970F94D5
:10D1D000EDBD87FF07C02C863A8E0B8F2696EFADEC
:10D1E0002697EC8FFDA19101402F26965FAD2697E3
:10D1F0006D817E818F8127969FAD2797FF2309F44C
:10D200005AC00F94EDBD87FF38C049815A816B81A8
:10D210007C814C195D096E097F09DB01CA018858C0
:10D220009341A109B109B7FD28C08C899D89AE89B8
:10D23000BF8984199509A609B709B595A79597954A
:10D2400087951F3F09F079CD80939F0C4EA35FA374
:10D2500068A779A7FD81FD8F2E812E8F3F813F8F9B
:10D2600027964FAD279748A389819A81AB81BC81CE
:10D27000888B998BAA8BBB8B1DA220E030E040EFFE
:10D2800051E46D817E818F8127969FAD27970F9402
:10D29000DFC49101402F26965FAD26970F94EDBD18
:10D2A00087FF70CD8BE594E10F94BB4F10927E0207
:10D2B0000E94DBEEA1CE0F943FC71816F4F68981C9
:10D2C0009A81AB81BC81288939894A895B89821B13
:10D2D000930BA40BB50BAC01BD0148585341610938
:10D2E000710977FDCACF488D598D452B09F40DC1C1
:10D2F000CEA0DFA0E8A4F9A4C80ED91EEA1EFB1E2A
:10D300002EA13FA148A559A5281B390B4A0B5B0B41
:10D31000C301B2010F9421C4A70196010F9453C415
:10D320004C885D886E887F88420E531E641E751E71
:10D3300054E145165104610471040CF40ACD8CEEDD
:10D3400048165104610471040CF0FDCC90E84916B4
:10D350005104610471040CF40ACD4C8A5D8A6E8A12
:10D360007F8A2EEF30E040E050E02419350946096D
:10D37000570929013A014C895D896E897F8985EDBC
:10D3800094E10F948852B301A20180ED94E10F94CF
:10D3900088524C855A8D6B8D7C8D89EC94E10F946D
:10D3A00078524D8D5E8D6F8D78A182EC94E10F9453
:10D3B0007852A88DB98D13970CF4A7C0C301B201A0
:10D3C0000F94F4BD20E030E040E850E40F9453BEE9
:10D3D0004B015C012C853A8D4B8D5C8D6D8D7E8D66
:10D3E0008F8D98A10F94DEC42BED3FE049E450E40B
:10D3F0000F9453BE20E030E040E05FE30F9453BE53
:10D400009B01AC01C501B4010F94D9C56C877D8720
:10D410008E879F87C701B6010F94F4BD2FE632E1D6
:10D4200043E85AE30F9453BE6B017C011E3F59F051
:10D430002AE939E949E15FE3812C912CA12C6EE3C3
:10D44000B62E1F3F59F42DEC3CEC4CE45EE37BEA36
:10D45000872E7AEA972EA92C7EE3B72E6C857D85E0
:10D460008E859F850F9453BE688779878A879B87AF
:10D470009B01AC010F94DFC4A70196010F94D9C59D
:10D4800069A37AA38BA39CA3288539854A855B85EC
:10D49000C701B6010F9453BEA50194010F9453BE6A
:10D4A0004B015C014C855D856E857F858CEB94E13D
:10D4B0000F947852B701A60186EB94E10F9478524D
:10D4C0008AE00F94304FBEAD87EA94E1B23010F09D
:10D4D00088E994E10F94BB4F488559856A857B851F
:10D4E00082E994E10F94785249A15AA16BA17CA1E1
:10D4F0008CE894E10F947852B501A40186E894E198
:10D500000F9478528AE00F94304F8C899D89AE89B0
:10D51000BF89840D951DA61DB71DB595A795979537
:10D5200087951F3F09F028CC80939F0C288D398D5B
:10D530002F5F3F4F398F288F3D813C874E814A8F27
:10D540005F815B8F27968FAD27978C8FC980DA809C
:10D55000EB80FC8098A99DA390CEE12E012E000CBB
:10D56000FF08F70183E0EE0FFF1F8A95E1F7EA5805
:10D57000FD4F668177816F507109072E000C880B73
:10D58000990B0F94F4BD9B01AC016D817E818F815D
:10D5900027969FAD27970F943FC718160CF4A6CB7C
:10D5A0008DED94E10F94BB4F0E94DBEE85E18E9DE3
:10D5B000F0018F9DF00D1124EB50F64E8FE7808720
:10D5C00022E330E049CD3F924F925F926F927F927B
:10D5D0008F929F92AF92BF92CF92DF92EF92FF9283
:10D5E0000F931F93CF93DF9380915A0787FD38C025
:10D5F00080915B078370A1F5C091941AD091951A20
:10D60000488159816A817B8180E693E10F94785249
:10D610004C815D816E817F8183E89DE60F94785215
:10D620004091901A5091911A6091921A7091931AA8
:10D6300080E89DE60F9478528AE0DF91CF911F91A8
:10D640000F91FF90EF90DF90CF90BF90AF909F90A1
:10D650008F907F906F905F904F903F900D94304FE0
:10D660006090881A7090891A80908A1A90908B1A0C
:10D67000A0908C1AB0908D1A00918E1A10918F1A6A
:10D68000C090901AD090911AE090921AF090931A4C
:10D6900088E50F94B542C82F882309F49AC00F94E7
:10D6A0003742362E472E582ED92F20E030E046E65E
:10D6B00053EC0F943FC787FD0DC020E030E046E6F5
:10D6C00053E4632D742D852D9D2F0F94EDBD1816F9
:10D6D0000CF081C066EE70E08DE493E10F949952F6
:10D6E00066EE70E088E493E10F94995285E493E14B
:10D6F0000F94BB4FC0E089E50F94B542882361F1D8
:10D700000F943742362E472E582ED92F20E030E086
:10D7100046E653EC0F943FC787FD0DC020E030E094
:10D7200046E653E4632D742D852D9D2F0F94EDBD9A
:10D7300018160CF055C066EE70E082E393E10F948A
:10D74000995266EE70E08DE293E10F9499528AE26D
:10D7500093E10F94BB4FC0E08AE50F94B542882354
:10D7600009F443C00F9437426B017C0120E030E0A4
:10D7700040E151EC0F943FC787FD0AC020E030E044
:10D7800040E151E4C701B6010F94EDBD18166CF5E8
:10D7900067EF7FEF88E193E10F94995269E070E0C1
:10D7A00083E193E10F94995280E193E1DF91CF916E
:10D7B0001F910F91FF90EF90DF90CF90BF90AF90AF
:10D7C0009F908F907F906F905F904F903F900D94BF
:10D7D000BB4FC1E090CF632C742C852C9D2E8BCF3A
:10D7E000A32CB42C052D1D2FB7CFCC23E1F0C30102
:10D7F000D4018093881A9093891AA0938A1AB093BF
:10D800008B1AC501D80180938C1A90938D1AA0931E
:10D810008E1AB0938F1AC092901AD092911AE092F9
:10D82000921AF092931ADF91CF911F910F91FF906E
:10D83000EF90DF90CF90BF90AF909F908F907F90B0
:10D840006F905F904F903F900895CF92DF92EF924C
:10D85000FF928AE50F94B542882309F45AC00F94C9
:10D86000374220E030E040E050EC0F94EDBDC12C99
:10D87000D12CE12C90ECF92E87FD0FC00F9437428C
:10D8800020E030E040E050E40F943FC718160CF45D
:10D8900062C00F9437426B017C012091A514309136
:10D8A000A6144091A7145091A814C701B6010F9473
:10D8B00053BE0F944BC6CB010F94E8A280E50F94A2
:10D8C000674281114EC0A70196016091901A709134
:10D8D000911A8091921A9091931A0F94DFC46093D9
:10D8E000901A7093911A8093921A9093931A0F94AE
:10D8F000DC5B4091901A5091911A6091921A70914C
:10D90000931A81E093E10F9478528AE00F94304F9C
:10D9100005C083E50F94B5428111A1CF80915A07CC
:10D9200087FD24C080915B07837001F50F94DC5B59
:10D930004091901A5091911A6091921A7091931A95
:10D9400082EF92E10F9478528AE0FF90EF90DF909F
:10D95000CF900D94304FC12CD12CE12C80E4F82EC7
:10D960009CCF0F9423428111AECFD8CF82E50F9484
:10D9700067428111DBCFFF90EF90DF90CF90089549
:10D980004F925F926F927F928F929F92AF92BF92CF
:10D99000CF92DF92EF92FF92CF93DF93CDB7DEB7B6
:10D9A0002C970FB6F894DEBF0FBECDBF40907B0D15
:10D9B00050907C0D60907D0D70907E0D20913D0209
:10D9C00030913E0240913F0250914002C301B201AA
:10D9D0000F94DFC469837A838B839C8380907F0D4F
:10D9E0009090800DA090810DB090820D2091410209
:10D9F000309142024091430250914402C501B4016A
:10DA00000F94DFC46D837E838F839887C090830DCE
:10DA1000D090840DE090850DF090860D2091450208
:10DA2000309146024091470250914802C701B60129
:10DA30000F94DFC469877A878B879C87209149027E
:10DA400030914A0240914B0250914C02C301B20105
:10DA50000F94DFC42B013C0120914D0230914E0206
:10DA600040914F0250915002C501B4010F94DFC4A0
:10DA70004B015C01209151023091520240915302BE
:10DA800050915402C701B6010F94DFC46B017C01B1
:10DA90000F94DC5B87E69CE00F94BB4F83E50F940B
:10DAA0006742882321F00F94234280933B028091A8
:10DAB0003B02811151C082E390E10F94BB4F8FE58F
:10DAC0009CE00F94BB4F49815A816B817C8184EE2D
:10DAD00091E30F9478524D815E816F81788583E860
:10DAE0009DE60F94785249855A856B857C8580E840
:10DAF0009DE60F9478528DE59CE00F94BB4F85E531
:10DB00009CE00F94BB4FB301A20184EE91E30F940C
:10DB10007852B501A40183E89DE60F947852B701CD
:10DB2000A60180E89DE60F9478528AE02C960FB605
:10DB3000F894DEBF0FBECDBFDF91CF91FF90EF9085
:10DB4000DF90CF90BF90AF909F908F907F906F901D
:10DB50005F904F900D94304F86E390E1AECF2F92BF
:10DB60003F924F925F926F927F928F929F92AF926D
:10DB7000BF92CF92DF92EF92FF920F931F93CF93BA
:10DB8000DF93CDB7DEB7CB54D1090FB6F894DEBF23
:10DB90000FBECDBF2DB73EB739AF28AF87E00F948A
:10DBA000BE3981110BC061E086E50E94143B8DA354
:10DBB000853060F082EC9BE00F94BB4FA8ADB9AD0F
:10DBC0000FB6F894BEBF0FBEADBF3EC33DA1332319
:10DBD00021F082EA9BE00F94BB4F6AE080E50E944F
:10DBE000143B182F8CEF810F8F3218F08EE79BE0DB
:10DBF000E3CF60E085E40F94D942882309F448C05C
:10DC000081E08FABE090941AF090951AD7012D9196
:10DC10003D914D915C916091870D7091880D80913F
:10DC2000890D90918A0D0F94DFC4AB01BC0188E58A
:10DC30000F94C24269877A878B879C87F70124817A
:10DC400035814681578160918B0D70918C0D80914B
:10DC50008D0D90918E0D0F94DFC4AB01BC0189E551
:10DC60000F94C2426D877E878F87988BBE01635F5A
:10DC70007F4FCE0109960F942943382E81110BC096
:10DC800063E68AE69BE00E94764682E59BE094CFBD
:10DC900092E09FABB7CF8CE40F946742082F8823A4
:10DCA00009F430C10F940F428EA3803118F08BE23B
:10DCB0009BE082CFFEA1F13009F426C160E083E54C
:10DCC0000F94D9428AAF882321F0011102C037E0B6
:10DCD0003EA38DA1833020F081E19BE00F94BB4FE8
:10DCE0009091960C9DAF80E00F94D14A0F948514CB
:10DCF0001D8A1E8A1F8A188E198E1A8E1B8E1C8EE4
:10DD000083EF9FE4A3ECB7E48D8F9E8FAF8FB8A312
:10DD100083EF9FE4A3ECB7EC89A39AA3ABA3BCA3C6
:10DD2000A12FB0E0BCA7ABA7EDB7FEB724E0129FD0
:10DD3000E019F10911240FB6F894FEBF0FBEEDBF34
:10DD40008DB79EB701969CAF8BAF01E021E04DA14E
:10DD50006FA9CE0109960F94D5539B01AC010F9486
:10DD60002CC8811161C20F94AFA2611571058105A4
:10DD7000910511F00F9436B9212C1BAA1CAA1DAADB
:10DD80001EAAAEA1A150BB0B2C96BFAFAEAF2C9775
:10DD9000E22DF0E0F8A7EFA32BA53CA5E217F307CF
:10DDA0000CF073C23196FEA7EDA73F932F93FF931C
:10DDB000EF938DEF9AE09F938F9387E09BE09F9383
:10DDC0008F931F920E945B468DB79EB709960FB640
:10DDD000F8949EBF0FBE8DBF9EA1992309F458C130
:10DDE0000F94E7B82AE030E040E050E00F9453C4CD
:10DDF0000F94F4BD20E030E040EA50E40F943FC7B8
:10DE00000FEF1FEF181614F001E010E00F94E7B8C1
:10DE100028E631E040E050E00F9453C40F94F4BD85
:10DE20002B013C010F94E7B827E130E040E050E0DF
:10DE30000F9453C46B5F7F4F8F4F9F4F0F94F4BD70
:10DE40004B015C01ADA1A430D1F4BC01A4018FEE63
:10DE50009AE00F947852B301A20187EE9AE00F94F2
:10DE6000785281EE9AE00F94BB4F0130110519F4FE
:10DE700083E40F94304F8DED9AE00F94BB4F312C1B
:10DE8000C801110FAA0BBB0B2A968CAF9DAFAEAF8A
:10DE9000BFAF2A972C96AEADBFAD2C973A161B0696
:10DEA0000CF0F6C02A966CAD7DAD8EAD9FAD2A9775
:10DEB0000F94F4BD6B017C01BAADBB2341F1AC0101
:10DEC0009B010F94DFC420E030E040E952E40F945E
:10DED00053BE9B01AC01C301B2010F94DFC42B01FF
:10DEE0003C0120E030E044EB53E40F943FC71816A8
:10DEF000FCF420E030E044EB53E4C301B2010F94A2
:10DF0000DEC4EDCF1EA2DACE22E02EA3D7CE0F9430
:10DF1000E7B824E130E040E050E00F9453C4675E7E
:10DF20007F4F8F4F9F4F0F94F4BDA7019601CFCF26
:10DF300020E030E0A901C301B2010F94EDBD87FFDD
:10DF40000BC020E030E044EB53E4C301B2010F9476
:10DF5000DFC42B013C01ECCF0091941A1091951A6B
:10DF6000F80124813581468157816D857E858F85B5
:10DF700098890F94DEC422966CAF7DAF8EAF9FAFB1
:10DF800022972BED3FE049E450E4C301B2010F9426
:10DF900053BE20E030E044E353E40F94D9C56B0155
:10DFA0007C010F94D4C56FA778AB89AB9AABD8012D
:10DFB0002D913D914D915C9169857A858B859C85EC
:10DFC0000F94DEC426966CAF7DAF8EAF9FAF2697C1
:10DFD000A50194016FA578A989A99AA90F9453BEA8
:10DFE0009B01AC0126966CAD7DAD8EAD9FAD2697A5
:10DFF0000F94DFC469837A838B839C83C701B60146
:10E000000F94CFC7A50194010F9453BE22962CAD57
:10E010003DAD4EAD5FAD22970F94DFC46D837E831F
:10E020008F83988740EF50E070E060E0CE0101966A
:10E030000E94A6EF40EF50E070E060E0CE01059650
:10E040000E94A6EFBDA1B43099F449815A816B8139
:10E050007C8181ED9AE00F9478524D815E816F81D1
:10E06000788583E89DE60F9478528AE00F94304FCC
:10E07000198A1A8A1B8A1C8AAE014F5E5F4FBE0145
:10E080006B5F7F4FCE0101960F946216339402CFDF
:10E0900001E021E040E06FA9CE0109960F94D5532D
:10E0A0006B017C01312CAC019B010F942CC88111B8
:10E0B00002C033243394A7019601C701B6010F941F
:10E0C0002CC88111E2C0EFA1F8A5EE0FFF1FEE0FE3
:10E0D000FF1F2BAD3CADE20FF31FC082D182E28265
:10E0E000F3822D8D3E8D4F8D58A1C701B6010F943F
:10E0F000EDBD87FF04C0CD8EDE8EEF8EF8A229A184
:10E100003AA14BA15CA1C701B6010F943FC71816F5
:10E1100024F4C9A2DAA2EBA2FCA2A70196016BA982
:10E120007CA98DA99EA90F94DFC46BAB7CAB8DAB92
:10E130009EABADA5BEA5BD01BB0F880B990B0F947F
:10E14000F4BD2B013C01AC019B016BA97CA98DA9FD
:10E150009EA90F94D9C56FA378A789A79AA76D8B9D
:10E160007E8B8F8B988FEBADFCADF8ABEFA710E0FB
:10E17000812C912C5401AFA5B8A96D917D918D9101
:10E180009D91B8ABAFA72FA138A549A55AA50F946B
:10E19000DEC49B01AC010F9453BE9B01AC01C501D1
:10E1A000B4010F94DFC44B015C011F5F211618F707
:10E1B000A30192010F94D9C50F94DDC7698F7A8F9F
:10E1C0008B8F9C8FBDA1B23068F18DA59EA50F9459
:10E1D00071836BA57CA58CEC9AE00F94995286EC28
:10E1E0009AE00F94BB4F43E0C701B6010F94232E72
:10E1F00080E20F94304F81E0EDA1E3300CF480E039
:10E20000E12C8E010F5D1F4F9E01235E3F4FAE013B
:10E21000475E5F4FBE016B5E7F4F0E94B7428AE050
:10E220000F94304F2394B4CD0F94FD420F946C148F
:10E230008DAD0F94D14A0F94C11B88AD99AD0FB627
:10E24000F8949EBF0FBE8DBFE8ADF9AD0FB6F89440
:10E25000FEBF0FBEEDBFC55BDF4F0FB6F894DEBF4C
:10E260000FBECDBFDF91CF911F910F91FF90EF9027
:10E27000DF90CF90BF90AF909F908F907F906F90E6
:10E280005F904F903F902F9008950F94FD42332060
:10E2900069F28BEB9AE00F94BB4F81E0FDA11F1652
:10E2A0000CF080E0EE24E3948E010F5D1F4F9E0181
:10E2B000235E3F4FAE01475E5F4FBE016B5E7F4FF7
:10E2C0000E94B742698D7A8D8B8D9C8D0052110909
:10E2D00026E042E00F947DB89F938F938AEA9AE0FC
:10E2E0009F938F9384EB9AE09F938F931F920E944A
:10E2F0005B462DB73EB7295F3F4F0FB6F8943EBF40
:10E300000FBE2DBF93CFAF92BF92CF92DF92EF920D
:10E31000FF920F931F93CF93DF93CDB7DEB7E697AE
:10E320000FB6F894DEBF0FBECDBF009170081091FC
:10E330007108F80101900020E9F731976F01C01AC8
:10E34000D10AF801CF01801B910B8C159D053CF47F
:10E3500081918F32B9F7DF0111971C92F3CF8BE1D6
:10E36000ECE3FBE1DE015C9601900D928A95E1F70A
:10E37000F12CE12CEC14FD040CF05DC0F801EE0D65
:10E38000FF1D8081811103C08FEFE81AF80A580140
:10E39000AE0CBF1CF5018081882309F44CC0FFEF4F
:10E3A000EF1AFF0AF801EE0DFF1D7F01E01AF10AD6
:10E3B00081918111FACFCE014C960E9415EB8BE131
:10E3C000FE017C96DE01119601900D928A95E1F78F
:10E3D000B501CE0101960E942FE3CE0101960F9464
:10E3E0005A408FE20F94304F8091471781113BC004
:10E3F0008DE197E00F94A42880911B1B84FF1BC024
:10E4000019821C8221E0A501BE01645E7F4FCE010E
:10E4100001960E94E8EC811129C08AE00F94304FE8
:10E420000F94DC5BB5018FE693E10F94C753CE01E7
:10E4300001960F945A408AE00F94304FCE014C96CB
:10E440000F945A40E6960FB6F894DEBF0FBECDBFCC
:10E45000DF91CF911F910F91FF90EF90DF90CF90C0
:10E46000BF90AF90089587E497E1C4CFCE014C965A
:10E470000E9484EA8BE1FE013196DE015C960190F8
:10E480000D928A95E1F7CE0101960F945A4072CF12
:10E49000BF92CF92DF92EF92FF920F931F93CF9391
:10E4A000DF9300D000D0CDB7DEB76FEF7FEF89E408
:10E4B0000F94EE42B82E6FEF7FEF8AE40F94EE4296
:10E4C000182F83E40F946742F82E8EE40F9467426E
:10E4D000C82E8AE50F946742E82ED12C811104C022
:10E4E00081E50F946742D82E012F2B2DFF2049F094
:10E4F00030E020E040E067E87DE081E00F94554A9D
:10E50000032F4F2D50E080E0B7FC05C0812F809590
:10E51000881F8827881F840F952F911D019731F43C
:10E52000E11019C0D11017C0C11015C00F94D153FC
:10E530008AE89AE026960FB6F894DEBF0FBECDBFEC
:10E54000DF91CF911F910F91FF90EF90DF90CF90CF
:10E55000BF900D94BB4F263010F4063028F00F9476
:10E56000D15381E79AE0E6CFE22E220FFF08002E7A
:10E57000000C110B60E070E080EC9FE7C1101DC043
:10E580000F9437429B01AC0160E070E0CB01DD20CD
:10E5900091F086E08E9DF0018F9DF00D1124E00F2B
:10E5A000F11FEE0FFF1FEE0FFF1FE55CF64F6081BE
:10E5B0007181828193810F94DFC426E02E9DF0014A
:10E5C0002F9DF00D1124E00FF11FEE0FFF1FEE0F36
:10E5D000FF1FE55CF64F60837183828393832696E9
:10E5E0000FB6F894DEBF0FBECDBFDF91CF911F9164
:10E5F0000F91FF90EF90DF90CF90BF9008954F92D2
:10E600005F926F927F928F929F92AF92BF92CF92C2
:10E61000DF92EF92FF92CF93DF9300D000D01F9252
:10E620001F92CDB7DEB783E50F946742F82ED090E6
:10E63000960C882319F00F942342D82E4090870D12
:10E640005090880D6090890D70908A0D80908B0D90
:10E6500090908C0DA0908D0DB0908E0D80918F0DAF
:10E660009091900DA091910DB091920D8D839E830C
:10E67000AF83B887FF2029F0D11003C080E00F944A
:10E68000D14A8CE40F946742882309F44BC080E0A0
:10E690000F94D14A80912E0790912F07C090D409F2
:10E6A000892B19F00F943342C82E0E9452F27C013C
:10E6B000892BC9F481E59AE00F94BB4F28960FB6D9
:10E6C000F894DEBF0FBECDBFDF91CF91FF90EF90EA
:10E6D000DF90CF90BF90AF909F908F907F906F9082
:10E6E0005F904F900895C7FC07C08C2D0C2C000C38
:10E6F000990B8E159F057CF089E39AE00F94BB4F30
:10E70000B701615071098EE29AE00F9499528AE044
:10E710000F94304FD3CF70E060E08C2D0E945EF2FA
:10E72000C092D4098091590783FD04C080915A0793
:10E7300085FF1FC060E084E50E94143B90E00F94C9
:10E740003F6E85E29AE00F94BB4F0F94104C8111FD
:10E7500004C082E29AE00F94BB4F6091D409062E68
:10E76000000C770B8DE09AE00F9499528AE00F9499
:10E77000304F86E50F946742F82E0F94104C882393
:10E7800041F183E40F946742882379F00F94374274
:10E7900069837A838B839C8380E00F94D14ABE0186
:10E7A0006F5F7F4F81E00F94A3528AE50F94674219
:10E7B000882359F00F94374269837A838B839C8333
:10E7C00060E0CE0101960F94304B8D2D0F94D14A0D
:10E7D0000AC0D11002C0FF2041F30F94DC5B8EEF22
:10E7E00099E00F94BB4FDD2051F08091960C811180
:10E7F00006C00F94D1538FED99E00F94BB4F0F9447
:10E80000DC5B81ED99E00F94BB4F8091960C8111F8
:10E8100059C082E390E10F94BB4F8AE00F94304FD0
:10E820000F94DC5B84EC99E00F94BB4FC090920C8A
:10E83000D090930CE090940CF090950C20E030E098
:10E84000A901C701B6010F943FC71816F4F542E0BD
:10E85000C701B6010F94232E8DE00F94304F8AE04C
:10E860000F94304FA30192016091870D7091880D34
:10E870008091890D90918A0D0F94EDBD81111FC07B
:10E88000A501940160918B0D70918C0D80918D0D7F
:10E8900090918E0D0F94EDBD811111C020918F0DBF
:10E8A0003091900D4091910D5091920D6D817E812E
:10E8B0008F8198850F94EDBD882309F4FFCE0F94C6
:10E8C000C11BFCCE86E390E1A6CF8FEB99E00F94BD
:10E8D000BB4FC8CF2F923F924F925F926F927F9221
:10E8E0008F929F92AF92BF92CF92DF92EF92FF9260
:10E8F0000F931F93CF93DF93CDB7DEB7E5970FB696
:10E90000F894DEBF0FBECDBF8DAB2091850C2CAB34
:10E9100081E08093850C80916F088D3409F482C565
:10E92000843511F40C94528A873409F091C1809196
:10E930006D0890916E088B31910509F4DCC108F0E7
:10E9400079C18430910508F030C120912A0C8230C1
:10E95000910508F48EC1213009F091C111E00297B0
:10E9600009F010E00E94933F19821A821B821C82D8
:10E970001D821E821F82188682E50F94B54288236D
:10E9800009F48FC10F9437426B017C0120E030E025
:10E99000A9010F94EDBD882309F4EAC04090870DCA
:10E9A0005090880D6090890D70908A0D80918B0D2C
:10E9B00090918C0DA0918D0DB0918E0D8CA79DA77F
:10E9C000AEA7BFA780906C0C90906D0CA0906E0CC1
:10E9D000B0906F0C8091700C9091710CA091720CA2
:10E9E000B091730C88AB99ABAAABBBABA5019401FA
:10E9F000C301B2010F94EDBD81110DC028A939A941
:10EA00004AA95BA96CA57DA58EA59FA50F94EDBD18
:10EA1000882309F4ADC0A3019201C501B4010F948C
:10EA2000DEC420E030E040E05FE30F9453BE68A70F
:10EA300079A78AA79BA72CA53DA54EA55FA568A988
:10EA400079A98AA99BA90F94DEC420E030E040E0B8
:10EA50005FE30F9453BE2B013C0120E030E0A9019D
:10EA6000C701B6010F94EDBD881F8827881F1817AE
:10EA700009F40EC180E090E0A0E8BFEB8CA79DA751
:10EA8000AEA7BFA728A539A54AA55BA5CA01B901AC
:10EA90000F9453BE4B015C01A3019201C301B2016B
:10EAA0000F9453BE9B01AC01C501B4010F94DFC4A8
:10EAB0000F94DDC74B015C01AC019B01C701B6019E
:10EAC0000F94DEC468AB79AB8AAB9BABA501940114
:10EAD000C701B6010F94DFC49B01AC0168A979A9F5
:10EAE0008AA99BA90F9453BE6B017C0120E030E002
:10EAF000A9010F943FC787FDD0C0C701B6010F948D
:10EB0000DDC76B017C01C301B2019058A5019401DE
:10EB10000F94D9C52CA53DA54EA55FA50F9453BE56
:10EB2000A70196010F9453BE28A539A54AA55BA558
:10EB30000F94DFC469837A838B839C83A50194013E
:10EB400068A579A58AA59BA50F94D9C52CA53DA537
:10EB50004EA55FA50F9453BEA70196010F9453BE17
:10EB6000A30192010F94DFC46D837E838F83988706
:10EB700020E030E0A90169817A818B819C810F942A
:10EB8000EDBD8111A2C020E030E0A9016D817E8140
:10EB90008F8198850F94EDBD811197C00F94D1534B
:10EBA00089E29DE00F94BB4F6AC08531910509F45D
:10EBB00066C08A31910509F49BC0049709F048C0EA
:10EBC00080E50F94B542C12CD12C7601882321F029
:10EBD0000E94F53B6B017C0183E50F94B5428823CD
:10EBE00061F00F94374220E030E04AE754E40F949C
:10EBF00053BE0F9452C66B017C010E9428F780918E
:10EC00008A17811105C060E08FE39DE00E9476467F
:10EC10000F94AFA2C60ED71EE81EF91E0F94AFA226
:10EC20006C197D098E099F0997FF29C080E00F9418
:10EC30000C5EF4CF8A32910509F498C260F48D31EC
:10EC4000910509F417C208F46FC04E9709F415C274
:10EC50000F94EE9814C08B35910509F43BC38C35A5
:10EC6000910509F43BC38A35910591F71092910CF7
:10EC700006C0213021F40E94933F0F94B40B3DA9AC
:10EC8000311102C00F94B7AC8CA98093850C6AC572
:10EC900080E090E0A0E8BFE3F1CEC12CD12C76015A
:10ECA00032CF89E40F94B542882331F00F94374274
:10ECB00069837A838B839C838AE40F94B54288238B
:10ECC00009F456CF0F9437424FCF412FBE016F5FEB
:10ECD0007F4F8CE69CE00F942EA30F94AFA260931D
:10ECE0007C0C70937D0C80937E0C90937F0CC7CF2F
:10ECF0000E946B48C4CF87E00F94BE398111BFCF0B
:10ED00008CE0E1EAF2E0DE01119601900D928A9525
:10ED1000E1F770E060E080E50E94203BBE016F5F9C
:10ED20007F4F0F943726ABCF87E00F94E60A81110F
:10ED300006C060E08FE40F94D9428111A0CF0E94F9
:10ED400028F710923C026091960C8CE40F94D94203
:10ED5000E82E80E00F94D14A0F94AFA260937C0C10
:10ED600070937D0C80937E0C90937F0C0F94851490
:10ED700081E08093E20B0F94E71C8AE50F946742D1
:10ED8000F82E882369F081E00F94E60A182F82E0BC
:10ED90000F94E60A11110C94B08A11E0811101C0A0
:10EDA00010E088E50F946742082F81110C94678A60
:10EDB00011110CC089E50F946742811342C1012FE4
:10EDC000F11204C001E011E0FF24F39482E50F94F6
:10EDD000B542882309F438C10F9437426CA37DA350
:10EDE0008EA39FA320E030E0A9010F94EDBD8823FE
:10EDF00081F0011105C0111103C0FF2009F410C1F9
:10EE000060E0CE0184960F9412160F94B94E0F94C1
:10EE1000684E002309F47FC0112309F479C01092D1
:10EE2000870D1092880D1092890D10928A0D109204
:10EE30008B0D10928C0D10928D0D10928E0D0F94E3
:10EE40005A1788E49DE20E94E8654B015C018CE45E
:10EE50009DE20E94E8652B013C01AC019B01C501CC
:10EE6000B4010F943FC718160CF0F3C0A50194012C
:10EE7000C301B2010F94D9C59B01AC010F9453BEDD
:10EE800020E030E040E85FE30F94DFC40F94DDC77B
:10EE900020E030E048E452E40F9453BE68A379A325
:10EEA0008AA39BA320E030E040EC5FE3C301B20102
:10EEB0000F9453BE905869837A838B839C8320E0A0
:10EEC00030E040EC5FE3C501B4010F9453BE9058AD
:10EED0006C8F7D8F8E8F9F8FAE01405E5F4FBE0126
:10EEE0006F5F7F4FCE014C960F9462160F94181FE0
:10EEF0001092870D1092880D1092890D10928A0D34
:10EF000010928B0D10928C0D10928D0D10928E0D13
:10EF100080E00F940720112319F081E00F9407205F
:10EF2000FF2009F47DC083E00F94BE39811178C0C1
:10EF30000F945A172091BD0C3091BE0C4091BF0C1C
:10EF40005091C00C60E070E086EE92E40F94DEC455
:10EF50002B013C012091C10C3091C20C4091C30C9B
:10EF60005091C40C60E070E086EE92E40F94DEC431
:10EF70004B015C0180918F0D9091900DA091910DAE
:10EF8000B091920D8093740C9093750CA093760CB5
:10EF9000B093770C0091941A1091951AD8012D9185
:10EFA0003D914D915C91C301B2010F94DEC4609319
:10EFB0006C0C70936D0C80936E0C90936F0CF80139
:10EFC0002481358146815781C501B4010F94DEC487
:10EFD0006093700C7093710C8093720C9093730C0F
:10EFE0008CE69CE00F94E8488823C1F11C8E1D8EAE
:10EFF0001E8E1F8E88E0ECE6FCE0DE01119601908B
:10F000000D928A95E1F7AE01445E5F4FBE016B5FE2
:10F010007F4FCE0101960F94621682E00F94072075
:10F020000F945A178091E10B8093E20B8E2D0F9471
:10F03000D14A0F946C1483E080937F020F94C11B1C
:10F040001ECE012F182FC2CE60E070E080E890E461
:10F05000C5CEA3019201C501B4010CCF60E08AE5E1
:10F060009DE00E9476460F94DC5B88E49DE00F945F
:10F07000BB4FD6CF0F948C7702CE0091941A10918B
:10F08000951AD8012D913D914D915C916091870D1C
:10F090007091880D8091890D90918A0D0F94DFC435
:10F0A000AB01BC0188E50F94C24269837A838B83EC
:10F0B0009C83F801248135814681578160918B0DB5
:10F0C00070918C0D80918D0D90918E0D0F94DFC4F9
:10F0D000AB01BC0189E50F94C2426D837E838F83AF
:10F0E0009887BE016B5F7F4FCE0101960F94294335
:10F0F000882309F4C4CD80E00F94D14A0F9485147D
:10F1000061E085E40F94D942182F01E021E041E04D
:10F11000682FCE0101960F94D5536B017C01AC0191
:10F120009B010F942CC8811119C049815A816B81B0
:10F130007C8185E79DE00F9478524D815E816F81DF
:10F14000788580E79DE00F947852B701A6018BE6A1
:10F150009DE00F9478528AE00F94304F0F946C1416
:10F1600011110F940F430F94C11B89CD80912A0C6C
:10F17000813009F084CD89E40F94B542182FE12C39
:10F18000882319F00F943342E82E8AE40F94B54295
:10F19000082F882379F00F943342F82E112309F4B5
:10F1A00090C0F5E0FE1508F089C08DE79DE00F9452
:10F1B000BB4F65CDF12C1111F4CF80E1E7E8FDE004
:10F1C000ACE6BCE001900D928A95E1F7112359F06D
:10F1D0008E2D0F94BC4460936C0C70936D0C8093D7
:10F1E0006E0C90936F0C002359F08F2D0F942644D2
:10F1F0006093700C7093710C8093720C9093730CED
:10F2000060E080E50F94D9428823C1F11123D1F049
:10F21000E091941AF091951A2081318142815381B5
:10F2200060916C0C70916D0C80916E0C90916F0CD4
:10F230000F94DEC460936C0C70936D0C80936E0C15
:10F2400090936F0C0023D1F0E091941AF091951AED
:10F2500024813581468157816091700C7091710CC9
:10F260008091720C9091730C0F94DEC46093700CBB
:10F270007093710C8093720C9093730C40E050E08B
:10F28000BA0186E40F94C2426B017C0120E030E0B9
:10F29000A9010F943FC71816CCF420E030E040E7F6
:10F2A00052E4C701B6010F94D9C569837A838B8371
:10F2B0009C83CE0101960F94A414E1CC002309F4A1
:10F2C0007CCF25E02F1508F078CF6FCF60E070E09D
:10F2D000CB01EBCF8FE08093910CD1CC80916C0867
:10F2E000882381F1893009F0CACC0DEBA02E02E011
:10F2F000B02E87E8C82E8DE0D82EE12C00E010E07B
:10F30000D5018D915D010F94B542F82E882361F0EF
:10F31000133011F4082FFE2C0F943742F60160834E
:10F32000718382839383EF2C1F5FF4E0CF0ED11C97
:10F33000143031F7EE2009F457C00F945A170F9488
:10F34000C11B9DCC1DEBC12E12E0D12EF12CE12C66
:10F3500000E010E0D6018D916D010F94B542382E7A
:10F360008823D9F10F9437424B015C01133059F0D7
:10F37000F701E558F24F20813181428153810F948A
:10F38000DEC44B015C01F701E957F24F2081318166
:10F3900042815381C501B4010F94DEC42B013C01AD
:10F3A0002DEB37E346E855EB0F943FC787FD0AC0C6
:10F3B0002DEB37E346E855E3C301B2010F94EDBDF1
:10F3C00018165CF41330C1F48092930D9092940D52
:10F3D000A092950DB092960D032D1F5FB4E0EB0E39
:10F3E000F11C143009F0B6CF002309F4A8CF83E94B
:10F3F0009DE00F94CE08A3CFF701EF54F34F5F01C8
:10F40000A301920160817181828193810F94DFC495
:10F41000D5016D937D938D939C931397812F0F94BA
:10F42000C60ADBCF80916D0890916E088D379105EB
:10F4300009F463C608F05FC28E34910509F402C76F
:10F4400008F022C18B31910509F45BC608F0B2C007
:10F450008531910509F4D1C508F07BC08131910552
:10F4600009F48AC508F045C0029708F0F1CB80E5A1
:10F470000F94B542C12CD12C7601882321F00E9433
:10F48000F53B6B017C0183E50F94B542882361F065
:10F490000F94374220E030E04AE754E40F9453BE23
:10F4A0000F9452C66B017C010E9428F7809170086E
:10F4B00090917108009709F459C50F949486809132
:10F4C0006D0890916E086EE97DE0892B11F466E974
:10F4D0007DE030E020E046E25DE682E00F941050EF
:10F4E00040E0C701B6010F942C7E80E00E941247D5
:10F4F000C6CB8231910511F40C947483449709F0C2
:10F50000A7CB80911B1B83FF70C581ED9DE00F94FD
:10F51000BB4F80911B1B83FF17C08CE39BE10E94B4
:10F5200015EB8BE1ECE3FBE1DE01119601900D920E
:10F530008A95E1F770E060E0CE0101960F94482CC7
:10F54000CE0101960F945A4082EC9DE00F94BB4F80
:10F5500096CB8831910509F465C5B0F486319105E3
:10F5600009F44FC5479709F073CB809170089091CB
:10F570007108FC012191222309F44DC52032D1F7F5
:10F58000DF0111971C92F6CF8931910509F4B5C5B9
:10F590004A9709F05DCB80911B1B83FF70CB83E5FD
:10F5A0000F94B542882309F46ACB0F94FF410E945F
:10F5B000FD6365CB8132910509F415C608F03EC0A4
:10F5C0008E31910509F4FFC568F48C31910509F479
:10F5D000F2C54D9709F03CCB80911B1B8E7F809329
:10F5E0001B1B4DCB8F31910509F401C6809709F0A3
:10F5F0002FCB80911B1B82FD0E9428F780911B1B43
:10F6000083FF3DCB60E080E50F94D942182F682F2F
:10F6100080917008909171080F942F2D83E50F94BD
:10F62000B542882321F00F94FF410E94FD630E94A0
:10F630009CE2111124CB0F94D64C21CB8B34910535
:10F6400009F4F8C5B0F48033910509F4EFC58934A5
:10F65000910509F0FDCA80E50F946742882309F4FB
:10F660000ECB0F940F42853608F084E68093030991
:10F6700006CB8C34910509F4E1C58D34910509F070
:10F68000E7CA0F94E94CFBCA8D36910509F49CC674
:10F6900008F08AC08C35910511F40C94788308F039
:10F6A00042C08335910511F40C946C8380F481354C
:10F6B000910511F40C944F838235910509F0C8CA65
:10F6C0008091910C8F7D80618093910CD8CA843594
:10F6D000910511F40C9474838535910509F0B8CA2D
:10F6E00083E50F946742882309F4C9CA0F94AFA237
:10F6F00060937C0C70937D0C80937E0C90937F0CB8
:10F700000F94374220E030E04AE754E40F9453BEB0
:10F710000F9452C660933A0770933B0780933C075F
:10F7200090933D07ACCA8A36910509F4ABC698F5AB
:10F730008836910509F419C68936910509F088CAF9
:10F740000E94673B182F87FD0AC08FE99EE00F9447
:10F75000BB4F812F0F94C72E8AE00F94304F2CA9F6
:10F760002093850CE5960FB6F894DEBF0FBECDBF93
:10F77000DF91CF911F910F91FF90EF90DF90CF908D
:10F78000BF90AF909F908F907F906F905F904F90C1
:10F790003F902F9008958B36910509F4AEC68C36B4
:10F7A000910509F46CCA54CA8337910511F40C947D
:10F7B000198408F05DC08037910509F460CA08F02B
:10F7C00048C08E36910509F4A7C68F36910509F019
:10F7D0003FCA83E50F946742882331F060E083E5F8
:10F7E0000E94143B809388140F94DC5B80EB9EE0B6
:10F7F0000F94BB4F80918814882309F4A0C610E0B1
:10F8000000E020E08091881490E0B0E0A0E0002EBD
:10F8100004C0B695A795979587950A94D2F780FF6F
:10F8200012C0FF24F394F20E222319F08CE20F94FD
:10F83000304FF801EE0FFF1FEA55F14F859194917B
:10F840000F94BB4F2F2D0F5F1F4F05301105D1F6C1
:10F850007FC48137910509F475C68237910509F097
:10F86000F7C90F9416988BEA9AE10E94A8F107CA8B
:10F870008737910511F40C94488470F5853791050C
:10F8800009F4DBC78637910509F0E2C900917008D9
:10F890001091710894E0F12C40E0915009F4E7C711
:10F8A000F8018081282F2B7F213409F0D9C72181CD
:10F8B000213309F0DCC7813409F4E7C7853409F442
:10F8C00041E098012E5F3F4F89012F5F3F4FF801C4
:10F8D00080818032C9F3E1CF8837910509F4DCC714
:10F8E0008937910509F0B4C91092E20B1092E10B2F
:10F8F0000F94E71CC4C98239E1E09E0711F40C940F
:10F90000248808F040C18C3D910511F40C94AA851F
:10F9100008F0CAC0893C910511F40C94C18408F028
:10F9200075C08B39910509F493C6B8F48C389105EC
:10F9300009F42AC68139910509F08AC970E060E0AE
:10F9400083E50F94EE42823008F4AFC70F94D15391
:10F9500080EF9EE00F94BB4F92C98E3B910509F456
:10F9600039C6883C910509F073C90E94673B182F7E
:10F9700087FD85C90091B00C84E40F94B542B82E80
:10F980008823D9F10F9437426B017C0120E030E0ED
:10F99000A9010F94EDBD882311F40C94BF8424E0D9
:10F9A0001202F0011124E455F34FC082D182E282A9
:10F9B000F38220E030E0A901C701B6010F943FC7F0
:10F9C0001816D4F420E030E040E05FE3C701B60150
:10F9D0000F9453BE9B01AC010F9453BE2BED3FE03F
:10F9E00049E450E40F9453BE60930D0270930E02ED
:10F9F00080930F02909310020B2D602F83E50F94DC
:10FA0000D9428093B00C0E94C3DD39C98D3C910569
:10FA100011F40C945685E0F58B3C910509F4DBC795
:10FA20008C3C910509F014C98091590787FF02C0E9
:10FA30000C940E8580915A078E7011F00C940E85EF
:10FA40004091BD145091BE146091BF147091C014C8
:10FA500085E19FE00F9478524091C1145091C214F7
:10FA60006091C3147091C41482E19FE00F947852A6
:10FA70004091C5145091C6146091C7147091C81478
:10FA800083E792E30F9478528AE00F94304FF7C8DF
:10FA90008E3C910511F40C945A85833D910509F033
:10FAA000D7C80E94C06CEBC88D3221E0920711F4D8
:10FAB0000C94E48608F044C08831A1E09A0711F460
:10FAC0000C944486F0F48D3D910511F40C94ED8571
:10FAD0008A3F910509F0BCC883E40F9467428823EC
:10FAE00021F00F9433420E94295160915502709188
:10FAF000560283E89FE00F9499528AE00F94304FAA
:10FB0000BEC88232E1E09E0711F40C94E0868C328C
:10FB1000914009F09DC864E071E083E50E94203BBC
:10FB20008C0168EE73E080E50E94203B893823E178
:10FB3000920710F088E893E1B8010E94B6B09FC820
:10FB4000803321E0920711F40C94668768F48E32BA
:10FB5000A1E09A0711F40C94DA878F32914009F0F2
:10FB600077C80E94EE658BC88039E1E09E0711F4EA
:10FB70000C9420888139914009F06AC80F9406439B
:10FB80000F94C11B7CC88C3022E0920711F40C94B6
:10FB9000CD8808F002C1863EA1E09A0711F40C94CA
:10FBA000498808F0C6C0843AE1E09E0711F40C943D
:10FBB0002C88B8F48A3921E0920709F460C88D399D
:10FBC000914009F045C883E50F946742882311F4FA
:10FBD0000C94388A0F9423428093D3090F943A40AF
:10FBE0004EC8853AA1E09A0711F40C9430888C3AFB
:10FBF000914009F02DC887E00F94BE3981113FC8AC
:10FC00007CE3C72E7DE2D72E87E89DE099A788A7E1
:10FC1000DE0111961D017D0110E000E0C6010E9489
:10FC2000E865E8A5F9A581909190A190B190F9A718
:10FC3000E8A7A50194010F94DEC42B013C01D70174
:10FC40004D925D926D927C92139720E030E040EAF5
:10FC500051EC0F943FC787FD0AC020E030E040EA36
:10FC600051E4C301B2010F94EDBD18167CF4F80104
:10FC7000E05AF24DE4911E164CF4B7FAB094B7F87E
:10FC8000B094F70180829182A282B382D7018D90D5
:10FC90009D90AD90BD907D0120E030E040EA51ECB8
:10FCA000C501B4010F943FC787FF02C00C9434888C
:10FCB00020E030E040EA51E4C501B4010F94EDBD0D
:10FCC000181614F40C9434880F5F1F4FB4E0CB0E59
:10FCD000D11C0330110509F0A1CF6DEBE62E6CE0CD
:10FCE000F62E10E0F10181919191A191B1911F0146
:10FCF000F70181939193A193B1937F01812F0F9489
:10FD0000C60A1F5F133071F70F94C11B60E081ECCE
:10FD10009FE00E94764663E972E084E690E00E94EC
:10FD2000B6B06AEB72E084E690E00E94B6B00C9444
:10FD30003F76863FE1E09E0711F40C94BF8878F48B
:10FD4000843F21E0920711F40C94BB88853F9140D9
:10FD500011F00C9428760F94A8390C943F76873FC5
:10FD6000A1E09A0711F40C94C388883F914011F0E8
:10FD70000C94287681E08093D5090F949C391092D9
:10FD8000D509882311F40C943F760F94DC5B8DEF3A
:10FD90009FE00F94BB4F0C943F768C36E3E09E07B8
:10FDA00011F40C943F7608F091C08D3B22E092074D
:10FDB00011F40C94F88808F07AC08835A2E09A070C
:10FDC00011F40C94DE888B35924011F00C94287657
:10FDD0000E94673B082F87FF02C00C943F7685E5A1
:10FDE0000F946742882369F10F9437424B015C01FD
:10FDF000E02E002E000CFF0820E030E0A9010F9457
:10FE00003FC787FF04C0B7FAB094B7F8B09420E0BA
:10FE100030E84BE354E4C501B4010F943FC79701A8
:10FE200053E0220F331F5A95E1F72553364F18162A
:10FE300014F40C94E288D9018D929D92AD92BC92FB
:10FE400013978CE40F946742882311F40C943F7647
:10FE50000F9437426B017C01002E000C110B20E047
:10FE600030E0A9010F943FC787FF04C0F7FAF09470
:10FE7000F7F8F09420E030E84BE354E4C701B60112
:10FE80000F943FC7980143E0220F331F4A95E1F7D3
:10FE90002553364F181614F40C94ED88D901149696
:10FEA000CD92DD92ED92FC9217970C943F768E3BAB
:10FEB000E2E09E0711F40C94FC888335934011F026
:10FEC0000C9428760E94E36A0C943F76873E23E0E8
:10FED000920711F40C94288AC8F48438A3E09A0796
:10FEE00011F40C94BD89803A934011F00C9428765B
:10FEF000209170083091710890911B1B9260909333
:10FF00001B1BC9010E9448EE0C943F76883EE3E03B
:10FF10009E0711F40C944E8A893E934011F00C9484
:10FF200028760F9471AE81110C943F760F94324075
:10FF30000F9429AE0F947C226D33710581059105D4
:10FF400020F08AE690E10E94E38A86E690E10E9432
:10FF5000E38A84EE8093030982E590E10F94BB4F1E
:10FF60008EE490E10E94E38A0C943F7660E086EA9A
:10FF70009DE00E947646A3CA8091580784FD17C071
:10FF800080915A0787FD13C080915B07837079F4D5
:10FF900060E089EB9DE00E9476465F988A988091A8
:10FFA000080181708093060112980C943F7688E5D1
:10FFB0000F94674281115F9889E50F946742811120
:10FFC0008A988AE50F946742882329F08091080176
:10FFD00081708093060185E40F946742882311F4B1
:10FFE0000C943F7612980C943F760F94DC5B82EE73
:10FFF0009DE00F94BB4F0C943F760E94AFEA0C94A7
:020000021000EC
:100000003F7680911B1B82FF02C00C943F760E94BA
:100010009EEA0C943F7660E00F942F2D1092030916
:100020000C943F7683E50F94B542882321F00F941A
:10003000FF410E94FD6384E50F94B5428823A9F037
:100040000F94FF416B017C010F942323C09232096E
:10005000D0923309E0923409F0923509CD28CE28A8
:10006000CF2819F081E0809336098091EC0988232C
:10007000F9F080E090E0A0EAB1E489839A83AB8351
:10008000BC831C8E1D8E1E8E1F8E18A219A21AA252
:100090001BA210E000E020E0AE014F5F5F4FBE0109
:1000A000645E7F4FCE0180960F9445650C943F7639
:1000B0000F94B24C882381F00E949CE20F94D64C9E
:1000C00087E09DE00E943DEA1092BC151092BD159C
:1000D0001092BE151092BF1561E085E598E10F946E
:1000E000C94F40E158E16CEE7DE085E00F94059A40
:1000F00080E00E9412470C943F760E94D7410C94F6
:100100003F7683E40F946742882361F182E09EE0AA
:100110000F94BB4F8091831C8823F9F0BE016F5F61
:100120007F4F80E89CE10E94D0E9CE0101960F94B8
:10013000A428CE0101960F9443AE809147178823DF
:1001400039F080E20F94304F87E497E10F94A428B0
:100150008AE00F94304F0C943F7688EF9DE00F9427
:10016000BB4FF6CF83E50F94B542882301F10F947E
:100170000F42182F8C3308F08CE3809334070F94D0
:10018000AFA26B017C01212F30E0A8EEB3E00F9409
:1001900085C4C60ED71EE81EF91EC0923007D09245
:1001A0003107E0923207F09233070C943F760F94B8
:1001B000CAAE0C943F7680917008909171080E94AD
:1001C00048EE0C943F7680911B1B83FD02C00C947B
:1001D0003F760F94D49880917008909171080E9496
:1001E000E0ED0C943F760E9483710C943F760F945F
:1001F0007C226C8F7D8F8E8F9F8FBE016F5F7F4FB4
:10020000CE014C960E941E63CE0101960F949486F7
:100210000F94DC5BBE016F5F7F4F81E19EE00F9426
:10022000C7538AE00F94304F0C943F760E94AF6D15
:100230000C943F760F94D64C0C943F760F94762313
:100240000C943F7670E060E083E50F94EE428E34CC
:10025000910539F40E9446F680E00E9412470C9402
:100260003F768CE79EE00F94BB4F6091D10B70916D
:10027000D20B83E79EE00F946E526091D30B709186
:10028000D40B86E69EE00F946E526091D10B709174
:10029000D20B8091D30B9091D40B681B790B80917A
:1002A0003609815021E030E0823010F030E020E06B
:1002B000621B730B8BE59EE00F946E528AE00F94E5
:1002C000304F83E59EE00F94BB4F8091D50B90910A
:1002D000D60BA091D70BB091D80B8C8F9D8FAE8F82
:1002E000BF8FBE016F5F7F4FCE014C960E941E6391
:1002F000BE016F5F7F4F86E49EE00F94C7538091ED
:10030000D90B9091DA0BA091DB0BB091DC0B8C8FA9
:100310009D8FAE8FBF8FBE016F5F7F4FCE014C961A
:100320000E941E63BE016F5F7F4F86E39EE00F94C5
:10033000C75320E030E04AE754E46091DD0B709150
:10034000DE0B8091DF0B9091E00B0F94D9C5AB01D0
:10035000BC018EE19EE00F9478528DE60F94304FF1
:100360008AE00F94304F0C943F768091881483FF7D
:1003700002C00C943F760E94673B87FF02C00C943A
:100380003F7689E40F94B542882311F40C946D8A6A
:100390000F940F4290E01816190614F481E090E0D3
:1003A00026E0289FF001299FF00D1124E55DF34F11
:1003B000808191810E94AAF661E080E00F9427B1CC
:1003C0000F9441B10C943F768091881483FF02C052
:1003D0000C943F760E94673BF82E87FF02C00C9476
:1003E0003F7689E40F94B542882311F40C94788AFF
:1003F0000F940F4290E01816190614F481E090E073
:1004000026E0289FF001299FF00D1124E55DF34FB0
:100410008081918110E00E94AAF661E081E00F9452
:1004200027B12091FB193091FC198091F919909115
:10043000FA1982179307F4F48FE89EE09F938F9345
:100440008AE99EE09F938F931F920E945B460F90D4
:100450000F900F900F900F9001E00F9441B1002387
:1004600011F40C943F7640E0612F8F2D0F94C13032
:100470000C943F7684E89EE0112301F3012FEDCF29
:1004800010E0EBCF60E080E50E94143BF82E31E0F5
:10049000381710F40C943F7681E40F946742609112
:1004A000C40D062F10E0811102C00FEF10E089E4A7
:1004B0000F94B542882311F40C948A8A0F940F424A
:1004C00090E01816190614F481E090E026E0289FC9
:1004D000F001299FF00D1124E55DF34F0481158192
:1004E000EF2DF0E0EC53F24F0F3F110519F010F033
:1004F0000FEF10E000830C943F7660E080E50E94EF
:10050000143B823010F00C943F76E82FF0E0EC536F
:10051000F24F10820C943F768EE40F94B5428823FC
:1005200011F40C943F760F94FF416093551570932E
:10053000561580935715909358150C943F7682EA80
:100540009EE00DCE83E50F94B542882369F00F94A9
:100550000F428D3320F480930C020C943F768CE391
:1005600080930C020C943F760F94DC5B10910C028C
:1005700087EB9EE00F94BB4F812F0F94B0AC8AE0C5
:100580000F94304F0C943F768091881483FF02C003
:100590000C943F7689E40F94B542882309F4C6C7CA
:1005A0000F940F4290E01816190614F481E090E0C1
:1005B00026E0289FF001299FF00D1124E55DF34FFF
:1005C000828193810F94274061E080E00F9427B1EE
:1005D0000C943F768091881483FF02C00C943F7680
:1005E00089E40F94B542882309F4AAC70F940F42F7
:1005F00090E01816190614F481E090E026E0289F98
:10060000F001299FF00D1124E55DF34F8281938164
:1006100010E00F94274060E081E00F9427B1209113
:100620009D0C30919E0C80919B0C90919C0C82179C
:1006300093071CF48DEC9EE002C08EEB9EE060E020
:100640000E94764660E0812F0F943A2F0C943F76FB
:1006500083E50F94B542882311F40C943F760F94F0
:100660000F42182F8C3308F08CE3809339070F94D6
:10067000AFA26B017C01212F30E0A8EEB3E00F9414
:1006800085C4C60ED71EE81EF91EC0923507D0924B
:100690003607E0923707F09238070C943F760E94B5
:1006A000DBEE0E9439F70F94E94C0F94EC4C10925A
:1006B000900C10928F0C10928E0C68EE73E080E01C
:1006C00090E00F94554C0F94F14C60E08CED9EE05F
:1006D0000E9476460C943F768091910C8F7E8062CA
:1006E0008093910C0C943F760E948C3B0C943F7647
:1006F0000E94673B87FF02C00C943F7680915807A9
:1007000084FD09C080915A0787FD05C080915B0771
:10071000837009F489C0FDEBCF2EF2E0DF2EA9E84B
:10072000EA2EA4E1FA2E10E0D6018D916D010F940E
:10073000B542882309F465C0133009F06DC00F94E9
:1007400037424B015C0120E030E040EA51E40F9475
:10075000EDBD87FF4EC0A50194016091A914709171
:10076000AA148091AB149091AC140F94D9C52B01AD
:100770003C01AC019B016091B80D7091B90D809165
:10078000BA0D9091BB0D0F9453BE6093B80D70934A
:10079000B90D8093BA0D9093BB0DA30192016091A6
:1007A000B9147091BA148091BB149091BC140F9439
:1007B00053BE6093B9147093BA148093BB14909392
:1007C000BC146091A40D7091A50D8091A60D90911F
:1007D000A70D0F94F2BDA30192010F9453BE0F9485
:1007E00052C66093A40D7093A50D8093A60D9093AF
:1007F000A70D8092A9149092AA14A092AB14B09263
:10080000AC141F5FF4E0EF0EF11C143009F08CCF34
:100810000E9404F70C943F760F943742F701648BE3
:10082000758B868B978BEDCF81E00F947B980C9422
:100830003F760E942C380C943F76809170089091FE
:100840007108009741F0DC012C91222321F00F94D4
:1008500094860C943F7680E00E9412470C943F7679
:10086000803529F4818180538A3008F42AC84111E7
:100870000F94DC5BFF2021F08DEE9EE00F94BB4FC8
:10088000C8010E94D7650C943F76FF24F39419C8E1
:100890000F94A31C0C943F7681E08093E20B80932D
:1008A000E10B0F94E71C0C943F768C01112788E430
:1008B0000F94B5428823C1F00F9433428A3A9105D0
:1008C0000CF44BC00F943342843B91400CF048C071
:1008D0000F94334226E0209FF001219FF00D112458
:1008E000E55DF34F9183808382E40F94B5428823C2
:1008F000A9F00F9433420597B4F10F9433428D3829
:100900009105A4F50F94334226E0209FF001219F2A
:10091000F00D1124E55DF34F9383828386E40F94F9
:10092000B542882311F40C943F760F94334297FD1F
:1009300020C00F9433428F3F910509F0ECF40F94DF
:10094000334226E0209FF001219FF00D1124E55D48
:10095000F34F958384830C943F768AEA90E0BACF74
:1009600083EB91E0B7CF85E090E0CECF8CE890E0CC
:10097000CBCF90E080E0E5CF8FEF90E0E2CF80E05A
:1009800040C80E94673B87FF02C00C943F760DEB86
:1009900012E079E8E72E74E1F72EE1ECCE2EE2E0EA
:1009A000DE2ED8018D918D010F946742882359F076
:1009B0000F9437420F9452C6F7016083718382838C
:1009C00093830E94B6F6F4E0EF0EF11CC016D10638
:1009D00041F70C943F760E94673B87FF02C00C945E
:1009E0003F766DEBE62E62E0F62E10E000E0D701D8
:1009F0008D917D010F946742882349F00F9437420F
:100A0000F801E757FB4E64A375A386A397A30C5F79
:100A10001F4F0031110559F70C943F7683E50F9471
:100A2000B542882391F00F9437426093BD147093C0
:100A3000BE148093BF149093C0146093C514709338
:100A4000C6148093C7149093C81480E50F94B542E0
:100A5000882351F00F9437426093BD147093BE14F5
:100A60008093BF149093C01482E50F94B5428823FD
:100A700051F00F9437426093C1147093C214809365
:100A8000C3149093C41484E50F94B542882311F4E1
:100A90000C943F760F9437426093C5147093C6143C
:100AA0008093C7149093C8140C943F760E94053C21
:100AB0000C943F765DEBE52E5CE0F52E10E088E5CA
:100AC000810F0F946742882351F00F943742F7014A
:100AD0006083718382839383812F0F94C60A1F5F83
:100AE000F4E0EF0EF11C133051F780915A0787FFA5
:100AF00002C00C949F7980915B07837011F00C9475
:100B00009F794091BD0C5091BE0C6091BF0C7091CB
:100B1000C00C85E29FE00F9478524091C10C509137
:100B2000C20C6091C30C7091C40C83E89DE60F94D5
:100B300078524091C50C5091C60C6091C70C7091D1
:100B4000C80C80E89DE60F9478528AE00F94304FED
:100B50000C943F7682E40F946742882341F08091A1
:100B6000810290918202909312028093110282E599
:100B70000F946742882341F08091110290911202F4
:100B8000909382028093810283E50F94B54288237B
:100B900031F00F94334290938202809381028091CE
:100BA000580790915907A0915A07B0915B07892B7C
:100BB0008A2B8B2B11F00C943F76609181027091FF
:100BC00082028CE29FE00F94995285E20F94304F9D
:100BD0008AE00F94304F0C943F760E94673B082FB9
:100BE00087FF02C00C943F7683E50F94B542002E38
:100BF000000C110B7801EE0CFF1C882359F10F94A7
:100C00003342F701E75CFD4F91838083000F111F92
:100C1000000F111F980125573D4F7901BC01990F15
:100C2000880B990B0F94F4BD2AE037ED43E25CE3A7
:100C30000F9453BE025D164FD8012D913D914D91F9
:100C40005C910F9453BEF701608371838283938319
:100C50000C943F760F94DC5B85E40F94304F80E377
:100C6000800F0F94304FF701E75CFD4F6081718179
:100C700080E39FE00F94995285E20F94304F8AE011
:100C80000F94304F0C943F7680E50F946742882391
:100C900011F40C943F760F9433428C01892B09F0A8
:100CA00082C083E50F946742882391F00F9433420A
:100CB0008F3F980731F485E89AE10F94F64C0C9435
:100CC0003F76BC0185E89AE10F94644D0C943F7621
:100CD0000F94DC5B70E060E08BE39FE00F9499522F
:100CE0008091871A08E5C02E02E0D02EC81AD108DC
:100CF00087FDD394CC0CDD1CCC0CDD1C0D2C000C22
:100D0000EE08FF088091861A98E8892E912C881A9F
:100D1000910887FD9394880C991C880C991C092CC8
:100D2000000CAA08BB088091851A90E08F3FC9F19A
:100D3000FC01EE0FFF1FE80FF91FE45CF54E818107
:100D40009281B3E0880F991FBA95E1F7B0E0A0E077
:100D500014E0B595A795979587951A95D1F70296C2
:100D60009C012F5F3F4F032E000C440B550B28199D
:100D700039094A095B09A4EBB0E00F9472C4A701DA
:100D80009601281939094A095B090F9453C4B9011E
:100D900088E39FE00F9499528AE00F94304F0C94AF
:100DA0003F7680E0DDCF0F94D153B80182E59FE01C
:100DB0000F94995283E49FE00F94BB4F0C943F76BD
:100DC0000E94256C0C943F7660E085E40E94143B01
:100DD000811174C080E50F946742882351F00F940D
:100DE00037426093FE197093FF198093001A909315
:100DF000011A89E40F946742882381F00F943742E7
:100E00002CEA35EC47E25EE30F9453BE6093021A7E
:100E10007093031A8093041A9093051A84E40F9434
:100E20006742882381F00F9437422CEA35EC47E281
:100E30005EE30F94D9C56093061A7093071A8093E6
:100E4000081A9093091A0F94DC5B4091FE19509197
:100E5000FF196091001A7091011A81E69FE00F94CA
:100E600078522CEA35EC47E25EE36091021A709109
:100E7000031A8091041A9091051A0F94D9C5AB01F9
:100E8000BC018DE59FE00F9478522CEA35EC47E2E7
:100E90005EE36091061A7091071A8091081A90918A
:100EA000091A0F9453BEAB01BC0189E59FE00F9472
:100EB00078528AE00F94304F0C943F760F94D153C0
:100EC00085E69FE00F94BB4F0C943F7680E50F942E
:100ED0006742882351F00F9437426093A00C7093BF
:100EE000A10C8093A20C9093A30C89E40F94674209
:100EF000882381F00F9437422CEA35EC47E25EE319
:100F00000F9453BE6093A40C7093A50C8093A60C11
:100F10009093A70C84E40F946742882381F00F9488
:100F200037422CEA35EC47E25EE30F94D9C5609373
:100F3000A80C7093A90C8093AA0C9093AB0C0F94FF
:100F4000DC5B4091A00C5091A10C6091A20C7091BF
:100F5000A30C8FE79FE00F9478522CEA35EC47E220
:100F60005EE36091A40C7091A50C8091A60C909109
:100F7000A70C0F94D9C5AB01BC018BE79FE00F9480
:100F800078522CEA35EC47E25EE36091A80C709150
:100F9000A90C8091AA0C9091AB0C0F9453BEAB019D
:100FA000BC0187E79FE00F9478528AE00F94304F9E
:100FB0000C943F7683E50F946742182F882369F0DD
:100FC0000F9433429C019093900280938F0291E0A2
:100FD000232B09F090E09093D60D80E50F946742A3
:100FE000882361F020918F0230919002232B11F021
:100FF0000F9423428093D60D0C943F7611110C94DC
:101000003F760F94DC5B8EEA9FE00F94BB4F80919C
:10101000D60D882391F086E99FE00F94BB4F609135
:101020008F02709190028DE99FE00F94995289E9A7
:101030009FE00F94BB4F0C943F7682E99FE0EDCF89
:101040000E9428F70C943F760F94FD420F940F43B3
:101050000F94C11B0C943F760E94FF720C943F7654
:101060000E9448720C943F760F94D1538FED9FE00D
:101070000F94BB4F61E081ED9FE00E9476460E9495
:101080004C4468E270E088EC90E00E94B6B00C94AA
:101090003F7684E50F9467428823A1F010921409EB
:1010A000109215091092160910921709109218093A
:1010B0008FEF0F94014161E070E084E50F94EE4200
:1010C0008093180983E50F946742882321F00F94D9
:1010D00033420F94014183E40F946742882331F037
:1010E00080912002803210F40F94D54080E50F9457
:1010F0006742882331F00F943342803210F40F940A
:10110000D54085E50F946742882311F40C943F760F
:101110000F943342803210F00C943F7641E050E05F
:1011200060E070E0082E04C0440F551F661F771F53
:101130000A94D2F7409550956095709500911409E6
:101140001091150920911609309117094023512358
:101150006223732340931409509315096093160971
:10116000709317099091200289130C943F76109286
:1011700087140C943F760E94E6F20C943F760F940D
:10118000F61C0C943F7661E083E50F94D94291E020
:1011900089270F9451320C943F7680911B1B82FF5C
:1011A00005C0806480931B1B0C943F7683FD02C0B6
:1011B0000C943F760F94D4980C943F760E94C740CD
:1011C0000C943F7680E090E8ABE3B4E4F9018083CF
:1011D0009183A283B3830C94217F80E090E8ABE3FA
:1011E000B4E4F90184839583A683B7830C943F7696
:1011F0000E94A6440C943F760E94673B182F87FFFD
:1012000002C00C943F768AE50F94B542812C912C54
:1012100090E2A92E91E4B92E882341F040E050E0FD
:10122000BA018AE50F94C2424B015C01412F64E090
:1012300083E00E9465C720E030E0A901C501B40148
:101240000F943FC718167CF580E090E0A0EAB0E468
:1012500089839A83AB83BC8320918F0D3091900D4D
:101260004091910D5091920DC501B4010F94DFC4CE
:101270006B017C0120E030E04AE753E40F94EDBDC0
:1012800087FD06C0C12CD12C8AE7E82E83E4F82E16
:10129000CC8EDD8EEE8EFF8EBE016F5F7F4FCE0156
:1012A0004C960F94F11585E50F946742882309F455
:1012B00059C00F9437426B017C0120E030E0A90156
:1012C000C701B6010F943FC787FF04C0F7FAF09437
:1012D000F7F8F094F7FAF094F7F8F094C982DA820C
:1012E000EB82FC8244E061E0CE0101960F94A76698
:1012F00020E030E0A901C501B4010F943FC71816E2
:101300005CF580E090E0A0EAB0E489839A83AB8347
:10131000BC83A501940160918F0D7091900D809117
:10132000910D9091920D0F94DEC46B017C0120E031
:1013300030E0A9010F943FC718161CF0C12CD12C26
:101340007601CC8EDD8EEE8EFF8EBE016F5F7F4FFD
:10135000CE014C960F94F11510921A090E944C443C
:101360000C943F7628E01202F0011124E553F64F69
:10137000C080D180E280F380A0CFA090BC0DB0905F
:10138000BD0DC090BE0DD090BF0D8BE40F94B54243
:10139000882339F10F9437427B018C0120E030E043
:1013A000A9010F943FC787FD0AC020E030E040E26A
:1013B00051E4B701C8010F94EDBD1816A4F48FE3F2
:1013C0000F94304F8BE40F94304F83E190E10F94F2
:1013D000BB4F8BE090E10F94BB4F88E090E10F94FE
:1013E000BB4F750186019701A801B501C6010F9495
:1013F000EDBD882361F00E9428F7C701D8018093D2
:10140000BC0D9093BD0DA093BE0DB093BF0D809108
:10141000580790915907A0915A07B0915B07892B03
:101420008A2B8B2B11F00C943F760F94DC5B409150
:10143000BC0D5091BD0D6091BE0D7091BF0D87E246
:1014400090E10F9478528AE00F94304F0C943F76DD
:1014500081E080932A0C1092DF1760E083E50F94FF
:10146000D94281110C943F760F949F870C943F765C
:101470000F94DC5B89E390E10F94BB4F8091D3091B
:10148000882349F086E390E10F94BB4F8AE00F94E4
:10149000304F0C943F7682E390E1F6CF0E94558B5B
:1014A0000C943F7610916D080F94AFA260937C0C62
:1014B00070937D0C80937E0C90937F0C112311F41C
:1014C0000C943F76812F0E9491EE0C943F7611117F
:1014D0000C94DF7611E00C94DA7683E50F94B54234
:1014E000882311F40C94E0810F9433420C94DA8138
:1014F00083E50F94B542182F811108C082E50F943F
:10150000B542082F882311F40C9440820F94334283
:101510000C940B8283E50F94B542882311F40C944C
:1015200070820F94FF418B010C94708283E50F94BD
:10153000B542882311F40C943F760F94334242C88D
:1015400083E50F94B542182F811107C082E50F94EF
:10155000B542882311F40C943F760F94334259C856
:10156000882309F4B7CF0C94E276DF92EF92FF92D2
:101570000F931F93CF93DF93EC01E090870CF090D3
:10158000880C8AE0D82E6AE070E0CE010F9480C902
:101590008C01009711F0FC011082CE010E945F6463
:1015A00081E00E946A740115110519F0E801D992D1
:1015B000EACFC701DF91CF911F910F91FF90EF907C
:1015C000DF900C945F644F925F926F927F928F9244
:1015D0009F92AF92BF92CF92DF92EF92FF920F93C2
:1015E0001F93CF93DF93CDB7DEB77C014DB65EB6C8
:1015F0006090870C7090880C8DB69EB66AE070E0A3
:10160000C7010F94EBBC6C018C010E191F09892BCB
:1016100021F4C7010F94FDBC8C01C80101962DB7C0
:101620003EB7281B390B0FB6F8943EBF0FBE2DBF37
:101630008DB79EB701965C01A801B7010F941EBD3E
:10164000F501E00FF11F1082C5010E945F6481E087
:101650000E946A74C114D10451F076019FEFE91A17
:10166000F90A0FB6F8949EBE0FBE8DBEC5CF0FB659
:10167000F8949EBE0FBE8DBEC3010E945F640FB67C
:10168000F8945EBE0FBE4DBEDF91CF911F910F91BA
:10169000FF90EF90DF90CF90BF90AF909F908F9092
:1016A0007F906F905F904F9008954F925F926F92EE
:1016B0007F928F929F92AF92BF92CF92DF92EF92E2
:1016C000FF920F931F93CF93DF93CDB7DEB7C0592F
:1016D000D1090FB6F894DEBF0FBECDBF0F944840BE
:1016E000882369F083E50F946742882301F120E0A5
:1016F00040E070E060E083E292EA0E94C943C05794
:10170000DF4F0FB6F894DEBF0FBECDBFDF91CF9194
:101710001F910F91FF90EF90DF90CF90BF90AF900F
:101720009F908F907F906F905F904F90089583E48B
:101730000F946742882319F00E9418A2E0CF80908E
:10174000700D9090710DA090720DB090730D8091FE
:10175000790D80FF05C0909188149860909388144B
:10176000869581708093D60D8BE09DE00E94E38A80
:101770008091FF0C9091000D9E012F5F3F4F7901EA
:10178000009799F09F938F9382E09DE09F938F93B2
:101790003F932F930F9484BDC7010E94B58A0F9089
:1017A0000F900F900F900F900F908091FD0C9091E3
:1017B000FE0C009799F09F938F9389EF9CE09F9385
:1017C0008F93FF92EF920F9484BDC7010E94B58A58
:1017D0000F900F900F900F900F900F906E0131E8C7
:1017E000C30ED11C6091DC0C7091DD0C8091DE0C7D
:1017F0009091DF0C860123E041E00F947DB89F9328
:101800008F9387EE9CE09F938F93FF92EF920F94BC
:1018100084BDC7010E94B58A8FED9CE00E94E38AD7
:1018200087E08093E40B80932D090F900F900F9029
:101830000F900F900F908091F80C8823F9F0609131
:10184000F90C7091FA0C8091FB0C9091FC0C23E048
:1018500041E00F947DB89F938F9386ED9CE09F931A
:101860008F93FF92EF920F9484BDC7010E94B58AB7
:101870000F900F900F900F900F900F908091010D8F
:101880008823A1F01F928F931F921F9289EC9CE0F6
:101890009F938F93FF92EF920F9484BDC7010E9494
:1018A000B58A0FB6F894DEBF0FBECDBF8091020D92
:1018B0008823A9F01F928F931F9281E08F9389EC68
:1018C0009CE09F938F93FF92EF920F9484BDC7018A
:1018D0000E94B58A0FB6F894DEBF0FBECDBF409010
:1018E000030D5090040D6090050D7090060D20E0E2
:1018F00030E0A901C301B2010F94EDBD811104C014
:101900008091790D82FF20C0860121E041E0C30172
:10191000B2010F947DB89F938F938091790D82FBD4
:10192000882780F91F928F938CEB9CE09F938F9375
:10193000FF92EF920F9484BDC7010E94B58A0FB643
:10194000F894DEBF0FBECDBF6091CE0C7091CF0C6E
:101950008091D00C9091D10C8E010F581F4F23E035
:1019600041E00F947DB8782E692E6091CA0C709179
:10197000CB0C8091CC0C9091CD0C860123E041E002
:101980000F947DB86F927F929F938F938BEA9CE028
:101990009F938F93FF92EF920F9484BDC7010E9493
:1019A000B58A6091D20C7091D30C8091D40C909137
:1019B000D50C23E041E00F947DB880EA9CE00E94C2
:1019C000E38ADF92CF9286E99CE09F938F93FF9208
:1019D000EF920F9484BDC7010E94B58A8091DB0C01
:1019E0008F938091DA0C8F938FE89CE09F938F9375
:1019F000FF92EF920F9484BDC7010E94B58A609157
:101A0000D60C7091D70C8091D80C9091D90C23E012
:101A100041E00F947DB89F938F9385E89CE09F935E
:101A20008F93FF92EF920F9484BDC7010E94B58AF5
:101A30008CE0E0EEFCE0ADEBBCE001900D928A950D
:101A4000E1F78CE0ECEEFCE0A1EBBCE001900D9244
:101A50008A95E1F780E00F94C60A81E00F94C60AE8
:101A600082E00F94C60A8091780D8093910C81E0FA
:101A70008093D3090F943A4087E09DE09F938F9322
:101A800080ED9DE39F938F93FF92EF920F9484BD1F
:101A90000FB6F894DEBF0FBECDBFC7010E94B58A56
:101AA0008091770D8F938091760D8F938091750D36
:101AB0008F938091740D8F93BF92AF929F928F926C
:101AC00087E79CE09F938F93FF92EF920F9484BDE2
:101AD000C7010E94B58A0FB6F894DEBF0FBECDBF16
:101AE0000ECECF93DF93C091C115C093970D81E6C1
:101AF000C89FE0011124CD53DA4E8091881480FFF5
:101B000005C00F94DC5BCE010E94D765CE010E9418
:101B10005F6480E0DF91CF910C946A746091390228
:101B200070913A02072E000C880B990B0F94F4BDAC
:101B30002AE037ED43E25CE30F9453BE20912E0977
:101B400030912F0940913009509131090F9453BEC3
:101B500060938B0270938C0280938D0290938E021F
:101B60000895E0915A0CE23030F4F0E0EC53F24F7B
:101B70008091480C808308958091101B8823C1F0C8
:101B800081508093101BECE3FBE1882351F08150DE
:101B9000990B2BE1289FF001299FF00D1124EE589D
:101BA000F44E8BE1A7E5BBE101900D928A95E1F738
:101BB0002091101B211105C080911B1B8062809316
:101BC0001B1B81E090E0A0E0B0E0211103C080E0A9
:101BD00090E0DC018093400C9093410CA093420C68
:101BE000B093430C1092450C81E080933F0C83E04E
:101BF00080937F0208950E944C4488EF93E2909373
:101C0000E80B8093E70B0895CF93DF93EC01CB01B2
